:020000040800F2
:1000000000060020E1010008E3010008E301000808
:10001000E3010008E3010008E3010008E301000830
:10002000E3010008E3010008E3010008652F000870
:10003000E3010008E3010008E3010008E301000810
:10004000E3010008E3010008E3010008E301000800
:10005000E3010008E30100080D3200083532000812
:100060005D32000885320008AD320008E301000867
:10007000E3010008E3010008E3010008E3010008D0
:10008000E3010008E3010008E3010008E3010008C0
:10009000E3010008E3010008E3010008D53200088D
:1000A000E3010008E3010008E3010008E3010008A0
:1000B000A9330008E3010008E3010008E301000898
:1000C000E3010008E3010008E3010008E301000880
:1000D000E3010008E3010008E3010008E301000870
:1000E00039330008E3010008E3010008E3010008D8
:1000F000E3010008E3010008E3010008E301000850
:10010000E3010008E3010008E3010008E30100083F
:10011000E3010008E3010008E3010008E30100082F
:10012000E3010008E3010008E3010008E30100081F
:10013000E3010008E3010008E3010008E30100080F
:10014000E3010008E3010008E301000819270008A3
:10015000E3010008E3010008E3010008E3010008EF
:10016000E3010008E3010008E3010008E3010008DF
:10017000E3010008E3010008E3010008E3010008CF
:10018000E3010008E3010008E3010008E3010008BF
:10019000E3010008E3010008E3010008E3010008AF
:1001A000E3010008E3010008E3010008E30100089F
:1001B000E3010008E3010008E3010008E30100088F
:1001C000E3010008E3010008E3010008E30100087F
:1001D000E3010008E3010008E3010008E30100086F
:1001E00002E000F000F8FEE772B6374880F30888B6
:1001F000364880F3098836483649086040F20000E6
:10020000CCF200004EF63471CEF200010860BFF36C
:100210004F8FBFF36F8F40F20000C0F2F0004EF638
:100220008851CEF200010860BFF34F8FBFF36F8F8C
:100230004FF00000E1EE100A4EF63C71CEF20001E4
:100240000860062080F31488BFF36F8F01F02CFF45
:1002500002F026FE4FF055301F491B4A91423CBF29
:1002600041F8040BFAE71D49184A91423CBF41F896
:10027000040BFAE71A491B4A1B4B9A423EBF51F83E
:10028000040B42F8040BF8E700201849184A914281
:100290003CBF41F8040BFAE701F00AFF02F054FEFC
:1002A000144C154DAC4203DA54F8041B8847F9E7A7
:1002B00000F042F8114C124DAC4203DA54F8041B22
:1002C0008847F9E701F0F2BE000600200022002076
:1002D0000000000808ED00E00000002000060020FB
:1002E0006837000800220020402200204022002021
:1002F000602E0020E0010008E0010008E001000895
:10030000E00100082DE9F04F2DED108AC1F80CD066
:10031000C3689D46BDEC108ABDE8F08F002383F3CF
:1003200011882846A047002001F072FAFEE701F08C
:1003300001FA00DFFEE7000038B500F0BBFB01F07A
:1003400083FE054601F0A6FE0446C8B90E4B9D4249
:1003500018D001339D4218BF044641F2883504BFCE
:1003600001240025002001F079FE0CB100F074F8A2
:1003700000F000FD284600F0BFF800F06DF8F9E746
:100380000025EFE70546EDE7010007B008B500F0EE
:1003900063FBA0F120035842584108BD07B541F264
:1003A0001203022101A8ADF8043000F073FB03B082
:1003B0005DF804FB38B5302383F3118817480368D0
:1003C0000BB101F0F1FA164A144800234FF47A7188
:1003D00001F0E0FA002383F31188124C236813B173
:1003E0002368013B2360636813B16368013B63606A
:1003F0000D4D2B7833B963687BB9022000F024FCE3
:10040000322363602B78032B07D163682BB902205A
:1004100000F01AFC4FF47A73636038BD402200206C
:10042000B50300086023002058220020084B1870F4
:1004300003280CD8DFE800F008050208022000F0CD
:10044000F9BB022000F0ECBB024B00225A6070475F
:100450005822002060230020234B244A10B51C465C
:10046000196801313FD004339342F9D16268A24246
:1004700039D31F4B9B6803F1006303F540439A4255
:1004800031D2002000F030FB0220FFF7CFFF194BE4
:100490001A6C00221A64196E1A66196E596C5A6425
:1004A000596E5A665A6E5A6942F080025A615A6908
:1004B00022F080025A615A691A6942F000521A61A8
:1004C0001A6922F000521A611B6972B64FF0E023DC
:1004D0003021C3F8084DD4E9003281F311889D46DC
:1004E00083F30888104710BD00C0000820C0000832
:1004F00000220020003802402DE9F04F93B0AA4BB3
:1005000000902022FF210AA89D6800F0DDFBA74A89
:100510001378A3B9A648012103601170302383F337
:10052000118803680BB101F03FFAA24AA0480023EA
:100530004FF47A7101F02EFA002383F31188009BA7
:1005400013B19D4B009A1A609C4A009C1378032BB0
:100550001EBF00231370984A4FF0000A18BF536063
:10056000D3465646D146012000F064FB24B1924B9D
:100570001B68002B00F01182002000F06DFA039040
:10058000039B002BF2DB012000F04AFB039B213B85
:10059000162BE8D801A252F823F000BFF905000895
:1005A00021060008B5060008670500086705000871
:1005B000670500083F0700080F0900082908000820
:1005C0008B080008B3080008D90800086705000870
:1005D000EB080008670500085D0900089906000897
:1005E00067050008A109000805060008990600082B
:1005F000670500088B0800080220FFF7C7FE0028E7
:1006000040F0F581009B0221BAF1000F08BF1C46A3
:1006100005A841F21233ADF8143000F03BFAA2E71E
:100620004FF47A7000F018FA071EEBDB0220FFF798
:10063000ADFE0028E6D0013F052F00F2DA81DFE8A9
:1006400007F0030A0D10133605230593042105A8AE
:1006500000F020FA17E054480421F9E75848042133
:10066000F6E758480421F3E74FF01C08404600F035
:100670003DFA08F104080590042105A800F00AFAE3
:10068000B8F12C0FF2D1012000FA07F747EA0B0B63
:100690005FFA8BFB4FF0000900F062FB26B10BF014
:1006A0000B030B2B08BF0024FFF778FE5BE74648DF
:1006B0000421CDE7002EA5D00BF00B030B2BA1D10D
:1006C0000220FFF763FE074600289BD0012000F0C0
:1006D0000BFA0220FFF7AAFE00261FFA86F8404612
:1006E00000F012FA044690B10021404600F01CFAD6
:1006F00001360028F1D1BA46044641F21213022114
:1007000005A8ADF814303E4600F0C4F92BE70120EF
:10071000FFF78CFE2546244B9B68AB4207D9284641
:1007200000F0E4F9013040F067810435F3E7234B32
:1007300000251D70204BBA465D603E46ACE7002E9A
:100740003FF460AF0BF00B030B2B7FF45BAF022089
:10075000FFF76CFE322000F07FF9B0F10008FFF6E1
:1007600051AF18F003077FF44DAF0F4A926808EBC2
:10077000050393423FF646AFB8F5807F3FF742AF9F
:10078000124B0193B84523DD4FF47A7000F064F901
:100790000390039A002AFFF635AF019B039A03F8F2
:1007A000012B0137EDE700BF002200205C23002071
:1007B00040220020B50300086023002058220020BA
:1007C00004220020082200200C2200205C220020AD
:1007D000C820FFF7DBFD074600283FF413AF1F2DAD
:1007E00011D8C5F1200242450AAB25F0030028BF0D
:1007F000424683490192184400F040FA019A804829
:10080000FF2100F061FA4FEAA8037D490193C8F384
:100810008702284600F060FA064600283FF46DAFD4
:10082000019B05EB830537E70220FFF7AFFD0028AA
:100830003FF4E8AE00F0A4F900283FF4E3AE00274F
:10084000B846704B9B68BB4218D91F2F11D80A9B22
:1008500001330ED027F0030312AA134453F8203CAF
:1008600005934046042205A900F0AEFA04378046FD
:10087000E7E7384600F03AF90590F2E7CDF8148042
:10088000042105A800F006F906E70023642104A866
:10089000049300F0F5F800287FF4B4AE0220FFF7CF
:1008A00075FD00283FF4AEAE049800F051F90590B4
:1008B000E6E70023642104A8049300F0E1F800288F
:1008C0007FF4A0AE0220FFF761FD00283FF49AAE4E
:1008D000049800F04DF9EAE70220FFF757FD0028E1
:1008E0003FF490AE00F05CF9E1E70220FFF74EFD27
:1008F00000283FF487AE05A9142000F057F9042121
:100900000746049004A800F0C5F83946B9E732203C
:1009100000F0A2F8071EFFF675AEBB077FF472AEBB
:10092000384A926807EB090393423FF66BAE022008
:10093000FFF72CFD00283FF465AE27F003074F4476
:10094000B9453FF4A9AE484600F0D0F8042105901F
:1009500005A800F09FF809F10409F1E74FF47A7057
:10096000FFF714FD00283FF44DAE00F009F9002810
:1009700044D00A9B01330BD008220AA9002000F0C2
:10098000ABF900283AD02022FF210AA800F09CF9F8
:10099000FFF704FD1C4800F041FF13B0BDE8F08FE5
:1009A000002E3FF42FAE0BF00B030B2B7FF42AAE7F
:1009B0000023642105A8059300F062F8074600288B
:1009C0007FF420AE0220FFF7E1FC804600283FF4D0
:1009D00019AEFFF7E3FC41F2883000F01FFF0598E5
:1009E00000F0F0F9464600F0BBF93C46BBE5064690
:1009F00052E64FF0000905E6BA467EE637467CE649
:100A00005C22002000220020A086010070B50F4B60
:100A10001B780133DBB2012B0C4611D80C4D296831
:100A20004FF47A730E6AA2FB03320146224628462F
:100A3000B047844204D1074B00221A70012070BDD8
:100A40004FF4FA7000F0EAFE0020F8E710220020D0
:100A5000082600209423002007B500230246012128
:100A60000DF107008DF80730FFF7D0FF20B19DF89A
:100A7000070003B05DF804FB4FF0FF30F9E700001A
:100A80000A4608B50421FFF7C1FF80F00100C0B29B
:100A9000404208BD30B4054C2368DD69044B0A466A
:100AA000AC460146204630BC604700BF0826002007
:100AB000A086010070B501F0CDF9094E094D3080D6
:100AC000002428683388834208D901F0BDF92B68D7
:100AD00004440133B4F5404F2B60F2D370BD00BF26
:100AE000962300206823002001F062BA00F1006024
:100AF00000F540400068704700F10060920000F58A
:100B0000404001F0EDB90000054B1A68054B1B8809
:100B10009B1A834202D9104401F096B90020704715
:100B2000682300209623002038B5084D044629B1DB
:100B300028682044BDE8384001F0A6B92868204460
:100B400001F08AF90028F3D038BD00BF68230020E7
:100B500010F003030AD1B0F5047F05D200F1005074
:100B6000A0F51040D0F80038184670470023FBE786
:100B700000F10050A0F51040D0F8100A70470000B6
:100B8000064991F8243033B10023086A81F82430F3
:100B90000822FFF7B1BF0120704700BF6C2300207F
:100BA000014B1868704700BF002004E070B5194B76
:100BB0001D68194B0138C5F30B0408442D0C0422A1
:100BC0001E88A6420BD15C680A46013C824213464D
:100BD0000FD214F9016F4EB102F8016BF6E7013A3A
:100BE00003F10803ECD181420B4602D22C2203F818
:100BF000012B0A4A05241688AE4204D1984284BFCC
:100C0000967803F8016B013C02F10402F3D1581A03
:100C100070BD00BF002004E08C3400087834000868
:100C2000022802BF024B4FF000429A61704700BF9A
:100C300000080240022802BF024B4FF400429A61B2
:100C4000704700BF00080240022801BF024A5369F2
:100C500083F40043536170470008024070B50446B6
:100C60004FF47A764CB1412C254628BF412506FB2E
:100C700005F000F0D3FD641BF4E770BD10B5002350
:100C8000934203D0CC5CC4540133F9E710BD00009B
:100C900010B5013810F9013F3BB191F900409C4279
:100CA00003D11AB10131013AF4E71AB191F90020E8
:100CB000981A10BD1046FCE703460246D01A12F9F6
:100CC000011B0029FAD1704702440346934202D027
:100CD00003F8011BFAE770472DE9F8431F4D14464E
:100CE00095F824200746884652BBDFF870909CB3E5
:100CF00095F824302BB92022FF2148462F62FFF7B8
:100D0000E3FF95F82400C0F10802A24228BF224662
:100D1000D6B24146920005EB8000FFF7AFFF95F891
:100D20002430A41B1E44F6B2082E17449044E4B2AB
:100D300085F82460DBD1FFF723FF0028D7D108E036
:100D40002B6A03EB82038342CFD0FFF719FF002801
:100D5000CBD10020BDE8F8830120FBE76C23002005
:100D6000024B1A78024B1A70704700BF9423002080
:100D70001022002010B5104C104800F0B5F82146A4
:100D80000E4800F0DDF82468626DD2F8043843F0B4
:100D90000203C2F804384FF47A70FFF75FFF084986
:100DA000204600F0D3F9626DD2F8043823F0020334
:100DB000C2F8043810BD00BF5835000808260020CE
:100DC000603500087047000030B5094D0A44914273
:100DD0000DD011F8013B5840082340F30004013BBB
:100DE0002C4013F0FF0384EA5000F6D1EFE730BD4A
:100DF0002083B8ED026843681143016003B11847CE
:100E00007047000013B5446BD4F894341A68117815
:100E1000042915D1217C022912D1197912890123C3
:100E20008B4013420CD101A904F14C0001F0F4FEF7
:100E3000D4F89444019B21790246206800F0D0F94F
:100E400002B010BD143001F077BE00004FF0FF3348
:100E5000143001F071BE00004C3001F049BF0000B9
:100E60004FF0FF334C3001F043BF0000143001F06D
:100E700045BE00004FF0FF31143001F03FBE0000CE
:100E80004C3001F015BF00004FF0FF324C3001F044
:100E90000FBF00000020704710B5D0F894341A68D6
:100EA00011780429044617D1017C022914D15979FB
:100EB000528901238B4013420ED1143001F0D8FD2A
:100EC000024648B1D4F894444FF4807361792068A5
:100ED000BDE8104000F072B910BD0000406BFFF794
:100EE000DBBF0000704700007FB5124B036000239A
:100EF0004360C0E90233012502260F4B0574044606
:100F00000290019300F18402294600964FF4807309
:100F1000143001F089FD094B0294CDE9006304F51A
:100F200023724FF48073294604F14C0001F050FE07
:100F300004B070BDAC340008DD0E0008050E0008DA
:100F40000B68302282F311880A7903EB82029061E8
:100F50004A79093243F822008A7912B103EB8203FD
:100F600098610223C0F894140374002080F3118860
:100F70007047000038B5037F044613B190F8543031
:100F8000ABB9201D01250221FFF734FF04F1140045
:100F900025776FF0010100F069FC84F8545004F1EA
:100FA0004C006FF00101BDE8384000F05FBC38BD77
:100FB00010B5012104460430FFF71CFF00232377FE
:100FC00084F8543010BD000038B5044600251430B4
:100FD00001F042FD04F14C00257701F011FE201DC7
:100FE00084F854500121FFF705FF2046BDE8384042
:100FF000FFF752BF90F8443003F06003202B07D175
:1010000090F84520212A4FF0000303D81F2A06D864
:1010100000207047222AFBD1C0E90E3303E0034AC7
:1010200082630722C26303640120704711220020FB
:1010300037B5D0F894341A681178042904461AD1C7
:10104000017C022917D11979128901238B4013429F
:1010500011D100F14C05284601F092FE58B101A9CA
:10106000284601F0D9FDD4F89444019B2179024629
:10107000206800F0B5F803B030BD0000F0B500EB1B
:10108000810385B09E6904460D46FEB1302383F38B
:10109000118804EB8507301D0821FFF7ABFEFB68C4
:1010A0005B691B6806F14C001BB1019001F0C2FDA9
:1010B000019803A901F0B0FD024648B1039B2946FF
:1010C000204600F08DF8002383F3118805B0F0BDB1
:1010D000FB685A691268002AF5D01B8A013B13404D
:1010E000F1D104F14402EAE7093138B550F8214062
:1010F000DCB1302383F31188D4F894241368527937
:1011000003EB8203DB689B695D6845B104216018CD
:10111000FFF770FE294604F1140001F0B3FC2046ED
:10112000FFF7BAFE002383F3118838BD7047000033
:1011300001F012B8012303700023C0E90133C36139
:1011400083620362C36243620363704738B5044637
:10115000302383F311880025C0E90355C0E9055504
:10116000416001F009F80223237085F311882846B5
:1011700038BD000070B500EB810305465069DA60A8
:101180000E46144618B110220021FFF79DFDA069FC
:1011900018B110220021FFF797FD31462846BDE81F
:1011A000704001F0B3B80000826802F00112826062
:1011B0000022C0E90422826101F034B9F0B400EBEE
:1011C00081044789E4680125A4698D403D43458138
:1011D00023600023A2606360F0BC01F04FB90000FF
:1011E000F0B400EB81040789E468012564698D404F
:1011F0003D43058123600023A2606360F0BC01F0E1
:10120000C9B9000070B50223002504460370C0E987
:101210000255C0E90455C564856180F8345001F079
:1012200011F863681B6823B129462046BDE8704069
:10123000184770BD0378052B10B504460AD080F816
:1012400050300523037043681B680BB10421984795
:101250000023A36010BD00000178052906D190F895
:101260005020436802701B6803B1184770470000A4
:1012700070B590F83430044613B1002380F8343050
:1012800004F14402204601F0EFF863689B68B3B9AB
:1012900094F8443013F0600535D00021204601F069
:1012A0008FFB0021204601F081FB63681B6813B1AE
:1012B000062120469847062384F8343070BD204626
:1012C00098470028E4D0B4F84A30E26B9A4288BFCD
:1012D000E36394F94430E56B002B4FF0300380F268
:1012E0000381002D00F0F280092284F8342083F37A
:1012F00011880021D4E90E232046FFF771FF002357
:1013000083F31188DAE794F8452003F07F0343EA7A
:10131000022340F20232934200F0C58021D8B3F597
:10132000807F48D00DD8012B3FD0022B00F0938056
:10133000002BB2D104F14C02A2630222E2632364C7
:10134000C1E7B3F5817F00F09B80B3F5407FA4D166
:1013500094F84630012BA0D1B4F84C3043F002038E
:1013600032E0B3F5006F4DD017D8B3F5A06F31D090
:10137000A3F5C063012B90D8636894F846205E689B
:1013800094F84710B4F848302046B047002884D07D
:101390004368A3630368E3631AE0B3F5106F36D0C4
:1013A00040F6024293427FF478AF5C4BA363022382
:1013B000E3630023C3E794F84630012B7FF46DAF5D
:1013C000B4F84C3023F00203C4E90E55A4F84C30B5
:1013D000256478E7B4F84430B3F5A06F0ED194F8E3
:1013E000463084F84E30204600F084FF63681B6866
:1013F00013B1012120469847032323700023C4E939
:101400000E339CE704F14F03A3630123C3E7237862
:10141000042B10D1302383F311882046FFF7C4FE3C
:1014200085F311880321636884F84F5021701B688D
:101430000BB12046984794F84630002BDED084F854
:101440004F300423237063681B68002BD6D0022121
:1014500020469847D2E794F848301D0603F00F0164
:1014600020460AD500F0F2FF012804D002287FF4BC
:1014700014AF2B4B9AE72B4B98E700F0D9FFF3E71B
:1014800094F84630002B7FF408AF94F8483013F0FE
:101490000F01B3D01A06204602D501F0A5FAADE738
:1014A00001F098FAAAE794F84630002B7FF4F5AEE5
:1014B00094F8483013F00F01A0D01B06204602D547
:1014C00001F07EFA9AE701F071FA97E7142284F8A6
:1014D000342083F311882B462A4629462046FFF7FD
:1014E0006DFE85F31188E9E65DB1152284F834209C
:1014F00083F311880021D4E90E232046FFF75EFE16
:10150000FDE60B2284F8342083F311882B462A460B
:1015100029462046FFF764FEE3E700BFDC340008FD
:10152000D4340008D834000838B590F83430044674
:10153000002B3ED0063BDAB20F2A34D80F2B32D81C
:10154000DFE803F0373131082232313131313131C6
:1015500031313737C56BB0F84A309D4214D2C36879
:101560001B8AB5FBF3F203FB12556DB9302383F3ED
:1015700011882B462A462946FFF732FE85F311884B
:101580000A2384F834300EE0142384F834303023F6
:1015900083F3118800231A4619462046FFF70EFEF2
:1015A000002383F3118838BD036C03B198470023EF
:1015B000E7E70021204601F003FA0021204601F070
:1015C000F5F963681B6813B1062120469847062386
:1015D000D7E7000010B590F83430142B044629D01A
:1015E00017D8062B05D001D81BB110BD093B022B23
:1015F000FBD80021204601F0E3F90021204601F04C
:10160000D5F963681B6813B1062120469847062365
:1016100019E0152BE9D10B2380F83430302383F304
:10162000118800231A461946FFF7DAFD002383F3D9
:101630001188DAE7C3689B695B68002BD5D1036C1E
:1016400003B19847002384F83430CEE700230375B4
:10165000826803691B6899689142FBD25A680360EB
:101660004260106058607047002303758268036908
:101670001B6899689142FBD85A6803604260106009
:101680005860704708B50846302383F311880B7DF6
:10169000032B05D0042B0DD02BB983F3118808BD83
:1016A0008B6900221A604FF0FF338361FFF7CEFF92
:1016B0000023F2E7D1E9003213605A60F3E700003B
:1016C000FFF7C4BF054BD9680875186802681A602F
:1016D000536001220275D860FEF714BE98230020E3
:1016E00030B50C4BDD684B1C87B004460FD02B4641
:1016F000094A684600F04EF92046FFF7E3FF009BD9
:1017000013B1684600F050F9A86907B030BDFFF783
:10171000D9FFF9E79823002085160008044B1A68C2
:10172000DB6890689B68984294BF00200120704756
:1017300098230020084B10B51C68D86822681A60EE
:10174000536001222275DC60FFF78EFF01462046C0
:10175000BDE81040FEF7D6BD9823002038B5074CF1
:1017600007490848012300252370656001F040FB0C
:101770000223237085F3118838BD00BF00260020A6
:10178000E43400089823002000F044B9034A51686B
:1017900053685B1A9842FBD8704700BF001000E006
:1017A0008B60022308618B82084670478368A3F12F
:1017B000840243F8142C026943F8442C426943F82C
:1017C000402C094A43F8242CC26843F8182C022202
:1017D00003F80C2C002203F80B2C044A43F8102CBD
:1017E000A3F12000704700BF1D03000898230020CC
:1017F00008B5FFF7DBFFBDE80840FFF761BF000059
:10180000024BDB6898610F20FFF75CBF9823002034
:10181000302383F31188FFF7F3BF000008B50146BA
:10182000302383F311880820FFF75AFF002383F346
:10183000118808BD064BDB6839B1426818605A60F0
:10184000136043600420FFF74BBF4FF0FF30704739
:10185000982300200368984206D01A6802605060FE
:1018600099611846FFF72CBF7047000038B5044651
:101870000D462068844200D138BD036823605C6057
:101880008561FFF71DFFF4E710B503689C68A2426D
:101890000CD85C688A600B604C6021605960996864
:1018A0008A1A9A604FF0FF33836010BD1B68121BC9
:1018B000ECE700000A2938BF0A2170B504460D463E
:1018C0000A26601901F08EFA01F07AFA041BA5428B
:1018D00003D8751C2E460446F3E70A2E04D9BDE84A
:1018E0007040012001F0C4BA70BD0000F8B5144B7F
:1018F0000D46D96103F1100141600A2A196982601D
:1019000038BF0A22016048601861A818144601F027
:101910005BFA0A2701F054FA431BA342064606D39A
:101920007C1C281901F05EFA27463546F2E70A2F9B
:1019300004D9BDE8F840012001F09ABAF8BD00BF13
:1019400098230020F8B506460D4601F039FA0F4AF3
:10195000134653F8107F9F4206D12A46014630466F
:10196000BDE8F840FFF7C2BFD169BB68441A2C1923
:1019700028BF2C46A34202D92946FFF79BFF2246E7
:1019800031460348BDE8F840FFF77EBF98230020AA
:10199000A823002010B4C0E9032300235DF8044B02
:1019A0004361FFF7CFBF000010B5194C236998427F
:1019B0000DD0D0E90032816813605A609A680A44F9
:1019C0009A60002303604FF0FF33A36110BD2346EC
:1019D000026843F8102F53600022026022699A4285
:1019E00003D1BDE8104001F0F7B9936881680B445A
:1019F000936001F0E5F92269E1699268441AA24214
:101A0000E4D91144BDE81040091AFFF753BF00BFE5
:101A1000982300202DE9F047DFF8BC8008F110077B
:101A20002C4ED8F8105001F0CBF9D8F81C40AA6819
:101A3000031B9A423ED81444D5E900324FF0000906
:101A4000C8F81C4013605A60C5F80090D8F81030F0
:101A5000B34201D101F0C0F989F31188D5E903310E
:101A600028469847302383F311886B69002BD8D020
:101A700001F0A6F96A69A0EB04094A4582460DD235
:101A8000022001F0F5F90022D8F81030B34208D155
:101A900051462846BDE8F047FFF728BF121A2244F6
:101AA000F2E712EB090938BF4A4629463846FFF7E4
:101AB000EBFEB5E7D8F81030B34208D01444211A31
:101AC000C8F81C00A960BDE8F047FFF7F3BEBDE809
:101AD000F08700BFA8230020982300200020704733
:101AE000FEE70000704700004FF0FF307047000035
:101AF00002290CD0032904D00129074818BF00206F
:101B00007047032A05D8054800EBC2007047044817
:101B100070470020704700BFBC350008202200201D
:101B20007035000870B59AB00546084601A91446FC
:101B300000F0C2F801A8FFF7BFF8431C5B00C5E93D
:101B400000340022237003236370C6B201AB023459
:101B50001046D1B28E4204F1020401D81AB070BD11
:101B600013F8011B04F8021C04F8010C0132F0E721
:101B700008B5302383F311880348FFF759FA00238F
:101B800083F3118808BD00BF0826002090F8443078
:101B900003F01F02012A07D190F845200B2A03D138
:101BA0000023C0E90E3315E003F06003202B08D1B9
:101BB000B0F848302BB990F84520212A03D81F2AC5
:101BC00004D8FFF717BA222AEBD0FAE7034A826358
:101BD0000722C26303640120704700BF182200205F
:101BE00007B5052917D8DFE801F0191603191920E0
:101BF000302383F31188104A01900121FFF7BAFACC
:101C000001980E4A0221FFF7B5FA0D48FFF7DCF9FB
:101C1000002383F3118803B05DF804FB302383F3C2
:101C200011880748FFF7A6F9F2E7302383F31188FC
:101C30000348FFF7BDF9EBE710350008343500081D
:101C40000826002038B50C4D0C4C0D492A4604F1ED
:101C50000800FFF767FF05F1CA0204F11000094907
:101C6000FFF760FF05F5CA7204F118000649BDE8E8
:101C70003840FFF757BF00BFD02A002020220020A5
:101C8000F0340008FA3400080535000870B5044641
:101C900008460D46FFF710F8C6B220460134037817
:101CA0000BB9184670BD32462946FEF7F1FF0028F1
:101CB000F3D10120F6E700002DE9F84F05460C4668
:101CC000FEF7FAFF2949C6B22846FFF7DFFF08B141
:101CD000013EF6B226492846FFF7D8FF08B1103674
:101CE000F6B2632E0DD8DFF88490DFF884A0214F80
:101CF000DFF888B0DFF888802E7846B92670BDE816
:101D0000F88F29462046BDE8F84F01F097BB252EF5
:101D100028D1072249462846FEF7BAFF40B9D8F82D
:101D200000302360B8F80430A38007350634E3E7B9
:101D3000082251462846FEF7ABFF98B90E4BA21C6D
:101D4000197809090232C95D02F8041C13F8011B55
:101D500001F00F015B45C95D02F8031CF0D1183496
:101D60000835C9E704F8016B0135C5E7DC35000823
:101D700005350008EB350008107AFF1F1C7AFF1F9D
:101D8000E4350008BFF34F8F024AD368DB03FCD46D
:101D9000704700BF003C024008B5094B1B7873B97F
:101DA000FFF7F0FF074B1A69002ABFBF064A5A60C7
:101DB00002F188325A601A6822F480621A6008BD03
:101DC0002E2D0020003C02402301674508B50B4B37
:101DD0001B7893B9FFF7D6FF094B1A6942F000420E
:101DE0001A611A6842F480521A601A6822F480520A
:101DF0001A601A6842F480621A6008BD2E2D002015
:101E0000003C02400B28F0B516D80C4C0C49237846
:101E10007BB90C4D0E460C234FF0006255F8047B45
:101E200046F8042B013B13F0FF033A44F6D101239B
:101E3000237051F82000F0BD0020FCE7602D002049
:101E4000302D0020FC350008014B53F8200070476E
:101E5000FC3500080C2070470B2810B5044601D94A
:101E6000002010BDFFF7CEFF064B53F82430184476
:101E7000C21A0BB90120F4E712680132F0D1043B19
:101E8000F6E700BFFC3500080B2810B5044621D842
:101E9000FFF778FFFFF780FF0F4AF323D360C300FB
:101EA000DBB243F4007343F002031361136943F49C
:101EB00080331361FFF766FFFFF7A4FF074B53F86A
:101EC000241000F0D9F8FFF781FF2046BDE810404C
:101ED000FFF7C2BF002010BD003C0240FC350008E7
:101EE000F8B512F00103144642D18218B2F1016F25
:101EF00057D82D4B1B6813F0010352D02B4DFFF721
:101F00004BFFF323EB60FFF73DFF40F20127032C6B
:101F100015D824F001046618244C401A40F2011729
:101F2000B142236900EB010524D123F001032361B1
:101F3000FFF74CFF0120F8BD043C0430E7E78307BE
:101F4000E7D12B6923F440732B612B693B432B6151
:101F500051F8046B0660BFF34F8FFFF713FF036860
:101F60009E42E9D02B6923F001032B61FFF72EFF7E
:101F70000020E0E723F44073236123693B4323619E
:101F80000B882B80BFF34F8FFFF7FCFE2D8831F8B5
:101F9000023BADB2AB42C3D0236923F001032361FE
:101FA000E4E71846C7E700BF00380240003C0240A3
:101FB000084908B50B7828B11BB9FFF7EDFE0123DE
:101FC0000B7008BD002BFCD0BDE808400870FFF77F
:101FD000FDBE00BF2E2D002010B50244064BD2B22C
:101FE000904200D110BD441C00B253F8200041F8CB
:101FF000040BE0B2F4E700BF502800400F4B30B5AF
:102000001C6F240407D41C6F44F400741C671C6FFD
:1020100044F400441C670A4C236843F48073236033
:102020000244084BD2B2904200D130BD441C00B2F1
:1020300051F8045B43F82050E0B2F4E70038024066
:10204000007000405028004007B5012201A900207F
:10205000FFF7C2FF019803B05DF804FB13B5044617
:10206000FFF7F2FFA04205D0012201A90020019450
:10207000FFF7C4FF02B010BD70470000034B1A68A1
:102080001AB9034AD2F874281A607047642D0020E8
:102090000030024008B5FFF7F1FF024B1868C0F3AB
:1020A000407008BD642D002070470000FEE700006E
:1020B0000A4B0B480B4A90420BD30B4BDA1C121AFB
:1020C000C11E22F003028B4238BF00220021FEF71E
:1020D000FBBD53F8041B40F8041BECE7A8370008CD
:1020E000602E0020602E0020602E002070B5D0E908
:1020F00015439E6800224FF0FF3504EB4213510157
:10210000D3F800090028BEBFD3F8000940F0804092
:10211000C3F80009D3F8000B0028BEBFD3F8000BAA
:1021200040F08040C3F8000B013263189642C3F8B8
:102130000859C3F8085BE0D24FF00113C4F81C380B
:1021400070BD0000890141F02001016103699B0617
:10215000FCD41220FFF71ABB10B5054C2046FEF741
:10216000E9FF4FF0A0436365024BA36510BD00BFBC
:10217000682D00205036000870B50378012B054605
:1021800050D12A4B446D98421BD1294B5A6B42F0D7
:1021900080025A635A6D42F080025A655A6D5A693C
:1021A00042F080025A615A6922F080025A610E217F
:1021B00043205B6900F022FC1E4BE3601E4BC4F819
:1021C00000380023C4F8003EC02323606E6D4FF436
:1021D0000413A3633369002BFCDA012333610C2061
:1021E000FFF7D4FA3369DB07FCD41220FFF7CEFAED
:1021F0003369002BFCDA0026A6602846FFF776FF3D
:102200006B68C4F81068DB68C4F81468C4F81C680C
:102210004BB90A4BA3614FF0FF336361A36843F0EE
:102220000103A36070BD064BF4E700BF682D0020DA
:10223000003802404014004003002002003C30C03F
:10224000083C30C0F8B5446D054600212046FFF734
:1022500079FFA96D00234FF001128F68C4F834385C
:102260004FF00066C4F81C284FF0FF3004EB431217
:1022700001339F42C2F80069C2F8006BC2F8080936
:10228000C2F8080BF2D20B686A6DEB65636210232B
:102290001361166916F01006FBD11220FFF776FACB
:1022A000D4F8003823F4FE63C4F80038A36943F47B
:1022B000402343F01003A3610923C4F81038C4F885
:1022C00014380A4BEB604FF0C043C4F8103B084B86
:1022D000C4F8003BC4F81069C4F80039EB6D03F191
:1022E000100243F48013EA65A362F8BD2C3600089F
:1022F00040800010426D90F84E10D2F8003823F460
:10230000FE6343EA0113C2F8003870472DE9F84331
:1023100000EB8103456DDA68166806F00306731E4C
:10232000022B05EB41130C4680460FFA81F94FEA68
:1023300041104FF00001C3F8101B4FF0010104F1F0
:10234000100398BFB60401FA03F391698EBF334EB0
:1023500006F1805606F5004600293AD0578A04F166
:102360005801490137436F50D5F81C180B43C5F885
:102370001C382B180021C3F8101953690127611E5E
:10238000A7409BB3138A928B9B08012A88BF5343B3
:10239000D8F85C20981842EA034301F1400205EBAB
:1023A0008202C8F85C00214653602846FFF7CAFE47
:1023B00008EB8900C3681B8A43EA845348346401EC
:1023C0001E432E51D5F81C381F43C5F81C78BDE8B4
:1023D000F88305EB4917D7F8001B21F40041C7F833
:1023E000001BD5F81C1821EA0303C0E704F13F03E2
:1023F00005EB83030A4A5A6028462146FFF7A2FEEE
:1024000005EB4910D0F8003923F40043C0F8003937
:10241000D5F81C3823EA0707D7E700BF0080001073
:1024200000040002826D1268C265FFF75FBE000003
:102430005831436D49015B5813F4004004D013F444
:10244000001F0CBF02200120704700004831436D7F
:1024500049015B5813F4004004D013F4001F0CBF73
:10246000022001207047000000EB8101CB68196A4F
:102470000B6813604B6853607047000000EB8103EA
:1024800030B5DD68AA691368D36019B9402B84BFE1
:10249000402313606B8A1468426D1C44013CB4FBFA
:1024A000F3F46343033323F0030302EB411043EAE5
:1024B000C44343F0C043C0F8103B2B6803F0030350
:1024C000012B09B20ED1D2F8083802EB411013F4F7
:1024D000807FD0F8003B14BF43F0805343F000539B
:1024E000C0F8003B02EB4112D2F8003B43F004433A
:1024F000C2F8003B30BD00002DE9F041244D6E6D67
:1025000006EB40130446D3F8087BC3F8087B380772
:102510000AD5D6F81438190706D505EB84032146E9
:10252000DB6828465B689847FA071FD5D6F8143849
:10253000DB071BD505EB8403D968CCB98B69488AC6
:102540005A68B2FBF0F600FB16228AB91868DA68FE
:1025500090420DD2121AC3E90024302383F311886C
:102560000B482146FFF78AFF84F31188BDE8F0810C
:10257000012303FA04F26B8923EA02036B81CB681F
:10258000002BF3D021460248BDE8F041184700BFB8
:10259000682D002000EB810370B5DD68436D6C6928
:1025A0002668E6604A0156BB1A444FF40020C2F880
:1025B00010092A6802F00302012A0AB20ED1D3F8E8
:1025C000080803EB421410F4807FD4F8000914BF0C
:1025D00040F0805040F00050C4F8000903EB421274
:1025E000D2F8000940F00440C2F80009D3F83408DA
:1025F000012202FA01F10143C3F8341870BD19B980
:10260000402E84BF4020206020682E8A8419013C1F
:10261000B4FBF6F440EAC44040F000501A44C6E768
:102620002DE9F8433B4D6E6D06EB40130446D3F89D
:102630000889C3F8088918F0010F4FEA40171AD02B
:10264000D6F81038DB0716D505EB8003D9684B693F
:102650001868DA68904230D2121A4FF000091A60F6
:10266000C3F80490302383F3118821462846FFF7EE
:1026700091FF89F3118818F0800F1CD0D6F83438F8
:102680000126A640334216D005EB84036D6DD3F8C6
:102690000CC0DCF814200134E4B2D2F800E005EB01
:1026A00004342F445168714515D3D5F8343823EAE2
:1026B0000606C5F83468BDE8F883012303FA04F27E
:1026C0002B8923EA02032B818B68002BD3D0214670
:1026D00028469847CFE7BCF81000AEEB01038342D1
:1026E00028BF0346D7F8180980B2B3EB800FE2D8B1
:1026F0009068A0F1040959F8048FC4F80080A0EB99
:1027000009089844B8F1040FF5D818440B449060B8
:102710005360C7E7682D00202DE9F74FA24C656D87
:102720006E69AB691E4016F480586E6107D0204672
:10273000FEF768FD03B0BDE8F04F00F047BC002E87
:1027400012DAD5F8003E98489B071EBFD5F8003E28
:1027500023F00303C5F8003ED5F8043823F0010345
:10276000C5F80438FEF778FD370505D58E48FFF724
:10277000BDFC8D48FEF75EFDB0040CD5D5F80838D9
:1027800013F0060FEB6823F470530CBF43F410539F
:1027900043F4A053EB6031071BD56368DB681BB9BA
:1027A000AB6923F00803AB612378052B0CD1D5F876
:1027B000003E7D489A071EBFD5F8003E23F0030374
:1027C000C5F8003EFEF748FD6368DB680BB176484C
:1027D0009847F30274D4B70227D5D4F85490DFF8A1
:1027E000C8B100274FF0010A09EB4712D2F8003BAD
:1027F00003F44023B3F5802F11D1D2F8003B002B16
:102800000DDA62890AFA07F322EA0303638104EB13
:102810008703DB68DB6813B1394658469847A36DD8
:1028200001379B68FFB29F42DED9F00617D5676D6E
:102830003A6AC2F30A1002F00F0302F4F012B2F582
:10284000802F00F08580B2F5402F08D104EB830380
:102850000022DB681B6A07F5805790426AD130037B
:10286000D5F8184813D5E10302D50020FFF744FE40
:10287000A20302D50120FFF73FFE630302D5022029
:10288000FFF73AFE270302D50320FFF735FE750355
:102890007FF550AFE00702D50020FFF7C1FEA1078A
:1028A00002D50120FFF7BCFE620702D50220FFF728
:1028B000B7FE23077FF53EAF0320FFF7B1FE39E7F0
:1028C000636DDFF8E4A0019300274FF00109A36DC9
:1028D0009B685FFA87FB9B453FF67DAF019B03EB4F
:1028E0004B13D3F8001901F44021B1F5802F1FD10B
:1028F000D3F8001900291BDAD3F8001941F09041F0
:10290000C3F80019D3F800190029FBDB5946606DA4
:10291000FFF718FC218909FA0BF321EA030323814D
:1029200004EB8B03DB689B6813B15946504698470C
:102930000137CCE7910708BFD7F80080072A98BF76
:1029400003F8018B02F1010298BF4FEA182884E7CF
:10295000023304EB830207F580575268D2F818C09F
:10296000DCF80820DCE9001CA1EB0C0C00218842FB
:102970000AD104EB830463689B699A6802449A60F5
:102980005A6802445A606AE711F0030F08BFD7F88B
:1029900000808C4588BF02F8018B01F1010188BFDE
:1029A0004FEA1828E3E700BF682D0020436D03EBD2
:1029B0004111D1F8003B43F40013C1F8003B7047CC
:1029C000436D03EB4111D1F8003943F40013C1F812
:1029D00000397047436D03EB4111D1F8003B23F4FC
:1029E0000013C1F8003B7047436D03EB4111D1F870
:1029F000003923F40013C1F80039704700F1604337
:102A000003F561430901C9B283F80013012200F004
:102A10001F039A4043099B0003F1604303F56143A0
:102A2000C3F880211A60704730B5039C01720433EB
:102A300004FB0325C0E90653049B03630021059BA7
:102A4000C160C0E90000C0E90422C0E90842C0E951
:102A50000A11436330BD0000416A0022C0E904113D
:102A6000C0E90A22C2606FF00101FEF7FFBE00005C
:102A7000D0E90432934201D1C2680AB9181D7047E7
:102A80000020704703691960C2680132C260C269E0
:102A9000134482690361934224BF436A03610021A6
:102AA000FEF7D8BE38B504460D46E3683BB162690F
:102AB000131D1268A3621344E362002007E0237A27
:102AC00033B929462046FEF7B5FE0028EDDA38BDB9
:102AD0006FF00100FBE70000C368C269013BC360FF
:102AE0004369134482694361934224BF436A43614B
:102AF00000238362036B03B11847704770B530231E
:102B0000044683F31188866A3EB9FFF7CBFF05467A
:102B100018B186F31188284670BDA36AE26A13F8DB
:102B2000015BA362934202D32046FFF7D5FF002347
:102B300083F31188EFE700002DE9F84F04460E46B5
:102B4000174698464FF0300989F311880025AA46A8
:102B5000D4F828B0BBF1000F09D141462046FFF759
:102B6000A1FF20B18BF311882846BDE8F88FD4E986
:102B70000A12A7EB050B521A934528BF9346BBF1E7
:102B8000400F1BD9334601F1400251F8040B43F8C2
:102B9000040B9142F9D1A36A40334036A362403519
:102BA000D4E90A239A4202D32046FFF795FF8AF31D
:102BB0001188BD42D8D289F31188C9E730465A46F8
:102BC000FEF75CF8A36A5B445E44A3625D44E7E7FA
:102BD00010B5029C0172043303FB0421C0E9061303
:102BE0000023C0E90A33039B0363049BC460C0E96C
:102BF0000000C0E90422C0E90842436310BD0000A0
:102C0000026AC260426AC0E904220022C0E90A22C4
:102C10006FF00101FEF72ABED0E904239A4201D1E8
:102C2000C26822B9184650F8043B0B607047002375
:102C30001846FAE7C368C2690133C36043691344A5
:102C400082694361934224BF436A43610021FEF7D6
:102C500001BE000038B504460D46E3683BB1236968
:102C60001A1DA262E2691344E362002007E0237A9E
:102C700033B929462046FEF7DDFD0028EDDA38BDE0
:102C80006FF00100FBE7000003691960C268013AB8
:102C9000C260C269134482690361934224BF436ADC
:102CA000036100238362036B03B118477047000080
:102CB00070B530230D460446114683F31188866AA9
:102CC0002EB9FFF7C7FF10B186F3118870BDA36A54
:102CD0001D70A36AE26A01339342A36204D3E169DF
:102CE00020460439FFF7D0FF002080F31188EDE77C
:102CF0002DE9F84F04460D46904699464FF0300AAC
:102D00008AF311880026B346A76A4FB94946204680
:102D1000FFF7A0FF20B187F311883046BDE8F88F98
:102D2000D4E90A073A1AA8EB0607974228BF1746C4
:102D3000402F1BD905F1400355F8042B40F8042B14
:102D40009D42F9D1A36A4033A3624036D4E90A23F5
:102D50009A4204D3E16920460439FFF795FF8BF3CB
:102D600011884645D9D28AF31188CDE729463A46DB
:102D7000FDF784FFA36A3B443D44A3623E44E5E77C
:102D8000D0E904239A4217D1C3689BB1836A8BB1FF
:102D9000043B9B1A0ED01360C368013BC360C36938
:102DA0001A44836902619A4224BF436A0361002383
:102DB00083620123184670470023FBE700F030B917
:102DC0004FF08043586A70474FF0804300225863A9
:102DD0001A610222DA6070474FF080430022DA6005
:102DE000704700004FF0804358637047FEE70000D3
:102DF00070B51B4B01630025044686B058608562A0
:102E00000E4600F0BFF804F11003C4E904334FF09C
:102E1000FF33C4E90635C4E90044A560E562FFF765
:102E2000CFFF2B460246C4E9082304F134010D4AC2
:102E3000256580232046FEF7B3FC0123E0600A4AA3
:102E40000375009272680192B268CDE90223074BC4
:102E50006846CDE90435FEF7CBFC06B070BD00BF77
:102E6000002600205C36000861360008ED2D0008C1
:102E7000024AD36A1843D062704700BF98230020EB
:102E80004B6843608B688360CB68C3600B694361A8
:102E90004B6903628B6943620B68036070470000F3
:102EA00008B5264B26481A6940F2FF110A431A61F9
:102EB0001A6922F4FF7222F001021A611A691A6B70
:102EC0000A431A631A6D0A431A651E4A1B6D11469E
:102ED000FFF7D6FF02F11C0100F58060FFF7D0FF7D
:102EE00002F1380100F58060FFF7CAFF02F15401DA
:102EF00000F58060FFF7C4FF02F1700100F580600B
:102F0000FFF7BEFF02F18C0100F58060FFF7B8FF0C
:102F100002F1A80100F58060FFF7B2FF02F1C401E1
:102F200000F58060FFF7ACFF02F1E00100F5806082
:102F3000FFF7A6FFBDE8084000F0EEB800380240F9
:102F4000000002406836000808B500F059FAFEF7A4
:102F500005FCFFF793F8BDE80840FEF773BE0000DC
:102F600070470000EFF3098305494A6B22F0010224
:102F70004A63683383F30988002383F31188704719
:102F800000EF00E0302080F3118862B60C4B0D4A50
:102F9000D96821F4E0610904090C0A43DA60D3F826
:102FA000FC20094942F08072C3F8FC200A6842F014
:102FB00001020A602022DA7783F82200704700BFFE
:102FC00000ED00E00003FA05001000E010B530232A
:102FD00083F311880E4B5B6813F4006314D0F1EE99
:102FE000103AEFF30984683C4FF08073E361094BBA
:102FF000DB6B236684F30988FEF790FB10B1064B68
:10300000A36110BD054BFBE783F31188F9E700BF0F
:1030100000ED00E000EF00E02F030008320300089D
:103020000F4B1A6C42F001021A641A6E42F0010250
:103030001A660C4A1B6E936843F0010393604FF0CD
:10304000804353229A624FF0FF32DA6200229A6183
:103050005A63DA605A6001225A611A60704700BFF1
:1030600000380240002004E04FF0804208B51169AA
:10307000D3680B40D9B2C9439B07116107D53023F0
:1030800083F31188FEF780FB002383F3118808BDCA
:103090001F4B1A696FEAC2526FEAD2521A611A695B
:1030A000C2F308021A614FF0FF301A695A69586179
:1030B00000215A6959615A691A6A62F080521A628B
:1030C0001A6A02F080521A621A6A5A6A58625A6A76
:1030D00059625A6A1A6C42F080521A641A6E42F0AF
:1030E00080521A661A6E0B4A106840F480701060A5
:1030F000186F00F44070B0F5007F1EBF4FF48030B1
:1031000018671967536823F40073536000F054B9CB
:103110000038024000700040334B4FF080521A6478
:10312000324A4FF4404111601A6842F001021A60BD
:103130001A689107FCD59A6822F003029A602A4B1C
:103140009A6812F00C02FBD1196801F0F9011960BC
:103150009A601A6842F480321A601A689203FCD5A9
:103160005A6F42F001025A671F4B5A6F9007FCD505
:103170001F4A5A601A6842F080721A601B4A5368EC
:103180005904FCD5184B1A689201FCD5194A9A606B
:10319000194B1A68194B9A42194B21D1194A1168D7
:1031A000194A91421CD140F205121A60144A136860
:1031B00003F00F03052BFAD10B4B9A6842F0020281
:1031C0009A609A6802F00C02082AFAD15A6C42F40A
:1031D00080425A645A6E42F480425A665B6E70476F
:1031E00040F20572E1E700BF003802400070004085
:1031F0000854400700948838002004E0116400203F
:10320000003C024000ED00E041C20F41074A08B512
:10321000536903F00103536123B1054A13680BB1ED
:1032200050689847BDE80840FFF7D0BE003C014019
:10323000E02D0020074A08B5536903F002035361EB
:1032400023B1054A93680BB1D0689847BDE80840A0
:10325000FFF7BCBE003C0140E02D0020074A08B546
:10326000536903F00403536123B1054A13690BB199
:1032700050699847BDE80840FFF7A8BE003C0140F0
:10328000E02D0020074A08B5536903F00803536195
:1032900023B1054A93690BB1D0699847BDE808404E
:1032A000FFF794BE003C0140E02D0020074A08B51E
:1032B000536903F01003536123B1054A136A0BB13C
:1032C000506A9847BDE80840FFF780BE003C0140C7
:1032D000E02D0020164B10B55C6904F478725A6139
:1032E000A30604D5134A936A0BB1D06A98476006C7
:1032F00004D5104A136B0BB1506B9847210604D5C7
:103300000C4A936B0BB1D06B9847E20504D5094A80
:10331000136C0BB1506C9847A30504D5054A936C08
:103320000BB1D06C9847BDE81040FFF74FBE00BF0F
:10333000003C0140E02D0020194B10B55C6904F4FD
:103340007C425A61620504D5164A136D0BB1506D6B
:103350009847230504D5134A936D0BB1D06D984758
:10336000E00404D50F4A136E0BB1506E9847A104C8
:1033700004D50C4A936E0BB1D06E9847620404D505
:10338000084A136F0BB1506F9847230404D5054AC0
:10339000936F0BB1D06F9847BDE81040FFF716BE92
:1033A000003C0140E02D002008B5FFF75DFEBDE8C0
:1033B0000840FFF70BBE0000062108B50846FFF7DE
:1033C0001DFB06210720FFF719FB06210820FFF748
:1033D00015FB06210920FFF711FB06210A20FFF744
:1033E0000DFB06211720FFF709FB06212820FFF718
:1033F00005FBBDE8084007211C20FFF7FFBA0000CD
:1034000008B5FFF745FE00F00BF8FDF791FEFDF75C
:1034100069FDFFF7A5FDBDE80840FFF7CFBC000040
:103420000023054A19460133102BC2E9001102F1AD
:103430000802F8D1704700BFE02D0020034611F8C4
:10344000012B03F8012B002AF9D1704753544D3357
:1034500032463F3F3F0053544D33324634307800BC
:1034600053544D3332463432780053544D33324640
:103470003434365858000000012033000010410059
:1034800001105A000310590007103100000000001D
:103490004C340008130400005634000819040000DE
:1034A00060340008210400006A34000800000000B5
:1034B000610E00084D0E0008890E0008750E000808
:1034C000810E00086D0E0008590E0008450E000818
:1034D000950E000800000000010000000000000040
:1034E00063300000E0340008F023002000260020B4
:1034F0004172647550696C6F740025424F415244AB
:10350000252D424C002553455249414C25000000D1
:1035100002000000000000007D100008E910000813
:1035200040004000A02A0020B02A00200200000035
:103530000000000003000000000000002D11000842
:103540000000000010000000C02A00200000000061
:103550000100000000000000682D002001010200B1
:10356000E11B0008F11A00088D1B0008711B000800
:10357000430000007835000809024300020100C042
:1035800032090400000102020100052400100105B7
:10359000240100010424020205240600010705821B
:1035A000030800FF09040100020A000000070501EA
:1035B00002400000070581024000000012000000E8
:1035C000C4350008120110010200004009124157E1
:1035D00000020102030100000403090425424F41D7
:1035E00052442500574647303031003031323334B1
:1035F00035363738394142434445460000400000E3
:1036000000400000004000000040000000000100F9
:1036100000000200000002000000020000000200A2
:103620000000020000000200000002000000000094
:103630007112000829150008D51500084000400047
:10364000C82D0020C82D002001000000D82D00202A
:103650008000000040010000030000006D61696E01
:103660000069646C650000000000802A0000000012
:10367000AAAAAAAA00000024FFFF00000000000080
:1036800000A00A000000000000000000AAAAAAAAE8
:1036900000000000FFFF000000000000000000002C
:1036A0000000004000000000AAAAAAAA0000000032
:1036B000FF7F00000000000000000000000000008C
:1036C00000000000AAAAAAAA00000000FFFF000054
:1036D00000000000000000000000000000000000EA
:1036E000AAAAAAAA00000000FFFF00000000000034
:1036F000000000000000000000000000AAAAAAAA22
:1037000000000000FFFF00000000000000000000BB
:103710000000000000000000AAAAAAAA0000000001
:10372000FFFF00000000000000000000000000009B
:10373000000000000A00000000000000030000007C
:103740000000000000000000000000000000000079
:103750000000000000000000000000000000000069
:103760000000000000000000FE0700000000000054
:1037700000400F0000000000FF009600000000085D
:10378000009600000000080004000000D835000882
:103790000000000000000000000000000000000029
:1037A0000000000000000000FFFFFFFFFFFFFFFF21
:1037B000FFFFFFFFFFFFFFFFFFFFFFFFFFFFFFFF19
:1037C000FFFFFFFFFFFFFFFFFFFFFFFFFFFFFFFF09
:1037D000FFFFFFFFFFFFFFFFFFFFFFFFFFFFFFFFF9
:1037E000FFFFFFFFFFFFFFFFFFFFFFFFFFFFFFFFE9
:10C000000006002099D20008657A0908C17909085C
:10C010002D7A0908C1790908F97909089BD2000825
:10C020009BD200089BD200089BD20008E99D0B0818
:10C030009BD200089BD200089BD200089BD200082C
:10C040009BD200089BD200089BD200089BD200081C
:10C050009BD200089BD2000805B00B082DB00B083E
:10C0600055B00B087DB00B08A5B00B08A15C0B0800
:10C07000C95C0B08F55C0B08215D0B084D5D0B08D6
:10C08000755D0B08A15D0B08255C0B089BD20008B1
:10C090009BD200089BD200089BD20008CDB00B08B1
:10C0A00005B20B0809B20B081DB20B0821B20B0830
:10C0B00025B20B0839B20B084DB20B082D630B08E3
:10C0C000D5640B089BD200089BD200089BD20008C5
:10C0D0009BD20008A1B10B08B5B10B08C9B10B0880
:10C0E00031B10B089BD200089BD2000871B20B083B
:10C0F00075B20B0889B20B088DB20B08CD5D0B0829
:10C100009BD200089BD2000861B20B089BD20008AA
:10C11000DDB10B08F1B10B089BD200089BD20008DF
:10C12000F95D0B08215E0B084D5E0B08795E0B086C
:10C13000A55E0B089BD200089BD200089BD200088A
:10C140009BD200089BD200089BD2000815A50B08C3
:10C15000CD5E0B08F95E0B08255F0B089BD200082B
:10C160009BD200089BD200089BD200089BD20008FB
:10C170009BD200089BD200089BD200089BD20008EB
:10C180009BD200089BD200089BD200089BD20008DB
:10C190009BD200089BD200089BD200089BD20008CB
:10C1A0009BD200089BD200089BD200089BD20008BB
:10C1B0009BD200089BD200089BD200089BD20008AB
:10C1C0009BD200089BD200089BD200089BD200089B
:10C1D0009BD200089BD200089BD200089BD200088B
:10C1E0003DF5000879250108D1AC010829FB0108BB
:10C1F000457C02082DF90308558405085D8A050869
:10C200007DF5050805460608C94D060801510608D2
:10C21000E1B106087DD006084D660708E9D4070895
:10C2200039730908C5830A0831E50A08490B0B0868
:10C2300095160B0839440B08014A0B080000000052
:10C2400081F0004102E000BF83F0004330B54FEAC7
:10C2500041044FEA430594EA050F08BF90EA020F34
:10C260001FBF54EA000C55EA020C7FEA645C7FEAC7
:10C27000655C00F0E2804FEA5454D4EB5555B8BFEA
:10C280006D420CDD2C4480EA020281EA030382EA5B
:10C29000000083EA010180EA020281EA0303362DED
:10C2A00088BF30BD11F0004F4FEA01314FF4801CC0
:10C2B0004CEA113102D0404261EB410113F0004FD2
:10C2C0004FEA03334CEA133302D0524263EB430389
:10C2D00094EA050F00F0A780A4F10104D5F1200E27
:10C2E0000DDB02FA0EFC22FA05F2801841F1000182
:10C2F00003FA0EF2801843FA05F359410EE0A5F156
:10C3000020050EF1200E012A03FA0EFC28BF4CF086
:10C31000020C43FA05F3C01851EBE37101F000453C
:10C3200007D54FF0000EDCF1000C7EEB00006EEB49
:10C330000101B1F5801F1BD3B1F5001F0CD34908D3
:10C340005FEA30004FEA3C0C04F101044FEA44522A
:10C3500012F5800F80F09A80BCF1004F08BF5FEAB1
:10C36000500C50F1000041EB045141EA050130BD91
:10C370005FEA4C0C404141EB0101013C28BFB1F5A3
:10C38000801FE9D291F0000F04BF01460020B1FAEE
:10C3900081F308BF2033A3F10B03B3F120020CDAC1
:10C3A0000C3208DD02F1140CC2F10C0201FA0CF09F
:10C3B00021FA02F10CE002F11402D8BFC2F1200C04
:10C3C00001FA02F120FA0CFCDCBF41EA0C019040BA
:10C3D000E41AA2BF01EB0451294330BD6FEA040403
:10C3E0001F3C1CDA0C340EDC04F11404C4F12002EE
:10C3F00020FA04F001FA02F340EA030021FA04F300
:10C4000045EA030130BDC4F10C04C4F1200220FA56
:10C4100002F001FA04F340EA0300294630BD21FA94
:10C4200004F0294630BD94F0000F83F4801306BF5A
:10C4300081F480110134013D4EE77FEA645C18BF4E
:10C440007FEA655C29D094EA050F08BF90EA020FE5
:10C4500005D054EA000C04BF1946104630BD91EADD
:10C46000030F1EBF0021002030BD5FEA545C05D1E0
:10C470004000494128BF41F0004130BD14F580041F
:10C480003CBF01F5801130BD01F0004545F0FE4193
:10C4900041F470014FF0000030BD7FEA645C1ABFC8
:10C4A000194610467FEA655C1CBF0B46024650EAFF
:10C4B000013406BF52EA033591EA030F41F400212B
:10C4C00030BD00BF90F0000F04BF0021704730B5B1
:10C4D0004FF4806404F132044FF000054FF0000186
:10C4E00050E700BF90F0000F04BF0021704730B547
:10C4F0004FF4806404F1320410F0004548BF40421C
:10C500004FF000013EE700BF42004FEAE2014FEA70
:10C5100031014FEA02701FBF12F07F4393F07F4F4B
:10C5200081F06051704732F07F4208BF704793F04E
:10C530007F4F04BF41F40021704730B54FF4607461
:10C5400001F0004521F000411CE700BF50EA010264
:10C5500008BF704730B54FF000050AE050EA01020D
:10C5600008BF704730B511F0004502D5404261EB7D
:10C5700041014FF4806404F132045FEA915C3FF4BE
:10C58000D8AE4FF003025FEADC0C18BF03325FEA5B
:10C59000DC0C18BF033202EBDC02C2F1200300FA0C
:10C5A00003FC20FA02F001FA03FE40EA0E0021FA31
:10C5B00002F11444BDE600BF70B54FF0FF0C4CF41F
:10C5C000E06C1CEA11541DBF1CEA135594EA0C0FD1
:10C5D00095EA0C0F00F0DEF82C4481EA030621EA0C
:10C5E0004C5123EA4C5350EA013518BF52EA033547
:10C5F00041F4801143F4801338D0A0FB02CE4FF0F9
:10C600000005E1FB02E506F00042E0FB03E54FF028
:10C610000006E1FB03569CF0000F18BF4EF0010E20
:10C62000A4F1FF04B6F5007F64F5407404D25FEA1C
:10C630004E0E6D4146EB060642EAC62141EA5551CF
:10C640004FEAC52040EA5E504FEACE2EB4F1FD0C11
:10C6500088BFBCF5E06F1ED8BEF1004F08BF5FEA8F
:10C66000500E50F1000041EB045170BD06F0004641
:10C6700046EA010140EA020081EA0301B4EB5C04EE
:10C68000C2BFD4EB0C0541EA045170BD41F48011E6
:10C690004FF0000E013C00F3AB8014F1360FDEBF0B
:10C6A000002001F0004170BDC4F10004203C35DAE7
:10C6B0000C341BDC04F11404C4F1200500FA05F36A
:10C6C00020FA04F001FA05F240EA020001F000420B
:10C6D00021F0004110EBD37021FA04F642EB060181
:10C6E0005EEA430E08BF20EAD37070BDC4F10C04AB
:10C6F000C4F1200500FA04F320FA05F001FA04F26F
:10C7000040EA020001F0004110EBD37041F100015A
:10C710005EEA430E08BF20EAD37070BDC4F1200565
:10C7200000FA05F24EEA020E20FA04F301FA05F2CD
:10C7300043EA020321FA04F001F0004121FA04F275
:10C7400020EA020000EBD3705EEA430E08BF20EA45
:10C75000D37070BD94F0000F0FD101F0004640007F
:10C7600041EB010111F4801F08BF013CF7D041EA01
:10C77000060195F0000F18BF704703F00046520005
:10C7800043EB030313F4801F08BF013DF7D043EAD6
:10C790000603704794EA0C0F0CEA135518BF95EA8C
:10C7A0000C0F0CD050EA410618BF52EA4306D1D113
:10C7B00081EA030101F000414FF0000070BD50EA32
:10C7C000410606BF1046194652EA430619D094EABC
:10C7D0000C0F02D150EA013613D195EA0C0F05D1A6
:10C7E00052EA03361CBF104619460AD181EA0301FA
:10C7F00001F0004141F0FE4141F470014FF00000B2
:10C8000070BD41F0FE4141F4780170BD70B54FF04C
:10C81000FF0C4CF4E06C1CEA11541DBF1CEA1355CC
:10C8200094EA0C0F95EA0C0F00F0A7F8A4EB0504AE
:10C8300081EA030E52EA03354FEA013100F08880A5
:10C840004FEA03334FF0805545EA131343EA12636E
:10C850004FEA022245EA111545EA10654FEA002623
:10C860000EF000419D4208BF964244F1FD0404F5DC
:10C87000407402D25B084FEA3202B61A65EB030538
:10C880005B084FEA32024FF480104FF4002CB6EBF5
:10C89000020E75EB030E22BFB61A754640EA0C0075
:10C8A0005B084FEA3202B6EB020E75EB030E22BFB5
:10C8B000B61A754640EA5C005B084FEA3202B6EBF6
:10C8C000020E75EB030E22BFB61A754640EA9C00B5
:10C8D0005B084FEA3202B6EB020E75EB030E22BF85
:10C8E000B61A754640EADC0055EA060E18D04FEA43
:10C8F000051545EA16754FEA06164FEAC30343EAE3
:10C9000052734FEAC2025FEA1C1CC0D111F4801FAF
:10C910000BD141EA00014FF000004FF0004CB6E7A8
:10C9200011F4801F04BF01430020B4F1FD0C88BF47
:10C93000BCF5E06F3FF6AFAEB5EB030C04BFB6EB52
:10C94000020C5FEA500C50F1000041EB045170BD45
:10C950000EF0004E4EEA113114EB5C04C2BFD4EB72
:10C960000C0541EA045170BD41F480114FF0000EF6
:10C97000013C90E645EA060E8DE60CEA135594EA72
:10C980000C0F08BF95EA0C0F3FF43BAF94EA0C0F75
:10C990000AD150EA01347FF434AF95EA0C0F7FF4EA
:10C9A00025AF104619462CE795EA0C0F06D152EA3E
:10C9B00003353FF4FDAE1046194622E750EA410622
:10C9C00018BF52EA43067FF4C5AE50EA41047FF433
:10C9D0000DAF52EA43057FF4EBAE12E74FF0FF3C98
:10C9E00006E000BF4FF0010C02E000BF4FF0010C69
:10C9F0004DF804CD4FEA410C7FEA6C5C4FEA430CE2
:10CA000018BF7FEA6C5C1BD001B050EA410C0CBF30
:10CA100052EA430C91EA030F02BF90EA020F002092
:10CA2000704710F1000F91EA030F58BF994208BFF9
:10CA300090422CBFD8176FEAE37040F001007047B6
:10CA40004FEA410C7FEA6C5C02D150EA013C07D10D
:10CA50004FEA430C7FEA6C5CD6D152EA033CD3D058
:10CA60005DF8040B704700BF8446104662468C4652
:10CA70001946634600E000BF01B5FFF7B7FF002885
:10CA800048BF10F1000F01BD4DF808EDFFF7F4FFAE
:10CA90000CBF012000205DF808FB00BF4DF808ED39
:10CAA000FFF7EAFF34BF012000205DF808FB00BF5C
:10CAB0004DF808EDFFF7E0FF94BF012000205DF87E
:10CAC00008FB00BF4DF808EDFFF7CEFF94BF012033
:10CAD00000205DF808FB00BF4DF808EDFFF7C4FF2C
:10CAE00034BF012000205DF808FB00BF4FEA410C75
:10CAF0007FEA6C5C02D150EA013C0AD14FEA430C58
:10CB00007FEA6C5C02D152EA033C02D14FF0000094
:10CB100070474FF0010070474FEA410212F50012D2
:10CB200015D211D56FF47873B3EB625212D94FEA74
:10CB3000C12343F0004343EA505311F0004F23FA5E
:10CB400002F018BF404270474FF00000704750EAB3
:10CB5000013005D111F0004008BF6FF00040704770
:10CB60004FF00000704700BF4A0011D212F50012CA
:10CB700011D20DD56FF47873B3EB62520ED44FEA35
:10CB8000C12343F0004343EA505323FA02F07047B5
:10CB90004FF00000704750EA013002D14FF0FF30F3
:10CBA00070474FF0000070474FEA4102B2F1E04396
:10CBB00024BFB3F5001CDCF1FE5C0DD901F0004C84
:10CBC0004FEAC0024CEA5070B2F1004F40EB8300D4
:10CBD00008BF20F00100704711F0804F21D113F100
:10CBE0003872BCBF01F00040704741F480114FEA39
:10CBF0005252C2F11802C2F1200C10FA0CF320FAC2
:10CC000002F018BF40F001004FEAC1234FEAD323DE
:10CC100003FA0CFC40EA0C0023FA02F34FEA430348
:10CC2000CCE77FEA625307D150EA01331EBF4FF0D1
:10CC3000FE4040F44000704701F0004040F0FE40EC
:10CC400040F40000704700BF80F0004002E000BFE9
:10CC500081F0004142001FBF5FEA410392EA030FE7
:10CC60007FEA226C7FEA236C6AD04FEA1262D2EB31
:10CC70001363C1BFD218414048404140B8BF5B4236
:10CC8000192B88BF704710F0004F40F4000020F0CF
:10CC90007F4018BF404211F0004F41F4000121F0E5
:10CCA0007F4118BF494292EA030F3FD0A2F101022F
:10CCB00041FA03FC10EB0C00C3F1200301FA03F16D
:10CCC00000F0004302D5494260EB4000B0F5000F90
:10CCD00013D3B0F1807F06D340084FEA310102F14F
:10CCE0000102FE2A51D2B1F1004F40EBC25008BF01
:10CCF00020F0010040EA03007047490040EB0000CB
:10CD0000013A28BFB0F5000FEDD2B0FA80FCACF1CB
:10CD1000080CB2EB0C0200FA0CF0AABF00EBC250F8
:10CD200052421843BCBFD0401843704792F0000FE6
:10CD300081F4000106BF80F400000132013BB5E739
:10CD40004FEA41037FEA226C18BF7FEA236C21D0AF
:10CD500092EA030F04D092F0000F08BF0846704714
:10CD600090EA010F1CBF0020704712F07F4F04D1E2
:10CD7000400028BF40F00040704712F100723CBFF5
:10CD800000F50000704700F0004343F0FE4040F41F
:10CD9000000070477FEA226216BF08467FEA2363DD
:10CDA0000146420206BF5FEA412390EA010F40F4C8
:10CDB000800070474FF0000304E000BF10F0004314
:10CDC00048BF40425FEA000C08BF704743F09643FB
:10CDD00001464FF000001CE050EA010208BF704716
:10CDE0004FF000030AE000BF50EA010208BF70479D
:10CDF00011F0004302D5404261EB41015FEA010CB2
:10CE000002BF84460146002043F0B64308BFA3F1A9
:10CE10008053A3F50003BCFA8CF2083AA3EBC2538B
:10CE200010DB01FA02FC634400FA02FCC2F12002AA
:10CE3000BCF1004F20FA02F243EB020008BF20F0E1
:10CE40000100704702F1200201FA02FCC2F1200247
:10CE500050EA4C0021FA02F243EB020008BF20EA3C
:10CE6000DC7070477BB972B90029BEBF00204FF05B
:10CE7000004106E008BF00281CBF6FF000414FF0E2
:10CE8000FF3000F007BAADF1080C6DE904CE0029BF
:10CE900009DB002B1ADB00F095F8DDF804E0DDE992
:10CEA000022304B07047404261EB4101002B1BDBC1
:10CEB00000F088F8DDF804E0DDE9022304B0404228
:10CEC00061EB4101524263EB43037047524263EB13
:10CED000430300F077F8DDF804E0DDE9022304B055
:10CEE000404261EB41017047524263EB430300F063
:10CEF00069F8DDF804E0DDE9022304B0524263EB97
:10CF00004303704753B94AB9002908BF00281CBF22
:10CF10004FF0FF314FF0FF3000F0BCB9ADF1080C1D
:10CF20006DE904CE00F04EF8DDF804E0DDE90223FF
:10CF300004B07047430803F05533C01A830803F068
:10CF4000333300F03330184400EB101000F00F3092
:10CF500000EB002000EB0040000E704707EE900A47
:10CF6000F5EEC07AF1EE10FA01D400F00BB8F1EE54
:10CF7000677A08B517EE900A00F004F8404261EBBA
:10CF8000410108BDD0B5FFF7BFFA0C4B00220646A1
:10CF90000F46FFF711FBFFF7E7FD0446FFF792FA94
:10CFA000074B0022FFF708FB02460B463046394686
:10CFB000FFF74AF9FFF7D8FD2146D0BD0000F03D4C
:10CFC0000000F0412DE9F047089D04468E46002BF5
:10CFD0004DD18A42944669D9B2FA82F252B101FA2D
:10CFE00002F3C2F1200120FA01F10CFA02FC41EA3D
:10CFF000030E94404FEA1C48210CBEFBF8F61FFAC2
:10D000008CF708FB16E341EA034306FB07F199425C
:10D010000AD91CEB030306F1FF3080F01F8199420F
:10D0200040F21C81023E63445B1AA4B2B3FBF8F0E9
:10D0300008FB103344EA034400FB07F7A7420AD970
:10D040001CEB040400F1FF3380F00A81A74240F298
:10D0500007816444023840EA0640E41B00261DB103
:10D06000D4400023C5E900433146BDE8F0878B4238
:10D0700009D9002D00F0EF800026C5E900013046F7
:10D080003146BDE8F087B3FA83F6002E4AD18B42D1
:10D0900002D3824200F2F980841A61EB030301207B
:10D0A0009E46002DE0D0C5E9004EDDE702B9FFDE67
:10D0B000B2FA82F2002A40F09280A1EB0C014FEA12
:10D0C0001C471FFA8CFE0126200CB1FBF7F307FB6F
:10D0D000131140EA01410EFB03F0884208D91CEB12
:10D0E000010103F1FF3802D2884200F2CB804346AF
:10D0F000091AA4B2B1FBF7F007FB101144EA01448E
:10D100000EFB00FEA64508D91CEB040400F1FF311C
:10D1100002D2A64500F2BB800846A4EB0E0440EA0A
:10D1200003409CE7C6F12007B34022FA07FC4CEA13
:10D13000030C20FA07F401FA06F31C43F9404FEA06
:10D140001C4900FA06F3B1FBF9F8200C1FFA8CFE1B
:10D1500009FB181140EA014108FB0EF0884202FA6F
:10D1600006F20BD91CEB010108F1FF3A80F0888030
:10D17000884240F28580A8F102086144091AA4B2ED
:10D18000B1FBF9F009FB101144EA014100FB0EFE6E
:10D190008E4508D91CEB010100F1FF346CD28E459D
:10D1A0006AD90238614440EA0840A0FB0294A1EB2E
:10D1B0000E01A142C846A64656D353D05DB1B3EB8B
:10D1C000080261EB0E0101FA07F722FA06F3F140BB
:10D1D0001F43C5E9007100263146BDE8F087C2F162
:10D1E0002003D8400CFA02FC21FA03F391400143DA
:10D1F0004FEA1C471FFA8CFEB3FBF7F007FB103613
:10D200000B0C43EA064300FB0EF69E4204FA02F4BE
:10D2100008D91CEB030300F1FF382FD29E422DD911
:10D22000023863449B1B89B2B3FBF7F607FB163346
:10D2300041EA034106FB0EF38B4208D91CEB0101C6
:10D2400006F1FF3816D28B4214D9023E6144C91A46
:10D2500046EA004638E72E46284605E70646E3E656
:10D260001846F8E64B45A9D2B9EB020864EB0C0E60
:10D270000138A3E74646EAE7204694E74046D1E76F
:10D28000D0467BE7023B614432E7304609E764441D
:10D29000023842E7704700BF02E000F000F8FEE706
:10D2A00072B6374880F30888364880F309883648D4
:10D2B0003649086040F20000CCF200004EF63471AE
:10D2C000CEF200010860BFF34F8FBFF36F8F40F2C3
:10D2D0000000C0F2F0004EF68851CEF20001086066
:10D2E000BFF34F8FBFF36F8F4FF00000E1EE100AD6
:10D2F0004EF63C71CEF200010860062080F31488DF
:10D30000BFF36F8FACF0CEFDADF018FD4FF0553090
:10D310001F491B4A91423CBF41F8040BFAE71D49E3
:10D32000184A91423CBF41F8040BFAE71A491B4ADC
:10D330001B4B9A423EBF51F8040B42F8040BF8E72E
:10D3400000201849184A91423CBF41F8040BFAE703
:10D35000ACF0ACFDADF046FD144C154DAC4203DA1B
:10D3600054F8041B8847F9E702F0D8F8114C124D25
:10D37000AC4203DA54F8041B8847F9E7ACF094BDDB
:10D38000000600200022002000C0000808ED00E098
:10D39000000000200006002090490E080022002016
:10D3A000AC2B0020B02B0020D04E0120E0C10008A3
:10D3B0003CC200083CC200083CC200082DE9F04F06
:10D3C0002DED108AC1F80CD0C3689D46BDEC108AC3
:10D3D000BDE8F08F002383F311882846A047002082
:10D3E000ABF058FDFEE7ABF0C5FB00DFFEE7000049
:10D3F00001F0FF01102A2BDB10F0070F08D010F806
:10D40000013B013A8B422DD010F0070F42B3F6D109
:10D41000F0B441EA012141EA014122F007047FF022
:10D4200000070023F0E80256083C85EA010586EA79
:10D43000010685FA47F5A3FA87F586FA47F6A5FAB5
:10D4400087F68EB9EED1F0BC01F0FF0102F00702C1
:10D4500032B110F8013B013A83EA010313B1F8D16C
:10D460000020704701387047002D06BF354603384D
:10D47000073815F0010F07D1013015F4807F02BF86
:10D48000013015F4C03F0130F0BC0138704700BFD7
:10D4900010F8012B11F8013B012A28BF9A42F7D05E
:10D4A000D01A7047034613F8012B002AFBD1181A33
:10D4B0000138704738B50022002304460D46FFF7B7
:10D4C000EDFA28B920462946BDE8384000F00AB8F0
:10D4D000204605F1004100F005F8404261EB4101B2
:10D4E00038BD00BFD0B50C4B002206460F46FFF7F3
:10D4F00063F8FFF739FB0446FEF7E4FF074B002211
:10D50000FFF75AF802460B4630463946FEF79CFEB6
:10D51000FFF72AFB2146D0BD0000F03D0000F0419E
:10D52000036800221B6818477FB503914021054618
:10D5300079F0BAFD039A18B90124204604B070BDF1
:10D54000134E039296F9A235002BF5D05EF07EF8CB
:10D55000437A039A53B95EF079F8847A039A2CB926
:10D560000C4B4021284679F0A7FDE6E7D6F8F03EBF
:10D57000B6F9A415B3F906309942DDDD064B0093E8
:10D580004021064B284679F097FD0024D5E700BFDF
:10D59000B84B002060240C087F240C086D240C0874
:10D5A000F0B50D469DB02021044679F07DFD0028A0
:10D5B00000F0A180514E96F9A235ABB1D6F8F02E0D
:10D5C000B6F9A435B2F90A1003F10A02914203DD5B
:10D5D00040F28D32934207DC494B2A4620212046F7
:10D5E00079F06AFD002084E096F99135022B05D18F
:10D5F000444B2A462021204679F05EFDB6F864357A
:10D60000A3F57A739BB241F6583293420FD83E4F3E
:10D61000D7F8583D06F5BA6292ED007AD3ED097A53
:10D62000B4EEE77AF1EE10FA03DD384BD5E7384B6C
:10D63000D3E706F2D45292ED007AD3ED0B7AB4EE32
:10D64000E77AF1EE10FAF0DCB6F99E35002B01DC3A
:10D65000304BC2E796F830260D2A06D801239340B6
:10D6600013F4215F01D02C4BB7E72C480EF004FED9
:10D67000012806D1D7F8640D80F022FD98B1012869
:10D680001AD00021602204A80391B0F0C1FB244904
:10D69000D7F8600D642303AA80F034F900BB03AB14
:10D6A0000093204B02E0204B0093204B2A46202180
:10D6B000204679F001FD95E796F8043F73B11C48C8
:10D6C00019214BF015FC48B11948D6F87C65192191
:10D6D0004BF034FC8642D4DD164BE5E7164BE3E70E
:10D6E0001649D7F8580D642303AA7CF0CBFF002815
:10D6F000D5D01DB0F0BD0120FBE700BFB84B002026
:10D7000088240C089B240C08B86B0020D3240C0838
:10D71000C3240C08ED240C0802250C08008100200D
:10D720007C250C0880250C0847250C0822250C08B0
:10D73000B83C002066250C0857250C0892250C08DB
:10D7400007B5044882F014F800F0010003B05DF85A
:10D7500004FB00BFF47800202DE9F043DFF844918A
:10D760000446D9F8B4020368A5B01B690D46984772
:10D77000804614F02DFB0021074660220CA80B9177
:10D78000B0F046FB64230BAA4146384613F022FE54
:10D79000064648B93A4A0BAB2946204679F094FE32
:10D7A000304625B0BDE8F083A9F6983067F0CCF993
:10D7B000B8F1000F03D194F91E30012B0AD1314882
:10D7C00011F00EFB80B9304A2946204679F07CFEE4
:10D7D0000026E5E710F0060FE2D0A9F5405011F061
:10D7E000FFFA08B9294AEFE703A9384613F028FCE5
:10D7F00028B19DF80D305B0601D5254AE4E7DFF836
:10D80000A880D8ED007AF5EEC07AF1EE10FA4FF06C
:10D810000003C5DD089309930A930DF1200907ABB6
:10D82000019305AA06AB04A9CDF80090384613F081
:10D83000E5FF48462FF08EF8D8ED007AB4EEE70AFF
:10D84000F1EE10FA01DB134ABEE79DED057AF4EE26
:10D85000C77AF1EE10FA01D80F4AB5E79DED047AC8
:10D86000F4EEC77AF1EE10FA01D80C4AACE79DED60
:10D87000067AF4EEC77AF1EE10FA91D8084AA3E7D7
:10D8800098250C08B82B0020A1250C08B8250C08F9
:10D89000DE250C08EC250C0801260C0817260C08C0
:10D8A0002D260C08B85B00207851002008B5064BE7
:10D8B00093F8CD329B0704D5044A79F005FE002089
:10D8C00008BD0120FCE700BFB85B002044260C081F
:10D8D00070B50C4C0546D4F8B40203685B690E467B
:10D8E000984710B10124204670BDA4F5405011F0B6
:10D8F00089FA04460028F5D1034A3146284679F0D2
:10D90000E3FDF0E7B85B002054260C082DE9F04653
:10D91000464ED6F8D83293F8CB509BB081468A4613
:10D9200065B9434B1B68986A03685B6B984704466C
:10D9300040B9404A5146484679F0C6FD28461BB0DA
:10D94000BDE8F0865DF082FE20215EF037FE58B122
:10D950005DF07CFE1F215EF031FE88B3364A5146F1
:10D96000484679F0B1FD002496F8AA3203F014037A
:10D97000142B05D1314A5146484679F0A5FD0024C3
:10D98000514648467AF044FC002188424FF060023C
:10D9900002A808BF0C460191B0F03AFAD6F8D802B6
:10D9A000036801AA1B6864219847054680B9244A88
:10D9B00001AB5146484679F087FD2C462546BDE728
:10D9C0005DF044FEA5215EF0F9FD0028C6D1CBE74D
:10D9D000002CF3D0D9F808303BB9D9F800305146C3
:10D9E0005B6B484698470446E8E751464846FFF7D0
:10D9F000D7FD514607464846FFF758FF3840C4B2A6
:10DA000051464846FFF790FD514604404846FFF70F
:10DA10005FFF51460440484679F07EFD5146044080
:10DA200048467AF00DFC0440C8E700BFB85B002010
:10DA30000083002068260C087F260C0899260C0815
:10DA4000B1260C0808B5FFF761FF054A92F8A81245
:10DA500060F3041182F8A812024A907108BD00BF59
:10DA6000B85B0020BD840020F7B505460F4679F06D
:10DA700057FB044678B10221284679F015FB06468B
:10DA800048B1154881F074FEC205C0F30723C0F306
:10DA9000002403D53446204603B0F0BD9B07F9D5DA
:10DAA0000D4881F073FE0D4B03F60853D3ED007A59
:10DAB000F8EEE77A30EE670ADFED097AB0EEC00AD9
:10DAC000B4EEE70AF1EE10FAE4DD064B3A46022125
:10DAD000284679F0F1FADEE7F4780020B86B0020F0
:10DAE0000000C842BC260C08F8B504460F4679F081
:10DAF000C9FD10210546204679F0D6FA58B12046D6
:10DB0000FFF71EFE064630B9044B3A461021204668
:10DB100079F0D2FA35462846F8BD00BFD0260C0869
:10DB200070B505460E4679F063FA044678B1802157
:10DB3000284679F0B9FA50B1074B93F82D3843B124
:10DB4000064B32468021284679F0B6FA002420465A
:10DB500070BD0446FBE700BFB85B0020E4260C085C
:10DB600038B50D4D0446D5F8640D80F0A9FA0128AA
:10DB700010D0D5F8640D80F0A3FA022804D0204616
:10DB8000BDE8384079F036BA04480EF075FB01283C
:10DB9000F5D138BD0020FCE7B86B002000810020E3
:10DBA000F0B5134C04F5005385B0D3F8E82E00927D
:10DBB000D3F8EC2E0192D3F8F02E0292D3F8F43E73
:10DBC00003936A4606460F467AF0D4FA394605466C
:10DBD000304679F0CBFA04F54054284094F8A83246
:10DBE00060F3C303C3F3C00084F8A83205B0F0BDEE
:10DBF000B82B00202DE9F84306462748DFF8A89007
:10DC0000DFF8A8800F4666F09FFF0446D9F8B402FB
:10DC100003681B699847054630B914F0060F03D115
:10DC2000D9F8E832022B09D13946304679F070FB39
:10DC3000054618B9002488F807400AE039463046FE
:10DC4000FFF78AFD04460028F4D02DB9012388F897
:10DC500007302046BDE8F8830821304679F024FAE1
:10DC60000028F3D00D4821F095FF0028EED00C4B92
:10DC700093F8E423B02101FB023203F50053B2F81C
:10DC8000EE21B3F992359A42E0DD064B3A4608217F
:10DC9000304679F011FACDE720500020D82C002032
:10DCA000B82B0020F8260C08B85B0020BD840020AB
:10DCB0002DE9F3410E46054614F08AF8804613F02C
:10DCC00081F9044640B9514A0121284679F0FCFB0C
:10DCD000204602B0BDE8F0814D4FD7F8B40203688A
:10DCE00031469B699847044658B9D7F8B40203688F
:10DCF0001B6C9847474A03460121284679F0E4FB0C
:10DD0000E6E7AB68002BE3D01021284679F0CCF988
:10DD100020B3D8ED937A98ED920A20EE270AADF061
:10DD200015FEDFED3D7AA7F5805320EE270AB3F903
:10DD30006435DFED3A7A20EE270A07EE903AF8EEE6
:10DD4000E77AB4EEE70AF1EE10FA07DD344B012270
:10DD50001021284679F0B0F90024B9E7402128467F
:10DD600079F0A2F938B3012E1ED0232E1CD0042E38
:10DD70001AD02C4CD4F8F03EB3F9083000EE103A2B
:10DD8000A4F50050B8EEC00A00F0BCFBB5EEC00A26
:10DD9000F1EE10FA1DDD244B00930122234B4021AC
:10DDA000284679F089F9D7E7D7F8B4020368DB6B26
:10DDB00098470028DDD01E4B1B68D86A0368DB69D2
:10DDC00098470128014619D11A4A284679F07CFB68
:10DDD000C2E7D7F8B40203685B69984730B1D4F85A
:10DDE000F03EB3F90830002BE5DDD4E7D7F8B402F4
:10DDF00003681B6898470B28DDD1F0E731462846B9
:10DE000002B0BDE8F04179F005BF00BF08270C085B
:10DE1000B85B002019270C08E02E65420000C842BC
:10DE20002D270C08B84B00207F240C0835270C0840
:10DE30000083002041270C0870B505460E46FFF709
:10DE40008BFC084B0446D87131462846FFF740FD4D
:10DE500031460028284608BF00247AF073F8204095
:10DE600070BD00BFBD8400202DE9F0414E4F3B78CE
:10DE7000002B40F096804D4CD4F8D85295F8CB50FA
:10DE800001263E701DB13B702846BDE8F0817AF056
:10DE90007FFA054630B9464A3870137843F00103DB
:10DEA0001370F1E753F0C8F9314652F0FFFAA4F5C8
:10DEB000405006F0A9FC3F4B1E710B2646F0D6FDE4
:10DEC000013E46F071FD16F0FF06F7D13A4800F02A
:10DED0007FFF13F07DFFD0F80022C4F8002390F8F4
:10DEE0007C32DA074DD413F0EBFA53F0A5F93C215C
:10DEF00053F0DEF80023C4F8C03200212E482F4E24
:10DF000000F0ECFF2C4810F06BFF01462C4885F028
:10DF1000A1FB2C4B1B68D86A036801211B6898473A
:10DF2000D4F8D80203689B6A98470121D4F8D80234
:10DF300082F0D8FB53F080F98046D4F8B40203682D
:10DF40001B68984796F824250146404652F086FC07
:10DF5000A6F5005006F04AFC50F098FB4FF0D4FEB6
:10DF600000233B7089F0B4FDB4F8AA3206F50056E0
:10DF700023F4087343F02003C6F8700DA4F8AA3206
:10DF800082E79B07B9D431460B4804F0E9FC0E4800
:10DF900081F0FCFBDFED0D7A20EE270A84EDB00A5C
:10DFA000ABE7002570E700BFB02B0020B85B002076
:10DFB000DC840020BD840020B82B0020B84B00205A
:10DFC0004459002000830020F47800200AD7233C25
:10DFD0002DE9F043374DD5F8D83293F8CB3087B0E0
:10DFE000002B64D062B1012901D0232908D195F911
:10DFF000A832002B04DB0024204607B0BDE8F083E4
:10E000007AF072FA04460028F5D013F0E1FE0746D4
:10E010001AF0F2FB8046384612F0E6FCD8B198F9C7
:10E020002430022B17D100264FF00009F1B203AAC9
:10E0300038460191CDF80C90CDF81090CDF81490A1
:10E0400013F064F8019918B103AA40461AF084F855
:10E050000136032EEAD11848012106F043FE164886
:10E06000012106F073FD0021D5F8D80282F03AFBB9
:10E07000124831F053F953F0DFF8002152F016FA4C
:10E080000F4B1B68D86A036800211B68984795F8F6
:10E09000AA32D5F8B4120B486FF3451385F8AA32AB
:10E0A0000B1A594259413C3087F038FFA4E701244C
:10E0B000A2E700BFB85B0020B82B0020347B002013
:10E0C00000830020D07C002010B5064CD4F8B402A8
:10E0D00003685B6A984718B1D4F8D83293F8CB003C
:10E0E00010BD00BFB85B002030B52DED028B89B0AC
:10E0F0000C46B0EE408AFFF7E7FF0546002838D00F
:10E10000B4EE488AF1EE10FA7CBFDFED1C8ADFED39
:10E110001C7A226863689FED1A0A68BFDFED198ACE
:10E12000029278BF68EE288A02A878BF68EEA78AB4
:10E13000D4ED027A0393F1EE677ACDED047A2EF0F6
:10E140000BF8B4EE488A00220123F1EE10FACDE973
:10E1500000238DED050ACDED060A9FED0A0A0A4857
:10E160008DED071AF0EE680A68BF134605A90CF09A
:10E1700063F9284609B0BDEC028B30BDE02E654244
:10E180000000C84200000000A47F002007B50191F4
:10E19000FFF79AFF30B10199044803B05DF804EB32
:10E1A00000F0F0BA03B05DF804FB00BFB82B00200C
:10E1B000014866F055BE00BF2050002008B500F5AC
:10E1C000405090F8A832C3F340128A420BD061F35A
:10E1D000451380F8A83231B153F02EF8BDE808405D
:10E1E0000F2152F065BF08BD70B500F540560546D9
:10E1F000D6F8E8328B420C4612D0012911D0022900
:10E2000016D059B953F018F81B2152F051FF0D4A9E
:10E2100005F5425006210C3055F0C0F8C6F8E8422A
:10E2200070BD53F009F81A2152F042FF064AEFE799
:10E23000012100F053FE52F0FFFF1D2152F038FF84
:10E24000024AE5E7AC270C08C1270C08BC270C08DC
:10E2500010B500F540520C4692F8CD3203F00101A2
:10E26000A14209D064F3000382F8CD32DB0704D465
:10E2700005F0ACFE024B9C7210BD06F07BF8F9E78E
:10E28000BD84002000F5405090F8CD3261F3410389
:10E2900080F8CD32014B1973704700BFBD84002058
:10E2A00010B504465DF0D2F920215EF087F904F53F
:10E2B0004053003893F8AA2218BF012060F382026D
:10E2C00083F8AA2210BD000010B5044650F0DEF914
:10E2D00004F54052436FD2F8D82204F58044D3604D
:10E2E000D4F8582D9366D4F8602DC2F8FC32D4F8D7
:10E2F000580D03685B6D9847D4F8580D0368BDE866
:10E3000010409B6D1847000070B52DED028B00F595
:10E3100040550446D5F8D83293F8CB30002B72D054
:10E3200095F9A832002B6EDB00F5804696F8A03EEA
:10E33000002B68D1D5F8B40203685B6998470028C0
:10E3400061D1324BD3F8B40203681B6898470B289D
:10E3500059D0D6F8603D9FED2E7AD3EDDB7AF0EE02
:10E36000E77AF4EEC77AF1EE10FA4CD5D5F8D80278
:10E37000443054F099FB0346DFED260A93ED000A82
:10E380009F20B7EE001A2AF0D9FCB5EEC00AF1EED4
:10E3900010FA38DD04F59A403C3081F003FADFEDE5
:10E3A0001E7AB0EEC00AB4EEE70AF1EE10FA2AD5F2
:10E3B00004F58054D6F8580DD4F8503807EE903A4A
:10E3C0000368D3F89830B8EEE78A984738EE400AE9
:10E3D000DFED127AB0EEC00AB4EEE70AF1EE10FA01
:10E3E00011D5D4F8543840F2E63203F2F3139342D5
:10E3F00009D8BDEC028BD5F8D8029FED090ABDE81B
:10E40000704083F059BCBDEC028B70BDB85B00203E
:10E410000000003400000000000070420000FA43D9
:10E420000AD7233C08B500F54050D0F8D80203685D
:10E430001B699847F6EE007A20EE270AB5EEC00A6F
:10E44000F1EE10FA48BF9FED010A08BD0000000080
:10E4500038B52DED028B00F580450446D5F8583DC2
:10E46000DFED110A93ED370A04F540547120B7EE41
:10E47000001A2AF063FCD4F8D802D5F8605D03686E
:10E480001B69B0EE408A984738EE400ABDEC028B1B
:10E49000DFED067A05F50575284620EE270ABDE86A
:10E4A000384070F007BF00BF0000000000007A4451
:10E4B00000F5B250D0ED9A5AD2ED007AD0ED9D6AB7
:10E4C00091ED006A26EEE77A67EEA57AA6EE257A48
:10E4D000E6EE267A81ED007AC2ED007A7047000000
:10E4E00000F50050B0F93C3E33B9B0F99E05002864
:10E4F000B8BF404280B2704783EAE370A0EBE3709C
:10E50000F8E7000070B52DED028B00F5405382B0A6
:10E5100093F8CD1211F00106044605D09FED2E0AA6
:10E5200002B0BDEC028B70BD8DED010A5DF08EF87E
:10E53000037F002BF2D0DFED298ADFED270A9DED66
:10E54000010AB0EE681A4E202AF0F8FB04F50055D7
:10E550004FF4C8723146B5F9A605B0EE408A2AF0EC
:10E560002BFCA5F8A605204610F0E8F9B5F9A6356C
:10E5700007EE900AB8EEE77A07EE903AF8EEE77AFF
:10E5800077EE676AB4EEE68AF1EE10FA0DD5204612
:10E59000FFF7A6FF07EE900A38EE668AB8EEE70AA4
:10E5A00020EE088A88EE260ABAE777EE877AB4EE7C
:10E5B000E78AF1EE10FAB1DDB5F99E3500EE103ABA
:10E5C00038EE678AB8EEC00A78EEE77A20EE088A5D
:10E5D00088EE270AA4E700BF0000000000007A448C
:10E5E00000207047002070477047000000F516506B
:10E5F00034307047004870474C570C0800F54050C5
:10E60000D0F8B40203681B6818470000034808608C
:10E610002F21117008221A60704700BF502B0C0880
:10E6200000F54050D0F8B4020368DB6C18470000D6
:10E6300000F54050D0F8B40203689B6C1847000006
:10E6400000F5405300F59E40D3F8B43240301B1A19
:10E65000584258417047000010B500F540500C4634
:10E66000D0F8B4020368DB6D984707EE900A9FED7F
:10E67000057AF8EE677A012067EE877AC4ED007AB2
:10E6800010BD00BF0AD7233C10B500F540500C4622
:10E69000D0F8B40203689B6D984707EE900A9FED8F
:10E6A000057AF8EEE77A012067EE877AC4ED007A02
:10E6B00010BD00BF0AD7233C10B500F540500C46F2
:10E6C000D0F8B40203681B6E9847DFED047A20EEA1
:10E6D000270A012084ED000A10BD00BF0AD7233CA1
:10E6E0005FF0F8BB63F09CBB5EF098BF4FF018BFC3
:10E6F00027F02EBF52F058B817F060B95CF0F8BBA5
:10E700005AF0A8BD0FF0B6BD10F00CBA06F022BD4D
:10E7100011F012BA05F0AEBC05F0FAB905F022B955
:10E7200061F058B90EF046BCFFF7EEBD0FF0E2BE47
:10E7300010F054B903F08EB80FF066BE0FF0E2BDD2
:10E740005CF0D2BE22F0C4BC06F0CAB802F052BCE3
:10E7500010F062B906F0B4BC04F0EEB806F00CBEDE
:10E7600005F092B906F06CB90FF010BDFFF7ACBD23
:10E7700028F0FCBA05F07CBE09F0BCBE09F0B8BDBB
:10E7800009F04CBD1FB500F540530446D3F8B40260
:10E79000039103685B6A984760B1DFED070A03994C
:10E7A000002304F5A7400093B0EE600A1A466C30CF
:10E7B0000BF098FC04B010BD0000000010B52DED6A
:10E7C000028B00F540530446D3F8B40203685B6A39
:10E7D000B0EE408A984720B90024BDEC028B204659
:10E7E00010BD9FED080A04F5A74028EE000A6C3022
:10E7F0000AF042FF04460028EED003480121FFF74B
:10E80000DDFCEAE70000C842B82B00200A4A92F972
:10E81000A822002A0B4605DA00228A604A600A60B4
:10E820000120704700F58040D0F8582D783207CA93
:10E8300083E80700F4E700BFB85B002070B5284B01
:10E84000036000F540530446D3F83C02254AC3F860
:10E850008C2008B119F008FA234B236004F500530B
:10E8600093F84C2242B9D3F848522DB1284626F0ED
:10E87000D5FB284619F0F4F904F5AB5077F048FFC2
:10E8800004F5A35008305FF0FFF804F5855504F552
:10E89000825614351436B54204D0183D284626F069
:10E8A00013F8F8E7114BC4F8983804F65C2053F0DD
:10E8B000D7FD04F5236053F0D3FD04F6042053F094
:10E8C000CFFD04F6581053F0CBFD04F62C1053F096
:10E8D000C7FD04F5106053F0C3FD204670BD00BFB6
:10E8E0000C2F0C0884350D0834160D08F4DD0C08C7
:10E8F00038B5494B044640F8043B5FF00BFC04F18B
:10E90000100016F0FDFC04F168004FF097FB04F5D1
:10E91000907021F067F804F5866015F0FDFA04F2B6
:10E92000545019F0A3F904F6980027F035FC04F5CB
:10E93000815010305FF0CCF904F588504AF0FEF9B0
:10E9400004F59D50103051F011FD04F5A35008302E
:10E950005FF082F804F5A550043017F0CDFF04F500
:10E96000AB5077F0C1FE04F5AB501C304FF028FFE0
:10E9700004F5AE50103060F077FD04F580530025AB
:10E98000264A83F8F45504F5B05004F5AF53143318
:10E990000430136045F07CFE04F5B250294618306F
:10E9A00011F0FEFC04F5E650183070F041FD04F55E
:10E9B00003501C3074F0DEFE04F50750343076F05E
:10E9C000EDFF04F50950183077F022FC04F50A50E9
:10E9D000303011F0E7FA04F51050103071F0DEF924
:10E9E00004F51150283065F053FF04F5005304F589
:10E9F000145083F824550A4D3C3078F049FA2B68BE
:10EA000013B1084889F032F82046074948F07EFFE4
:10EA10002C60204638BD00BF34160D08348E00200F
:10EA200098850020D0270C085C150D0810B50FF054
:10EA3000F9FE5CF00BFE0368BDE810405B68184708
:10EA4000FFF7F4BF10B5044606F098F8204610F022
:10EA5000F1F9204603F0BEFD2046BDE8104003F06A
:10EA600021BF0000FFF7EEBF70B500F54C5504352F
:10EA70000446284616F01EFB19F0BEFE90F9213020
:10EA800093B390F840337BB304F5405304F25456EB
:10EA9000D3F8D802443054F007F80346DFED130AE8
:10EAA00093ED000A9F20B7EE001A2AF047F994F977
:10EAB0008835012B284608BF86ED0E0A002116F086
:10EAC000BFF8DFED0B7A04F2AC7494ED287A20EEF7
:10EAD000270ADFED087AA7EE270A304684ED280AD8
:10EAE000BDE8704019F098BD70BD00BF0000000087
:10EAF000CDCCCC3D6666663FFFF7B6BF10B50121B1
:10EB0000044610F0D3F960B1114BD3F8B402036896
:10EB10009B6A984728B9204602F072F9204602F015
:10EB20007FF94FF40011204610F0C0F918B129F018
:10EB300051FB27F0FDF94FF48021204610F0B6F983
:10EB400028B129F047FBBDE8104027F0F5B810BD0B
:10EB5000B85B0020FFF7D2BF7FB500F580460446C2
:10EB6000D6F8580D9FED550A6C302DF0F5FA04F5E6
:10EB7000B25001A918308DED010ACDED020A8DEDDC
:10EB8000031A11F0B9FA0221204610F08FF970B182
:10EB90000121204610F08AF948B9494BD3F8B40254
:10EBA00003689B6A984710B9204602F029F90121B1
:10EBB000204610F07BF948B9414BD3F8B402036802
:10EBC0009B6A984710B9204602F02AF90121204695
:10EBD00010F06CF910B9204602F07CF94FF40031C6
:10EBE000204610F063F930B104F54053D3F8D80251
:10EBF00003685B6C98474021204610F057F968B1D4
:10EC000004F59D551035284650F06EFF04F58053ED
:10EC100093F9683413B1284651F0A8F84FF4806195
:10EC2000204610F043F920B104F59D50103050F00B
:10EC3000F5FF2021204610F039F958B104F5405570
:10EC4000D5F8B40203681B699847C0B1D6F8600DC7
:10EC50007DF094FD8021204610F028F9E0B129F0E4
:10EC6000B9FA27F08DF81021204610F01FF910B3E3
:10EC7000D6F8580D04B0BDE870407AF0C5BA204609
:10EC80000CF0EAF80028E1D1D5F8B40203685B691A
:10EC900098470028DAD0DDE74FF48021204610F0B5
:10ECA00005F90028DBD14FF40021204610F0FEF8D2
:10ECB0000028D4D1D7E704B070BD00BFE02E654274
:10ECC000B85B0020FFF748BF10B50121044610F0E3
:10ECD000EDF810B1204602F0FDF88021204610F03A
:10ECE000E5F858B14FF48021204610F0DFF828B93C
:10ECF00029F070FABDE8104027F01EB810BD0000E2
:10ED0000FFF7E2BF10B5044605F086FC204605F08B
:10ED1000E5FA204605F0C6FC204610F07BFF2046B1
:10ED2000BDE8104003F032BCFFF7ECBF70B54FF602
:10ED3000FF71044610F0BAF804F5405528B1D5F833
:10ED4000A8220721204602F0F7F8D5F8D83293F828
:10ED5000CB308BB92046FFF7A3FAD5F8D80204F5DB
:10ED60000053026893F83016166A93F8BA25B04734
:10ED7000D5F8D80282F06CFF5EF07AF95DF006FFFC
:10ED8000204610F045FF95F8A8320F4A04F580445C
:10ED9000DB43D4F8585DC3F3C01353712B681E6F67
:10EDA0004FF074FC4FF0DCF82846B047D4F8604DC3
:10EDB0004FF06CFC04F505744FF0D2F82046BDE826
:10EDC000704070F0DDB800BFBD840020FFF7AEBF1B
:10EDD00070B500F5805606F5CB6300F54054D3F8C6
:10EDE0005022C4F8EC22D3F85C32C4F8F032054665
:10EDF000D6F8580800F58C40503029F073FFD4F84D
:10EE0000EC32C4F8F832D4F8F032C4F8F402C4F8A2
:10EE1000FC324FF6FF71284610F048F838B1D6F8AA
:10EE2000582828460921BDE8704002F05BB870BD43
:10EE300030B500F54053D3F8E842002C4CD093F89D
:10EE4000A922D10748D56FF3000283F8A92200F563
:10EE50000052012CD2F8E81ED2F8EC5EB1F908405D
:10EE60000BBFD3EDBC5AD3EDBF5AD3EDBB7AD3ED74
:10EE7000BE7A07EE104AB5F9084006EE904A0CBF7C
:10EE8000F8EEE66AF8EEE66AB8EEC77A25EEE66ACC
:10EE900000F5B250A7EE276A67EEA67AD0ED9A6A1F
:10EEA000E7EE257A90ED9D7A27EE877AA6EE267A10
:10EEB000BDEEC77A17EE103A0B8190ED9A7AD2F830
:10EEC000EC3E67EE877A90ED9D7AE6EE477AFDEEAE
:10EED000E77A17EE902A1A8130BD000038B5054652
:10EEE0002DED028B00F5405471B128460FF022FB46
:10EEF000D4F8F4321B1A03F2F31340F2E6329342D1
:10EF00000CD8BDEC028B38BDD4F8E832022BF8D116
:10EF10000FF0F4FAB0F57A7FE7D2F2E7C4F8F40222
:10EF200000F58C405030642390FBF3F308EE103A68
:10EF3000DFED097AB8EEC88A28EE278AB0EE480AD3
:10EF4000ACF04AFB84EDBE0AB0EE480AACF09AFC85
:10EF500084EDBF0AD5E700BF35FA8E3C00F5B2500C
:10EF60000121183012F0A6BEFFF7F8BF10B5044615
:10EF70000FF0EAFC102120460FF098FF70B12046F8
:10EF800001F096FE4FF4001120460FF08FFF28B9D4
:10EF900029F020F9BDE8104026F0CABF10BD0000DE
:10EFA000FFF7E4BFF8B50446254606F00FF9224BFB
:10EFB00045F83C3B214BA465C4E91734204BC4E918
:10EFC0001934204BE36604F1800018F0E1FA04F1F3
:10EFD0009C0018F0DDFA04F1B80018F0D9FA4FF6E9
:10EFE000FF76194BC4F8CC30A4F8D06004F1D400FB
:10EFF00018F0CEFA4FF0FF37144B1549C4F83071B2
:10F0000028461D6048F082FCA4F87870A4F894604B
:10F0100004F5A27018F0BCFA04F5B07018F0B8FA54
:10F0200004F5BE7018F0B4FA002384F89031C4F8E7
:10F03000B4312046F8BD00BFB0820C0879E7000863
:10F040007DE7000881E700080000FFFF8C840020B6
:10F05000B4EB0C0810B5044606F0B8F80A4B236070
:10F060000123A38704F1400018F092FA04F1500044
:10F0700018F08EFA04F1600018F08AFA04F17000BA
:10F0800018F086FA204610BD588A0C082DE9F04386
:10F09000044689B0FFF72CFCA14B236004F5175000
:10F0A0001C3004F5005502F083F804F5165328339C
:10F0B000C5F8FC3E04F53C57062385F8003F4FF0A9
:10F0C0007C5805A907F10C00CDF8148053F082FD9F
:10F0D00007F1240087F0C6FE04F59A4600233C366B
:10F0E00085F83C3F04F53D57192304A985F8483FAE
:10F0F000C5F8446F07F11400CDF8108053F06AFD95
:10F1000007F12C0087F0AEFE4FF00108182304F53C
:10F110003E5004F5405785F8903F85F8848FC5F838
:10F120008C6F0C3724305EF0A7F804F54055384654
:10F1300077F06AFF06AE7B4BEB603146381D8DF8E9
:10F14000188049F001FA04F54150043077F046FF89
:10F15000754B764F6B6404F5415031461C30069771
:10F1600053F038FD04F5415031462830069753F0EE
:10F1700031FD04F541503146343004F542580697CC
:10F1800008F10C0853F026FD694BC5F88C3008F1E6
:10F19000080087F067FE04F5425704F544593837F4
:10F1A00009F11C093846143758F04CFA4F45F9D18B
:10F1B0000723C5F840320023A5F844324FF4CB7042
:10F1C00018F04CFDC5F83C0204F54950083087F0B2
:10F1D00049FE04F54A500C3087F044FE554B1A683E
:10F1E0000AB9C3F8008004F5AB47534BC5F88C301F
:10F1F000543704F54A50C5F8B472383079F094F9B0
:10F200004E4B07934FF07E584D4BC5F8EC82C5F836
:10F21000F8820694009304F54C5096E80C004FF4E5
:10F220000071043015F0C4FB04F56050303069F013
:10F23000BBFA04F59A4003A90C30CDF80C8053F0CA
:10F24000EFFC04F59A4003A92030CDF80C8053F070
:10F25000C1FC04F59A4004F580452C3018F098F96B
:10F2600005F63C5300261E605E609E6005F648531E
:10F2700004F59A401E605E609E6004F5B253183338
:10F28000C5F8543D002385F8753D4FF400417830B2
:10F2900016F01AF904F59B40783067F013FC04F57A
:10F2A0009C40343049F086FA264BC5F8343E04F5CC
:10F2B0009C40254B2549483004F59C48186008F1CE
:10F2C000680848F023FBFF2385F8783E85F8803EE8
:10F2D0001F49404648F01AFB1E4A136813B11E48E6
:10F2E00088F0C4FB1D491E48C2F8008004F59D4209
:10F2F000103208604FF0140E1FFA83FC0EFB0C0155
:10F300000133097C0029F7D1164BA3F800C0164B36
:10F31000D3F80080B8F1000F2AD01448E0E700BF0E
:10F320000C2F0C0858270C0898270C080000A04048
:10F3300084350D08B48800208C2F0C0875E7000870
:10F34000FC2E0C08A8270C08388E00200C420D0853
:10F35000C0C60D08C88E0020E4270C085885002080
:10F3600040710C08568500201485002005280C08E3
:10F3700004F59D401A6003A9574B0393243053F0C2
:10F3800029FC04F59D40443005F020FF534BC5F89F
:10F39000C43E04F59E40043005F018FF04F5A24970
:10F3A0004F4BC5F8043F04F59E4009F11809403061
:10F3B00004F5A045FFF7F6FD484605F007FF494B69
:10F3C000C5F8183109F13C0085F030FA464BC5F814
:10F3D000543104F5A540583005F0F8FE434BC5F80C
:10F3E000D83204F5A6401C3005F0F0FE404BC5F8BD
:10F3F0001C3304F5A64085F858835C3005F0E6FE22
:10F400003C4BC5F85C3304F5A740183005F0DEFE30
:10F41000394BC5F8983304F5A740C5F8D463C5F84F
:10F42000D863C5F8DC636C3005F0D0FE334BC5F80B
:10F43000EC3304F5A840C5F82884303005F0C6FE4A
:10F440002F4BC5F8303404F5A840783005F0BEFEE7
:10F450002C4BC5F8783404F5A940343005F0B6FEDD
:10F46000294BC5F8B43405F22C5304F5AA401E60AC
:10F470005E604830FFF7EEFD384605F0A7FE234BEF
:10F48000C5F8D43504F5AC40103005F09FFE204B94
:10F49000A5F84C8604F5AC40C5F810366030FFF78F
:10F4A000D9FD1C4BC5F86036012385F8E93605F512
:10F4B000DE6304F5AD401E605E609E607C3005F04A
:10F4C00085FE154BC5F8FC3605F23C7520462E60CE
:10F4D0006E6009B0BDE8F083CDCC4C3DAC7F0C082C
:10F4E00050800C0854830C08E4830C08A0840C089A
:10F4F00040850C08E0850C0878860C0818870C08F5
:10F50000A8870C0840880C08E0880C08B48B0C080D
:10F51000508D0C08108B0C08148E0C0838B5054B58
:10F520001C6823680A461D68034B01462046A8470D
:10F53000002038BD00830020B82B002010B587F0D4
:10F54000F7FE064C064B18602046FFF79FFD20464D
:10F55000044A0549BDE81040ABF018BFB82B0020A5
:10F5600000830020ACE500203DE800080120704742
:10F5700090F890308B4286BF00EB8100D0F8940069
:10F580000020704790F890308B4286BF00EB8100DE
:10F59000D0F8940000207047FA207047014B93F890
:10F5A0006A057047B84B0020034BD3F8E802431EAE
:10F5B00058425841704700BFB85B0020034BD3F856
:10F5C000E802831E58425841704700BFB85B0020D4
:10F5D000034BD3F8D80208B181F07CB901487047D9
:10F5E000B85B0020782F0C0838B5036A2E4D43F421
:10F5F000E0520262426A42F4E0524262826A42F49B
:10F60000E0528262D5F8602D0446E2B143F4F8433B
:10F610000362D5F8600D7CF071FC38B1636A43F485
:10F6200080436362A36A43F48043A362D5F8600D0C
:10F630007CF086FD38B1636A43F400536362A36AC9
:10F6400043F40053A362194B1D6845B119212846A4
:10F6500049F04EFC18B1236A43F480732362144BC3
:10F6600093F8043F6BB1636A43F48073636245B1FE
:10F670001921284649F074FC18B1A36A43F4807339
:10F68000A362236A43F080432362636A43F08043AA
:10F690006362084BD3F8D83293F8C1301BB9A36A20
:10F6A00043F08043A36238BDB86B0020648500201E
:10F6B000B84B0020B85B002013B54FF44470CDE97F
:10F6C000002118F0C5FA044628B1DDE900215AF0FE
:10F6D0000FFD024B2360204602B010BDCC310C0858
:10F6E00000207047704700000320704708207047D3
:10F6F000014B93F86C057047B84B0020034B93F90E
:10F700002406003818BF0120704700BFB84B002006
:10F71000014B93F96E057047B84B0020704700000D
:10F720007047000008B50C4BD3F8600D70B910237A
:10F730000A4AD2F8D82243F0400022B192F8CB20F6
:10F740000AB143F0C00040F0010008BD7CF0D6FBD8
:10F750000028ECD01823EBE7B86B0020B85B002042
:10F7600038B5C5780B46352D044628BF35253522DA
:10F7700000211846AEF04CFB2A4604F10C01BDE80E
:10F780003840AEF0FBBA00001FB5184C94F8FE13D9
:10F7900004F52C7010F0F2FB78B194F8FE1304F528
:10F7A0002C7010F0EDFB40B194F8FE1304F52C70B2
:10F7B00004B0BDE8104010F0E5BB002301930293B4
:10F7C000039312F005FB01A912F0DCF820B101A8A7
:10F7D0002DF0C0F804B010BD21F0B8FC90F8C43290
:10F7E000B02202FB030090ED2F0AF3E7B84B002094
:10F7F00008B50D4BD3F8D802A8B1443053F054F9F2
:10F80000034693ED000ADFED090A9F20B7EE001AC8
:10F8100029F094FADFED067A20EE270ABDEEC00A41
:10F8200010EE103A18B208BDB85B002000000000CE
:10F830000000C8422DE9F04FDFF8D880344F8DB07A
:10F840000446042508F5005617F8019BB8F9C4359D
:10F8500009F1FF3A43FA0AF3D90742D5207C54F064
:10F860002BFD8346207C55F02BFC00F121039B45AA
:10F8700005D2207C0DB0BDE8F04F53F099BFBAF12E
:10F88000030F2ED8DFE80AF00234393ED6F8580DBF
:10F8900003689B68984700F194035A69D3F800A065
:10F8A000D3F804E0D8681969D3F818C008925A6AE6
:10F8B0001B6ACDF82520CDF8293062222123CDE91D
:10F8C000003206900791207CCDF80CA0192303AAE2
:10F8D000C221CDF810E0CDF814C08DF8249054F07A
:10F8E00055FD013D15F0FF05AED10DB0BDE8F08F1F
:10F8F000D6F8580D0368DB68CCE7D6F8580D0368D6
:10F900001B69C7E7D6F8603D03F52A73C5E700BF5A
:10F9100098320C08B84B002013B5044607480191F3
:10F9200008F02EFC30B90199204602B0BDE8104025
:10F9300055F0EABD042002B010BD00BFF87A0020E7
:10F94000014808F077BA00BFF87A002059F030BBC0
:10F9500010B588B0044656F063FF0C4BD3F8D802BC
:10F9600038B90B4A0621204608B0BDE8104056F0D1
:10F970003FBF69461E2280F0B1FF064A6B46062152
:10F98000204656F035FF08B010BD00BFB85B002020
:10F99000C42F0C08227D0C08034A92F8E43E013380
:10F9A00082F8E43E56F040B8B84B002007B5084650
:10F9B000019117F0C3FE38B10448019902F09AFC96
:10F9C000002003B05DF804FB0420FAE70C8300205C
:10F9D000162A10B40C4605D0542A03D05DF8044B07
:10F9E00055F0B0BD0323237001205DF8044B704730
:10F9F00008B555F04DFF40F41C6040F00D0008BD07
:10FA000010B5044618F02CF9204610BD10B50C4C6A
:10FA100094F9A832002B0FDBD4F8B4020368DB6C36
:10FA2000984758B9D4F8B40203689B6C98470028EB
:10FA30000CBF0220032010BD0120FCE70420FAE7E0
:10FA4000B85B002010B44C69012C05D101465DF86B
:10FA5000044B034802F0CCBF5DF8044B55F0FEBFE9
:10FA6000B82B00202DE9F341B1F90430002B0646F4
:10FA70000C46154635DB4FF00008CDE900281A4F3B
:10FA8000B1F902209FED190AD7F8E81E4FF47A73F6
:10FA900059F068FD0123CDE900539FED140AB4F934
:10FAA0000020D7F8EC1E4FF47A73304659F05AFD17
:10FAB0009FED0F0AB4F90420D7F8F01E43463046F4
:10FAC000CDE9005859F04EFDCDE900589FED070AE9
:10FAD000B4F90620D7F8F41E4FF47A73304659F083
:10FAE00041FD02B0BDE8F081B84B00200000FA44AF
:10FAF00000007A44044B187820B9044B93F8AA020A
:10FB0000C0F38010704700BF5C840020B85B002009
:10FB10000B4B93F82D287AB993F8CD2292060BD18E
:10FB200093F9A822002A09DB93F8A93213F0200FD9
:10FB300014BF042001207047052070470320704740
:10FB4000B85B002008B5074B93F9B835032B03D0F9
:10FB5000BDE8084056F0C4BE034A022156F048FEF4
:10FB6000042008BDB84B0020DC2F0C08094BD3F84B
:10FB70002826920701D455F0D7BC03F5005303F5AE
:10FB8000536393ED000ADFED047AB8EEC00A20EE6D
:10FB9000270A7047B84B00200AD7233C10B594B011
:10FBA000044603A817F0F4FC1C4BD3F8B402036816
:10FBB00003A95B6D984778B3002103A817F080FD77
:10FBC00050B3247C87F084FF059BDDED047A089315
:10FBD000069B09930023F8EEE77A9FED117A0B93C9
:10FBE0000C930D930E930F931093119312934FF662
:10FBF000F853ADF84C300023962267EE877A8DF8E3
:10FC00004E303323CDE90032079007AA5721204612
:10FC1000CDED0A7A54F0BAFB14B010BDB85B0020E9
:10FC20000AD7233C30B52DED0A8B774C0546D4F826
:10FC3000B402036899B05B6A984700285BD004F56A
:10FC40000054D4F82834062B00F2C980DFE803F012
:10FC50000404045788AB53006C489FED6D8A0AF08A
:10FC600009FC9FED6C0A0168426883680D930BA83C
:10FC70000B910C922CF070FAF0EE489AB0EE40CA5C
:10FC8000F0EE60BAB0EE419AB0EE48AAF0EE488AC3
:10FC9000F0EE48AAB0EE48BA40F6F8542D7C87F052
:10FCA00017FF00231593169301238C228DF85E30E5
:10FCB0003323CDE900320B90B1EE499AF1EE688A18
:10FCC000B1EE488A0BAA552128468DED0CCACDED20
:10FCD0000DBA8DED0E9A8DED0FBACDED10AACDEDCA
:10FCE000118A8DED12AACDED139A8DED148AADF81F
:10FCF0005C4054F04BFB19B0BDEC0A8B30BD43485F
:10FD00000AF0B8FB9FED430A0168426883680D93CF
:10FD10000BA80B910C922CF01FFA3C48F0EE60BA45
:10FD2000B0EE419AB0EE40CA0AF0A8FB9FED390A46
:10FD30002CF012FA3548B0EE40BAF0EE60AAF0EEC0
:10FD4000418A0AF09FFB9FED330A2CF005FA4FF42D
:10FD50004064B0EE40AAF0EE609AB0EE418A9DE7B2
:10FD60002A489FED2B9A0AF089FB9FED2A0A2CF076
:10FD7000F3F92648B0EE40BAF0EE60AAF0EE418A00
:10FD80000AF080FB9FED230A2CF0E6F9F0EE49BA69
:10FD9000B0EE40AAF0EE609AB0EE418AB0EE49CAE9
:10FDA00040F607447AE71948DFED198A0AF06AFB42
:10FDB0009FED180A2CF0D0F9F0EE68AAB0EE40AA38
:10FDC000F0EE609AB0EE418AB0EE68BAB0EE689A92
:10FDD000F0EE68BAB0EE68CA40F63F445EE79FEDC9
:10FDE0000C8A0024F0EE489AB0EE48AAF0EE488A59
:10FDF000F0EE48AAB0EE48BAB0EE489AF0EE48BA33
:10FE0000B0EE48CA4AE700BFB85B0020A47F0020DC
:10FE1000000000000AD7233C2DE9F0412DED068BB0
:10FE20003B4D95F8A93299068CB004466AD505F584
:10FE300080579FED380AD7F8580DDFED378A6C30C0
:10FE40002CF08AF98DED041A21EE281AD5F8B46247
:10FE50008DED020ABDEEC11ACDED030A11EE103A86
:10FE60001DB2336894F810809B6D304660EE289A7E
:10FE700020EEA89A984707EE900AF8EEE77A304607
:10FE800067EEA87AFDEEE77A17EE903A1CB2336877
:10FE9000DB6D984707EE900AB8EE678AD7F8603DA9
:10FEA000DFED1E7A93ED0FAA336828EE288A1B6EC9
:10FEB000B4EEE78AF1EE10FA58BFB0EE678A30462A
:10FEC0009847BCEEC88A0023089318EE103AB72270
:10FED0002AEE28AA20EE280AADF82C301A23CDE904
:10FEE00000323E2105AA4046CDED059A8DED069AD9
:10FEF0008DED07AA8DED090AADF82850ADF82A401E
:10FF000054F044FA0CB0BDEC068BBDE8F08100BFA4
:10FF1000B85B00209F0CB3450AD7233C00FF7F4706
:10FF20002DE9F04F2DED028B1A4B047CD3F8583D90
:10FF30008DB0D3F88480D3F88870D3F88C60D3F870
:10FF4000905093ED258AD3F898B0D3F89CA0D3F8BD
:10FF5000DC9087F0BDFD00238DF82C301622252380
:10FF6000CDE90032029002AA532120468DED078A86
:10FF7000CDF820B0CDF824A0CDF82890CDF80C8095
:10FF800004970596069554F001FA0DB0BDEC028B6E
:10FF9000BDE8F08FB86B0020054BD3F8D8322BB1F9
:10FFA00093F8CA00002808BF02207047022070475B
:10FFB000B85B002008B5034BD3F8B40203681B6894
:10FFC000984708BDB85B0020024B93F8A902C0F324
:10FFD00040107047B85B002070B52C4E2DED028BA1
:10FFE0000546D6F8B40291ED018A036886B05B6AD3
:10FFF0000C46984750B9BDEEC88A18EE103ADB0798
:020000040801F1
:1000000004D4022006B0BDEC028B70BDD4E904011B
:1000100029F04CFF0028F4D002A817F0B9FA02AA80
:100020002146284659F00EFA0028EAD0184902A8BD
:1000300017F090FB03460028E3D1DFED160A00908D
:100040000246B0EE600A144802A90AF04BF8D8B193
:10005000D6F8B40203685B6A9847044608B10020EA
:10006000D0E70E480222042105F046FC60B1DFED26
:10007000090A094800942346B0EE600A224602A904
:100080000AF030F80028EAD10420BBE7B85B002072
:10009000E478002000000000A47F0020B82B00209E
:1000A00008B591F82030032B1CD1D1ED027A9FEDD9
:1000B0000E7A91ED060A0D4BF0EEE77AF4EEC77A70
:1000C000DFED0B7AD3F8B402F1EE10FA4CBF012148
:1000D000002120EE270A0FF0EDF9002814BF0020C0
:1000E000042008BD0220FCE700000034B85B0020BB
:1000F0000000C84210B52DED028BD1ED007AF5EE6F
:10010000C07AF1EE10FA82B00C4604DA042002B094
:10011000BDEC028B10BD9FED197AF4EEC77AF1EEBB
:1001200010FAF3D891ED030A9FED158AF0EEC07A2C
:10013000F4EEC87AF1EE10FA19D5D4ED037A11482D
:10014000D4ED010A94ED000AF4EEC87AD4ED027AF7
:10015000FDEEE77AF1EE10FACDED017A9DF904108B
:10016000ACBF0122002202F027F80020CFE7F7EE13
:10017000000A28F0DFFC0028C8D0DEE70000B44306
:10018000000000340C83002091ED010AB5EEC00A96
:10019000F1EE10FA08B501DC042008BD9FED107ADD
:1001A000104BD1ED007AD3F8B40220EE070A9FED90
:1001B0000E7A0368F4EEC77AF1EE10FA05DDDB6E15
:1001C00098470028E8D00020E7E79FED087AF4EE92
:1001D000C77AF1EE10FACCBF9B6E5B6EF0E700BF02
:1001E0000000C842B85B00209A9939403333F33F8E
:1001F00008B5D1ED007A9FED157AF0EEE77AF4EECE
:10020000C77AF1EE10FA1DD5D1ED017AF0EEE77A5A
:10021000F4EEC77AF1EE10FA14D50D48022203214C
:1002200005F06AFB80B10A480121FDF7C7FF0948C4
:1002300090F8803F012B03D000F67C702FF0C4FAB9
:10024000002000E0022008BD0420FCE7000000348C
:10025000B82B0020B86B002010B5D1ED007AFCEE71
:10026000E77A17EE903A9CB2012C02D0022C06D00D
:100270004CB9064821465FF06FFC002010BD0448D1
:1002800003F062F9F9E70420F8E700BF007A0020E4
:10029000B82B00201FB5D1ED017A0B7CFCEEE77A7C
:1002A000CDED027AD1ED007A0093FCEEE77AD1ED44
:1002B000030ACDED037A91ED020A9DF808309DF80E
:1002C0000C20014602480DF0C7FE05B05DF804FBA6
:1002D000B82B002010B50A4C94F8CD32DB070CD4B3
:1002E00002220521A4F5405005F006FB28B90222A0
:1002F0001146A4F5405005F0FFFA002010BD00BFE4
:10030000B85B002010B5D1ED007AFCEEE77A044628
:1003100017EE903A13F0FF030FD10F4BD3F8B4024E
:1003200003689B6F984708B1002010BD0B4A204618
:10033000062156F05DFA0420F7E7012B09D1064BA0
:10034000D3F8B4020368DB6F98470028ECD1044A65
:10035000EDE70220E9E700BFB85B002000300C08A1
:1003600010300C089FED0B7A01F10C03F1EC017ACF
:10037000F4EE677AF1EE10FA0AD6F0EEE77AF4EED0
:10038000C77AF1EE10FA03DC9942EFD101207047F1
:100390000020704700007A4430B52DED028B8DB0FF
:1003A0000023054603930493059311F011FD03A95F
:1003B00011F0E8FA58B311F00BFD00F55A7393E809
:1003C000070006AC84E80700DDED060A9DED070A8C
:1003D0002D7CF1EE600AB1EE400AABF01FFB204627
:1003E000B0EE408A2CF0B6FADFED0B7A089B0B9347
:1003F000012228EE278A0C23CDE90032A82109AA80
:1004000028468DED098A8DED0A0A53F0BFFF0DB025
:10041000BDEC028B30BD00BFE02E6542242938B50B
:1004200005460FD003D81B2907D1012412E040292B
:10043000FBD0A1F14203012BF7D92846BDE8384093
:1004400059F0C2BB0C2153F0C5F9044610B128463F
:10045000FFF7A2FF204638BD38B5194C94F8CD32CD
:10046000DB070D460AD4D4F8D83293F8CB303BB929
:100470000122114604F10C00FDF7F6FC002038BD06
:1004800094F9A832002B4FF0020212DA0521A4F5EC
:10049000405005F031FA0028F0D095ED000ADFED6C
:1004A000097AD4F8B40220EE270A01210FF002F8ED
:1004B000E4E70921A4F5405005F01EFADEE700BF8D
:1004C000B85B00200000C84210B5214C94F8CD3232
:1004D000DB070ED4D4F8D83293F8CB304BB194F973
:1004E000A832002B07DA0122082104F10C00FDF7E5
:1004F0006FFD002010BDD1ED007A9FED167AF0EE71
:10050000E77AF4EEC77AF1EE10FA0BD51248022220
:10051000112105F0F1F9A0B9022211460E4805F0AB
:10052000EBF9E6E7D4F8B40203681B68984704289F
:10053000DFD0D4F8B40203681B6898471428E5D1CB
:10054000D7E7064840F6C41108F0F0FAD1E700BF3B
:10055000B85B002000000034B82B0020907E002003
:1005600070B58B8BC12B05460C463CD8BB2B0CD8E9
:10057000542B6AD02ED8113B99B2052918D921469F
:100580002846BDE870405AF0B7B9BC3B052BF6D8F9
:1005900001A151F823F000BF850601089306010868
:1005A0007F0501087F0501082F06010839060108AB
:1005B000052BE4D801A151F823F000BF6F06010814
:1005C0007F0501087F0501087F060108E105010894
:1005D0004B060108732B22D0B22B24D0552BCED141
:1005E0000222092145E04AF21146B34237D00AD827
:1005F000D12B26D0B3F5967F35D0D02BBFD1BDE817
:100600007040FFF729BE4AF21246B34223D04AF2A5
:100610001346B342B3D1BDE87040FFF755BFBDE804
:100620007040FFF767BDBDE87040FFF7ADBD2146E4
:10063000BDE87040FFF7D0BC2146BDE87040FFF731
:1006400061BEBDE87040FFF725BE21462846BDE8E3
:100650007040FFF725BDBDE87040FFF7FDBEBDE867
:100660007040FFF737BEBDE87040FFF7C1BD022202
:1006700005210A4805F040F948B9042070BD02225E
:100680000621F6E70221064806F0A2FAF4E7002068
:10069000F4E70221024806F065FAEDE7B82B0020E6
:1006A000F87A002008B591ED007AF6EE007AB4EE03
:1006B000E77AF1EE10FA06DD044801220521FDF784
:1006C00087FC002008BD0420FCE700BFC45B0020BD
:1006D00030B52DED028BCD7893B0272D28BF27257F
:1006E0000C462722002108A8ADF092FB2A4604F10F
:1006F0000C0108A8ADF042FB424BD3F8B4020368EA
:100700005B6A9847002841D09DF8465068063DD462
:1007100000244FF07E532906049307940694059411
:1007200027D504A82AF0F0FFEA0701940294039465
:1007300005F006032ED4002B2ED10D9B01930E9BAA
:1007400002930F9B0393304809F07AFA9DED100A4B
:10075000044630B340F2ED40B7EE001AFFEE000A57
:1007600028F0ECFA2848234601AA04A909F070FAF7
:100770000CE0099B04930A9B05930B9B069304A82A
:100780000C9B07932AF0C6FF0028CDD113B0BDEC17
:10079000028B30BD062BD6D001211B4809F0ECF9A5
:1007A000F4E7DFED1A0A4FF49E60B7EE001A28F066
:1007B000C5FAF6EE000AB0EE408A28F0BBF9E8B9B7
:1007C000B6EE000A124BB4EEC08AF1EE10FAD3F87E
:1007D000643D08DD38EE400A30EE008A93ED070AEA
:1007E00028EE000ABEE730EE480AD3ED087A30EE74
:1007F000000AF0EEE77A27EEC00AB3E79FED030A9E
:10080000B0E700BFB85B0020A47F0020000000001C
:10081000B86B00202DE9F0439DB0814608460EA933
:10082000FEF79EFF844BD3F8B40203685B6A9847D7
:1008300050B19DF86C30012B09D0DA1F022A06D97D
:100840007E48012109F098F91DB0BDE8F083BDF89C
:100850006840A20504F0070604F0380704F4E075C8
:1008600001D5002DF0D04FF00008CDF81480CDF860
:100870001880CDF81C803EBB9FED716A9DED107A0B
:10088000DDED117ADDED0F6A27EE067A67EEC67AA6
:1008900066EE866A083B012BCDED056A8DED067A82
:1008A000CDED077A04D8674806AA05A9FDF700FE32
:1008B0009DF86C30073B022B06D863487EF062FF40
:1008C000014605A82BF068FCCDF82080CDF82480E7
:1008D000CDF82880F7B9DDED147A129B0893F1EE7C
:1008E000677A139B099308A94846CDED0A7AFFF76A
:1008F00039FD0028A4D09FED520A08A82BF080FCF7
:100900009DF86C30083B012B04D84E4809AA08A971
:10091000FDF7CEFDCDF82C80CDF83080CDF83480B9
:10092000EDB99FED476A9DED167ADDED177ADDEDA5
:10093000156A9DF86C3027EE067A67EEC67A66EE89
:10094000866A083B012BCDED0B6A8DED0C7ACDED5F
:100950000D7A04D83B480CAA0BA9FDF7A9FD14F4A5
:10096000806233D1DFED397A9DED180A9DF86C1065
:1009700020EE270ADFED327A0839012920EE270A16
:100980008CBF0021012114F4006305BFDFED2F7A35
:10099000DDED190ADFED2E0A60EEA70A04BFDFEDD8
:1009A000287A60EEA70AAEB9002F35D1B3FA83F3E7
:1009B000B2FA82F25B0952090291019300920BABE9
:1009C00008AA05A91D4809F045FA3DE79FED200A50
:1009D0000021D8E77FB9B3FA83F35B0901200093C4
:1009E000B2FA82F3CDE901105B0914480BAA08A9F9
:1009F00009F0C8FC28E7002D7FF422AF0120B3FAEC
:100A000083F3B2FA82F2CDE900105B090B48520978
:100A10000BA909F05FFC17E7002D3FF411AFB3FA03
:100A200083F3B2FA82F2CDE900165B09520905A9F7
:100A3000024809F091FA07E7B85B0020A47F002084
:100A40000000C842B82B0020F4780020E02E654258
:100A5000000000002DE9F047A2B08046084614A926
:100A6000FEF77EFE7E4BD3F8B40203685B6A9847BC
:100A7000C0B1BDF88040A30504F0070904F4E07795
:100A800000D57FB10CAE304616F082FDB9F1000FF3
:100A900029D1DDE9150129F009FA30B971480121A0
:100AA00009F06AF822B0BDE8F0879DF8841009AA21
:100AB000404658F0B1FC0028F0D0DDED177A9FEDEC
:100AC0006A7A099B009367EE877A10ADFDEEE77AAC
:100AD000DDE9151217EE903A284616F079FD95E8F3
:100AE0000F0086E80F00002514F0380A06950795D8
:100AF000089514D1DDED1A7A189B0693F1EE677A0A
:100B0000199B079306A94046CDED087AFFF72AFC0A
:100B10000028C3D09FED540A06A82BF071FB09955D
:100B20000A950B959FB99FED506A9DED1C7ADDEDFE
:100B30001D7ADDED1B6A27EE067A67EEC67A66EE51
:100B4000866A8DED0A7ACDED096ACDED0B7A14F443
:100B5000806805BFDFED457A9DED1E0A9FED440AD2
:100B600020EE270A04BFDFED407A20EE270A14F4B6
:100B7000006405BFDFED3D7ADDED1F0ADFED3C0AC5
:100B800060EEA70A04BFDFED387A60EEA70AB9F17C
:100B9000000F31D1BAF1000F52D13046CDED050A28
:100BA0008DED040A16F024FD03289DED040ADDED09
:100BB000050A3FF473AF10A93046CDED050A8DED5F
:100BC000040A10951195129516F072FE00283FF454
:100BD00065AFB4FA84F46409B8FA88F3DDED050A68
:100BE0009DED040ACDF804A000945B0906AA10A9A3
:100BF0001C4809F09FF955E7BAF1000F0FD1012306
:100C0000B4FA84F4CDE901A36409B8FA88F315486D
:100C100000945B0909AA06A909F0B4FB42E7002F7A
:100C20007FF43CAF0123CDE90073B8FA88F2B4FA3F
:100C300084F30C485B09520909A909F04BFB31E721
:100C4000002F3FF42BAFB4FA84F3B8FA88F2CDF852
:100C500000905B0952093146024809F043FA21E746
:100C6000B85B0020A47F00200000C842E02E65424F
:100C70000000000010B44B7A8C7ACA7A43EA04234D
:100C800043EA0243542B07D0562B09D0522B0BD1E9
:100C90005DF8044BFFF71CBD5DF8044BFFF7BABDD0
:100CA0005DF8044BFFF7D6BE5DF8044B58F0BCBCB2
:100CB0002DE9F0432DED028B00F540560446D6F8A1
:100CC000B402DFED4C8A036891B05B69984704F584
:100CD00080490027002840F08880D9F8603DD3ED96
:100CE000DE7A93EDD88AFDEEE77A28EE288A17EEB1
:100CF000903A1DB204F53E5808F1140801A9404687
:100D00000DF08AFF18B950F097FA3B4B0193372248
:100D1000002102A8ADF07CF8A3238DF808309523BC
:100D20008DF8093086F0DCFED9F8583DCDF80B007F
:100D3000D6F8D802D3F8DC20D3F8E030CDF80F1085
:100D40004430CDF81320CDF8173051F0ADFE0346F6
:100D5000DFED2A0A93ED000AB7EE001A9F2027F074
:100D6000EDFF10EE103AD6F8D802CDF81B3003682C
:100D70001B69984710EE103A04F59A46CDF81F30DB
:100D80003C3618EE103A3046CDF823307EF0FEFCAB
:100D900020EE280A404610EE103ACDF82730D9F858
:100DA000083DCDF82B30019BCDF82F300DF056FFCC
:100DB00010EE103A3046CDF83330CDF83770ADF83C
:100DC0003B507EF0EFFCBDEEC00A04F59D5010EEE6
:100DD000103A372202A91030ADF83D304FF07EFBBB
:100DE00011B0BDEC028BBDE8F08308EE107A00254F
:100DF00080E700BF0AD7233C2292CA7F0000000090
:100E000010B500F58044D4F8580D77F0A7FBD4F85E
:100E1000601DD4F8580DBDE8104077F005BC000007
:100E200070B54FF4805105460EF040F800284FD0C1
:100E300005F5804605F59D54D6F8580D03689B6866
:100E40009847103400F19402692120464FF0DEF9F2
:100E5000D6F8580D0368DB6898476A2100F19402C0
:100E600020464FF0D3F9D6F8580D03681B69984710
:100E70006B2100F1940220464FF0C8F9D6F8602D9E
:100E80006C21204602F52A724FF0C0F92021284635
:100E90000EF00CF8E0B105F54053D3F8B402036846
:100EA0001B69984778B1D6F8602D204690326E21A4
:100EB0004FF0ACF9D6F8602D2046BC32BDE870404A
:100EC0006F214FF0A3B9284609F0C6FF0028EAD1E8
:100ED00070BD000008B510F07BFFBDE8084010F0C1
:100EE00003BD00007FB50E464FF6FF710446154660
:100EF0000DF0DCFFE8B1102200216846ACF088FF5D
:100F0000A3238DF8003095238DF8013003238DF84D
:100F1000023086F0E5FD1022CDF8030004F59D5067
:100F2000CDF80710104469468DF80B6003954FF01B
:100F300055FB04B070BD00007FB50E464FF6FF7143
:100F4000044615460DF0B2FFE8B1102200216846B4
:100F5000ACF05EFFA3238DF8003095238DF80130AF
:100F600004238DF8023086F0BBFD1022CDF803007B
:100F700004F59D50CDF80710104469468DF80B60BC
:100F800003954FF02BFB04B070BD000030B52DED84
:100F9000048B87B004460D46182200216846B0EE47
:100FA000409AF0EE608AB0EE418AACF031FFA323A4
:100FB0008DF8003095238DF8013006238DF802302E
:100FC00086F08EFDCDF8030004F59D50CDF8071096
:100FD0001822694610308DF80B508DED039ACDED37
:100FE000048A8DED058A4FF079FA07B0BDEC048BC9
:100FF00030BD000010B54FF4801104460DF056FFCF
:1010000030B104F5B2501830BDE810400FF04EB9C1
:1010100010BD00002DE9F0438FB014460546894607
:101020003122002101A8DDE916769846ACF0F0FEE9
:10103000A3238DF8043095238DF8053008238DF80F
:10104000063086F04DFD2368049363680593A3681A
:1010500006933B68CDF81D307B68CDF82130BB6826
:10106000CDF825303368CDF80700CDF8293005F5E7
:101070009D507368CDF80B10CDF82D303122B36838
:101080008DF80F9001A910308DF81C80CDF831300B
:101090004FF024FA0FB0BDE8F083000070B52DEDDD
:1010A000068B8CB0144605460E462C22002101A862
:1010B000B0EE409AF0EE608AB0EE418AB0EE61AADE
:1010C000F0EE429AACF0A4FEA3238DF804309523F1
:1010D0008DF805300B238DF8063086F001FDDFED2D
:1010E0001A7A94ED007ACDF8070027EE277A29EED8
:1010F000279A8DED077A94ED017ACDF80B1027EE43
:10110000277A68EEA78A8DED087A94ED027A8DF839
:101110000F6028EE278A05F59D5067EE277A2C226E
:1011200001A910308DED049ACDED058A8DED068A6A
:10113000CDED097A8DED0AAACDED0B9A4FF0CEF9DF
:101140000CB0BDEC068B70BDE02E6542A020704750
:1011500030B5154B044689B004F59D55D3F8D80237
:10116000694610351E227FF0B9FB6A460F492846B2
:101170004FF050FB04F54053D3F8B40203681B68EA
:10118000984704F50053014693F8242528464FF06C
:1011900065FB04F5B250183011F058F804F5907062
:1011A0001FF03EF809B030BDB85B0020227D0C086E
:1011B0002A4B2B4A70B54360002343618361C361AE
:1011C000C363284B426303644FF08042264B436461
:1011D0000446826358305AF0B9F8244E244BA36574
:1011E000A82560195AF068FA66513035B5F56A7F5E
:1011F000F7D104F56A705BF01BFE002104F5F66080
:1012000081F05CFF1B4BC4F864389FED1B1ADFEDC7
:101210001B0A9FED1B0A04F6780077F091FF9FED03
:10122000161A9FED180AF0EE410A04F5096077F0EE
:1012300087FF9FED111A9FED130AF0EE410A04F6A5
:10124000A80077F07DFF20460F4946F05FFB20465F
:101250000E4946F05BFB204670BD00BFE83B002016
:101260000000C8410AD7233C0000E0408C7A0C08FB
:10127000A07A0C080C7D0020000000009A99993E8D
:101280000000B44300804A43506E0C08B0700C0854
:1012900070B54C4D4C49ADF50E7DD02206465AA88E
:1012A000ACF06CFD0FCD0EAC0FC40FCD0FC40FCD45
:1012B0000FC495E80F0084E80F0000245AAB1819FA
:1012C0000021B7EE000A103445F0EEFDD02CF5D128
:1012D0003E4B0FCB02AC84E80F0001A9204645F03D
:1012E00097FD90B19DF90430DFED396AE06807EEB3
:1012F000103AB8EEC77AF0EE007AE7EE267AB7EE4B
:10130000000A80EE270A46F0A9FE00240EAB181949
:1013100000211034B7EE000A45F0C6FD402CF5D18F
:101320002C49902236A8ACF029FD0022092136A8CC
:1013300045F066FE96F9E469D6B9274D0FCD1EAC8F
:101340000FC40FCD0FC40FCD0FC495E80F0084E874
:101350000F00324604211EA845F052FE9FED1F0AE1
:101360001F4846F07BFE1F48B7EE000A46F076FEA7
:101370001D4C9FED1E0A0FCC06AD0FC594E80F0063
:1013800085E80F00002106A845F08EFD9FED170AA5
:101390000021284645F088FD04F1100160221EA8B6
:1013A000ACF0ECFC00241EAB18190021B7EE000ACB
:1013B000103445F079FD602CF5D15BF04DFB0DF557
:1013C0000E7D70BDF4200C0824200C0834210C087C
:1013D000CDCCCC3D44210C08D4210C0800000000E9
:1013E000386D0C08476D0C0814220C0800003442BC
:1013F0002DE9F04790B00DF106011D205BF01EFCB9
:10140000002800F09E809DF80630614A0133DBB26F
:1014100011210BA88DF8063085F04AFD00220DF150
:1014200007010BA845F07AFA9DF80630594A1121B8
:1014300005460BA885F03CFD00220DF107010BA825
:1014400045F06CFA9DF80630534A112106460BA868
:1014500085F02EFD00220DF107010BA845F05EFA84
:101460009DF806304D4A03F03F03112107460BA8B3
:1014700085F01EFD00220DF107010BA845F04EFA84
:101480008046002D5DD0002E5BD0002F59D0002863
:1014900057D0284645F05AFC002852D1304645F036
:1014A00055FC00284DD1384645F050FC002848D165
:1014B000404645F04BFC002843D1394C94E80F00DE
:1014C0000DF10C0C10348CE80F0094E80F000DF1B6
:1014D0001C0989E80F0002A9604645F099FC98B301
:1014E000BDF8084002A9484645F092FC00284AD0C1
:1014F000BDF8083054BB23B340F2E2449C420FFADB
:1015000084FA0FFA83F927D80DF10A013046ADF8B5
:101510000A9047F099F80DF10A012846ADF80AA0A3
:1015200047F092F80DF10A013846ADF80AA047F0ED
:101530008BF800230DF10A014046ADF80A3047F060
:101540009DF810B0BDE8F0870024CBE740F2D662EA
:10155000002B08BF1346D1E70DF10A013046ADF864
:101560000AA047F071F80DF10A012846ADF80A907B
:1015700047F06AF80DF10A013846ADF80A9047F0D5
:1015800063F80123D6E7002CDBD040F2D663B5E741
:10159000586D0C08646D0C08706D0C087D6D0C089E
:1015A00094220C0837B500F51551782228310446ED
:1015B0004DF090FB00220C21254845F021FD2046EE
:1015C000FFF716FF04F515500022B7EE000A0221BE
:1015D0003C3045F09DFD012504F511511D4A009553
:1015E00000232831452045F00FFD1B4A1368D90719
:1015F00005D41A49156004F5105310330B6004F537
:101600001750164901221C3045F050FD012504F504
:101610009D51134A009500231031FD2045F0F4FC44
:10162000104B1A68D20705D40F4A1D6004F5AB545D
:101630001C3414600C48012145F054FD46F06CFB4D
:101640000A4A138843F00103138003B030BD00BF82
:10165000906D0C0818C10D080483002000220020A2
:10166000D01C0D08088300200C2200204885002093
:101670000F299DBF302303FB01005030002070472D
:10168000014B93F9AF057047B84B0020024B93F81C
:10169000CD0200F001007047B85B0020044BB3F8A6
:1016A0007435DB075ABF0069C0F340100020704753
:1016B000B84B0020014BD3F8F40E7047B84B002014
:1016C00008B503689B68984730B9044B93F9CC027E
:1016D000B0FA80F0400908BD0020FCE7B85B0020AC
:1016E00038B50D1E2DDB174C94F8002FEBB29A4243
:1016F00027D3D4F8FC3E0122595DA4F5005004F034
:10170000FBF8F0B159F0A2FF03215AF057FFC0B91E
:1017100059F09CFF0D215AF051FF90B994F994357E
:10172000EB40DB075CBF94F9AE15E940A4F500502F
:1017300048BF0221BDE8384058BF01F00101FCF765
:1017400053BD38BDB84B0020022A10B50C4605D158
:10175000BDE810400948352204F0CEB8084BD3F854
:10176000B40203681B689847A04205D159F06EFF88
:10177000BDE8104059F0F4BE10BD00BFB82B0020EA
:10178000B85B002029B1022907D1044BC3F8AC1281
:101790007047024B0122C3F8AC227047B85B0020AF
:1017A00031B1022907D1044B012283F8B0227047DE
:1017B000014B83F8B0127047B85B002010B500F5FC
:1017C0000053DFED186AD3F8EC2ED3F8E83EB2F9F7
:1017D0000820B3F908309FED147A07EE902AF8EE4E
:1017E000E77A0446C7EEA60A00F5B2500121183088
:1017F00007EE903AF8EEE77A60EE870A87EEA60ADF
:1018000020EE070A10F082FB4FF016FD26214FF064
:101810004FFC04F54250054ABDE8104006210C304B
:1018200051F0BCBD0000C84235FA8E3C5C780C0813
:1018300000F58042002382F8743D044A00F54250CE
:1018400013720621024A0C3051F0A8BDBD8400205D
:1018500068780C0870B500F58045044695F8741D4D
:10186000002957D02C4B2D4AD3F8B402904204D112
:10187000D3F8D83293F8CB3023B92046BDE8704076
:10188000FFF7D6BF264E95F8750D04F5405301229B
:1018900093F9A8323272D0BB002B3BDB85F8752D53
:1018A0000139C9B204F5005385F8741DD3F8EC2E44
:1018B000D3F8E83EB2F90820DFED1A6AB3F9083030
:1018C0009FED197A07EE902AF8EEE77AB1FA81F1E6
:1018D000C7EEA60A04F5B2504909183007EE903A4F
:1018E000F8EEE77A60EE870A87EEA60A20EE070A8E
:1018F00010F00CFB95F8743D63B904F54250337257
:101900000A4ABDE8704006210C3051F047BD002B5B
:10191000C6DAB2E770BD00BFB85B00208C81002042
:10192000BD84002000007A4535FA8E3C7C780C0896
:101930006D2900F3E380012901DC5AF08DBC8B1E78
:101940006B2BFAD80FF2040C5CF823F05B1B010838
:10195000551B01085B1B01085B1B01083B190108B3
:101960005B1B01083B1901083B190108551B0108C5
:101970003B1901085B1B0108551B0108551B010899
:101980003B1901085B1B01085B1B01085B1B01087D
:101990003B1901083B190108551B01085B1B010895
:1019A000551B01083B190108551B0108551B01086F
:1019B0003B1901083B1901083B1901083B190108B3
:1019C0003B190108551B01085B1B01083B19010865
:1019D0003B1901083B1901085B1B01083B19010871
:1019E000551B01083B1901083B1901085B1B010845
:1019F000551B01083B1901083B1901083B19010857
:101A00005B1B01085B1B01085B1B01083B190108FC
:101A10003B1901085B1B01083B1901083B19010830
:101A20005B1B01085B1B01085B1B01083B190108DC
:101A30003B1901085B1B01085B1B01083B190108EE
:101A40003B1901083B1901083B1901083B19010822
:101A50003B1901085B1B01085B1B01085B1B0108AC
:101A60005B1B01085B1B01085B1B01083B1901089C
:101A7000551B0108551B01083B1901083B190108BA
:101A80003B1901083B1901083B1901083B190108E2
:101A90005B1B0108551B01083B1901083B19010894
:101AA0003B1901083B1901083B1901083B190108C2
:101AB0003B1901083B1901083B1901083B190108B2
:101AC0003B1901083B1901083B1901083B190108A2
:101AD0005B1B01083B1901083B1901083B19010870
:101AE0003B1901083B1901083B1901083B19010882
:101AF0003B1901083B190108551B0108A12921DCEC
:101B000096297FF71AAFA1F197030A2B3FF615AF7D
:101B10000FF2040C5CF823F05B1B01085B1B01084F
:101B20003B1901085B1B01083B1901083B1901081F
:101B30003B1901083B190108551B0108551B0108F9
:101B40005B1B0108B42908D0DB2903D0B2297FF43C
:101B5000F4AE704700235AF051BB704770B563294B
:101B60008AB000F3D180012904DC0AB0BDE87040DE
:101B70005AF014B98B1E612BF7D801A454F823F046
:101B80007F1D0108931D0108B31D0108BB1D01083D
:101B90006B1B0108EF1D01086B1B01086B1B010883
:101BA000A31E01086B1B01086B1B0108A11D010886
:101BB000C91E01086B1B01089F1E0108031F0108B5
:101BC000111F01086B1B01086B1B0108211F010875
:101BD0002F1F01083D1F01086B1B01085F1F010833
:101BE000711F01086B1B01086B1B01086B1B0108AF
:101BF0006B1B01086B1B0108831F01089D1F010857
:101C00006B1B01086B1B01086B1B0108A11F01085E
:101C10006B1B01086B1B01086B1B01086B1B010888
:101C2000A51F01086B1B01086B1B01086B1B01083A
:101C30006B1B01086B1B01086B1B01086B1B010868
:101C40006B1B01086B1B0108B51F01086B1B01080A
:101C50006B1B0108151F0108191F01081D1F010832
:101C60006B1B01086B1B01086B1B01086B1B010838
:101C70006B1B01086B1B01086B1B01086B1B010828
:101C80006B1B01086B1B0108A91F0108AD1F010890
:101C9000B11F01086B1B0108B91F0108BD1F010816
:101CA0006B1B0108FF1F0108C11F01086B1B010806
:101CB0006B1B01086B1B01086B1B01086B1B0108E8
:101CC0006B1B01086B1B01085B2001086B1B0108E3
:101CD0006B1B01086B1B01086B1B01086B1B0108C8
:101CE0006B1B01086B1B01086B1B01086B1B0108B8
:101CF0006B1B01086B1B01086B1B01086B1B0108A8
:101D00006B1B0108712001089F291DDC96297FF7B4
:101D10002CAFA1F19703082B3FF627AF01A454F88D
:101D200023F000BF75200108792001086B1B010812
:101D30008D2001086B1B01086B1B01086B1B010840
:101D40006B1B010869200108B42900F0DC80DB2945
:101D500017D0B2297FF409AF002A00F07781022A58
:101D60000FD1AF4BD3F8B40203689B6F984740B9CB
:101D700058F0A0F9AB4A042151F010FB01E0022A0F
:101D800001D0012430E035220E21A74803F0B4FD34
:101D9000F7E7111E18BF0121A348FCF725FAF0E769
:101DA000012A04D0022A14BF00210221F4E71146BF
:101DB000F2E70621FFF7C8FCE3E7022AE1D1984DDC
:101DC000D5F8B4020368DB6A984704460028D8D0E7
:101DD000A5F58053D3F8F03EB3F90830002BD0D1ED
:101DE000A5F54050FFF7EAFC20460AB070BD022A74
:101DF000C7D18B4ED6F8B41206F5FA529142C0D034
:101E0000D6F8D82292F8CB20002ABAD006F5805412
:101E1000A6F58056B4F9B02F2AB9D6F8F03EB3F93A
:101E20000830002BADD01C22002103A805ADABF07B
:101E3000EFFF284615F0ACFBB4F9B03F93B9162379
:101E4000ADF80E30D4F8303D7848642BB8BF642329
:101E500003A906932BF02AF920B14FF0EDF92721C1
:101E60004FF026F904F62C5494E80F0085E80F0093
:101E7000D6F8F03E6D48B3F90830002BCCBF1023E4
:101E8000152303A9ADF80E302BF010F900283FF40C
:101E900078AF4FF0D1F927214FF00AF971E703210C
:101EA00088E7022A624D03D0002385F8043F68E7E3
:101EB0001921A5F5706047F01BF804460028F3D0FF
:101EC000012385F8043F8FE7012A0BD0022A11D0A5
:101ED000002A7FF456AF564B83F8D8254FF0ACF963
:101EE0002B21D9E7524B019283F8D8254FF0A4F962
:101EF0002C21D1E74E4B83F8D8254FF09DF92D21A9
:101F0000CAE70F2156E74B48114684F0CFF938E76E
:101F100009214FE704214DE705214BE7172149E748
:101F2000901E4142414144485DF016FE29E7022AD5
:101F30007FF427AF3C4801F007FB22E7012A06D0D7
:101F4000022A07D0002A7FF41CAF1146EBE71146A6
:101F50000192E8E7384801215DF0FEFDEAE7374BE2
:101F6000911ED3F8583D4A424A4183F8202008E7A1
:101F7000931E59425941314BD3F8580D78F0ECF982
:101F8000FFE6274B013A93F8AA12012A8CBF0022E0
:101F9000012262F3041183F8AA12F2E6112109E783
:101FA000122107E7152105E7002103E7102101E7CA
:101FB0000221FFE60121FDE60721FBE60B21F9E600
:101FC000022A1E4B0ED1012483F8A04E4FF034F9A3
:101FD0004A214FF06DF858F06DF8194A062151F07A
:101FE000DDF901E7002283F8A02E4FF025F94B21FF
:101FF0004FF05EF858F05EF8124A0621BCE6012A5E
:1020000009D0022A0AD0002A7FF4BBAE01210E4873
:102010000CF03AFEB5E601920021F8E71146F6E72A
:10202000B85B0020B7780C08B82B0020347B002068
:10203000B84B00200C7D0020007A0020B86B0020F7
:1020400094780C08A5780C084C5B0020184BD3F84A
:10205000B4020368DB6F984793E61146FFF792FBE3
:10206000144803F0F5FF8CE61146FFF799FB88E66C
:102070001B219FE61C219DE6022A7FF482AE0E48BA
:10208000FCF7A6FE58F016F80C4AB6E7114659F0D0
:10209000A5FD0B4874F0FCFF044600283FF471AE28
:1020A000034A92F8AB3243F0020382F8AB329BE66C
:1020B000B85B00207C7A0020B82B0020D0780C0878
:1020C000C45B002010B5044604487DF05DFB04F1BC
:1020D0000801BDE8104027F067BE00BFF47800207B
:1020E00038B504462DED028B11487DF053FB0546B3
:1020F00029F096FD0F48B0EE408A0CF071FE90B1C9
:10210000DFED0D7AB4EEE78AF1EE10FA0BDDD5EDD6
:10211000000A95ED010AA9F081FCDFED087A20EEB6
:10212000270A84ED080ABDEC028B94ED080A38BD3D
:10213000F4780020B82B002000401C46E02E6542B9
:10214000074B93F99505022805D0032806D00038DF
:1021500018BF0120704781F00100704704207047CC
:10216000B84B002003688B4216D00429C0E9001345
:1021700002D007290ED07047084B9FED097A03F66D
:102180005803D3ED007AF8EEE77A67EE877AC0ED70
:10219000087A704700238362704700BFB83B002075
:1021A0000AD7233C08B50246FFF7CAFFBDE808403E
:1021B00001461046FFF7D6BF70B52DED048B0446DF
:1021C000F0EE408AB0EE608A0D46164685F080FC3F
:1021D0009FED329ADFED329AE06176B3236843B91E
:1021E000304B03F65803D3ED007AF8EEE77AC4EDEE
:1021F000097A68EE898A002DB7EE000AFFEE007AB0
:10220000B8BFB0EE670A68EE808AC4ED058A264B37
:10221000B4EEE98AF1EE10FAD3F8580D30DA77F01F
:1022200079F820EE090A84ED060ABDEC048B2046FD
:102230000321BDE87040FFF795BF94ED090A98EEC1
:10224000890A26F025FD002D84ED050A0BDAB4EE8F
:10225000E90AF1EE10FADADBDFED147A30EE670A04
:1022600084ED050AD3E7D2D0DFED117AB4EEE70AA8
:10227000F1EE10FACBD8DFED0D7A30EE270AEFE75A
:1022800077F048F8B4EE480AF1EE10FA48BFB0EE25
:10229000408A28EE098A84ED068AC6E70000C84213
:1022A00000000034B83B0020B86B002000A00C47B1
:1022B000000000B410B52DED028B0446B0EE608A2C
:1022C000F0EE408A85F004FCDFED090AE06168EE7B
:1022D000A08A68EE200AC4ED098ABDEC028BC4ED29
:1022E0000A0A20460621BDE81040FFF73BBF00BFA9
:1022F0000000C84208B54A680346084642B98A68E1
:1023000032B9C96821B9BDE808400748FFF74ABF9C
:1023100003F1080115F0CCFA28B1BDE808400248E5
:102320000221FFF71FBF08BD0C83002008B507215D
:10233000FFF718FF80ED0A0A08BD000008B5036822
:10234000032B23D1D0ED057A9FED127AF0EEE77AD8
:10235000F4EEC77AF1EE10FA1AD50F4B90ED090A98
:1023600003F65803D3ED007AF8EEE77A37EEC00AA9
:1023700026F08EFCDFED097AB0EEC00AB4EEE70A73
:10238000F1EE10FA94BF0120002008BD0120FCE707
:102390000020FAE700000034B83B0020000048436A
:1023A00030B50368023B85B00446082B6DD8DFE8E2
:1023B00003F0050D30374B613F616100FFF782FE8E
:1023C00084ED090A94ED090A05B030BD85F080FB63
:1023D000E369DFED310AE061C31A07EE903AF8EEE7
:1023E000677A94ED050A67EEA07AD4ED060AF1202B
:1023F00020EEA71A67EEE00A26F0A0FCD4ED057ADD
:1024000077EEC07AC4ED057AD4ED097A37EE800A0A
:10241000D6E7FFF765FEDFED217A20EE270ACFE74A
:102420001F4BD3EDC07AF8EEE77AC0ED097AC9E721
:102430001C4DD5F86C0D7BF041FB0028C2D0D5F8BF
:102440006C3D1B6B6362BDE785F042FBE3699FED6A
:10245000127AD4ED0A6AE061C31A07EE903AF8EEF8
:10246000677A67EE877A94ED097AA6EEA77A84ED0B
:10247000097AA7E70B4B9FED0C0AD3F8580D6C3087
:1024800029F06AFE84ED091A9CE7064BD3F8603DFB
:10249000D3F84433D6E700BF6F12833A0000C84236
:1024A000B85B0020B86B00209F0CB3450368092B74
:1024B00008D8DFE803F0050A05050505070705103C
:1024C0000023836290ED0A0A7047044BD3F8603D05
:1024D000D3F84833F5E7C36AF3E700BFB86B0020D1
:1024E000F8B50023214FCB6297F8CD32204E13F080
:1024F000010F04460D462DD1D7F8B40203685B6F77
:10250000984738B3D7F8B40203F0ACFBDFED197A83
:1025100085ED0B0AB0EEC00AB4EEE70AF1EE10FA50
:1025200003D409213046FFF71DFE1148FFF738FF9D
:102530000F4884ED000AFFF7B9FF336884ED010A04
:102540000A2B0FD8DFE803F00C1010101010100C3D
:10255000100C0C003368092BE7D105480021E2E795
:102560000223A3602046F8BD0123FAE7B85B0020F0
:102570000C83002000000034034B01221A6000226B
:102580009A60DA601A6170470C83002013B501A9C4
:1025900004460CF0C1FA04F5804320B9012283F807
:1025A0001D2E02B010BDDDED017ADFED096A03F5E5
:1025B0006162B8EEE77AD2ED007A67EEA67AB4EE01
:1025C000E77AF1EE10FA54BF01220022E7E700BFDC
:1025D0000000C8422DE9F04F2DED068B00F5005BA1
:1025E00000F5B2599BF9E6358DB0054600F58044FB
:1025F00009F1180933B100F54058D8F8D83293F8EA
:10260000CB707FB90021A4F8941E48460FF046FE17
:1026100094F8951E48460DB0BDEC068BBDE8F04F12
:102620000FF046BE85F054FA0190D4F8600D9FED8E
:10263000958A90EDDBAA79F061FC09AE002800F0E4
:10264000CC80D4F8603D03F55C7393E8070086E81E
:10265000070030468DED0B8A2AF07CF9B0EE409AE7
:1026600028460CF0BDFB05F59A4A0AF13C0A002801
:1026700000F0B68050467DF08DF807C886E8070068
:1026800030468DED0B8A2AF065F9F0EE409AD8F8C5
:10269000B40203681B689847122840F0AA80002300
:1026A00084F8943ED8F8B40203685B69984728B16F
:1026B000DBF8F03EB3F90830002B0DDC98F9A832B6
:1026C000002B09DA019BC4F8983E50467DF05EF875
:1026D00004F69C6383ED000A94F8943E5BB1019B81
:1026E000D4F8980E181A41F28833984240F28F803D
:1026F000002384F8943ED4F8580D9FED630A6C30A3
:1027000029F02AFD8DED090ACDED0A0A8DED0B1A8F
:1027100096E8070006AB03AE9FED5C0A83E807006E
:1027200086E80700304629F017FD2846B0EE408ABB
:10273000F0EE608A8DED060ACDED070A8DED081AE0
:102740000CF04EFB002874D0DFED517AF4EEE79ADE
:10275000F1EE10FA94BF01250025D4F8600D79F050
:10276000CDFB30B1DFED4A7AB4EEE79AF1EE10FA24
:1027700009D9002D64D1D8F8B40203681B689847C2
:10278000022864D00027D4F8600D79F0D9FC054602
:10279000002873D0B5EEC0AAF1EE10FA6DD5DFEDCA
:1027A0003D7AB4EEE7AAF1EE10FAACBF012600269E
:1027B00050467CF0F7FF5EB9DFED377AB0EEC00A25
:1027C000B4EEE70AF1EE10FA5AD8002D08BF002740
:1027D00094F8941E84F8957E17E7B0EE489A3FE788
:1027E00028460CF0CFFA00287FF444AFDFED259A9D
:1027F0004DE7D8F8D83293F8CB30002B3FF452AFE6
:1028000098F9A832002BBFF64DAF012348E7504698
:102810007CF0BCFF04F69C63D3ED007A30EE670ACF
:10282000DFED1E7AB4EEE70AF1EE10FA3FF760AF83
:1028300061E728460CF0A6FA0546002884D18CE70B
:10284000D4F8600D79F05AFB002894D19BE7B0EEE4
:10285000680AA8F0C1FEF0EE408AB0EE480AA8F07F
:10286000BBFEDFED0F7A20EE280AB4EEE70AF1EEA8
:1028700010FACCBF0127002785E700252E4697E7F1
:102880003746A5E7000000009F0CB345D302373957
:102890000000FA420000C8C2000070420000484236
:1028A00055CF7D3F38B504460CF09AFA04F5B25581
:1028B000183548B920460CF065FA014620B928467B
:1028C000BDE838400EF06CBF04F54054D4F8B402B3
:1028D00003689B6C984720B9D4F8B4020368DB6C9A
:1028E00098470146EBE7000030B5044689B06846DA
:1028F00004F5B25514F04CFE183504A814F048FE47
:10290000694628460FF006F898B104A928460FF04A
:1029100051F870B1059B019323680022DB6C694676
:102920002046984728B104F5365001210C3080F03C
:1029300091FE09B030BD000000F5805292F8D42815
:10294000D2070BD400F54052D2F8D82292F8CB101F
:1029500009B1FFF7C9BF03689B6C184770470000B7
:1029600030B587B0044602A8019114F011FE04F5B9
:10297000B25002A918300EF0CDFF019A18B9002507
:10298000284607B030BD236802A9DB6C2046984773
:1029900005460028F3D004F5365001210C3080F0B4
:1029A00059FEEDE7F0B5044685B004F5B256684629
:1029B00018360F46154614F0EBFD694630460EF00A
:1029C000F9FF10B9002005B0F0BD394630460EF0D1
:1029D00059FE0028F6D0002DF5D004F58054284685
:1029E00094F8D43843F0020384F8D438EBE70000BD
:1029F0002DE9F04F2DED0A8BBDB0044624220D4683
:102A000018A80021ABF004FA2422002121A8ABF081
:102A1000FFF9242200212AA8ABF0FAF904F5405668
:102A20002422002133A8ABF0F3F90023CDE90D33C4
:102A30000F9396F8A93213F0080839D104F500591C
:102A400043F0080399F8E42E079286F8A93215F0AE
:102A5000D3FE90F9213003B390F84033EBB104F288
:102A60005457384615F0D8FDC34694F876355FFACA
:102A70008BF18B421FD9384615F0ACFD0BF1010BE1
:102A800082460028F1D1C94A0221284653F0B0FEFF
:102A900096F8A9326AF3C30308E0C54A0221284622
:102AA00053F0A6FE96F8A9326FF3C30386F8A93255
:102AB0004FF001083EE304F540530C330121184662
:102AC0000BEE903AFBF76CF8824608B9B94ADBE79F
:102AD00020460BF0A7FED9F8F03EB3F908A0BAF1F2
:102AE000000F01D0B44AD9E796F9A832002B01DBD8
:102AF000B24AC9E7204601F087FE04F54C5304337F
:102B0000184652460CA90CEE103A12F0E9F80028CB
:102B100014BF022301230393F123CDE9133A8F213C
:102B20000A23CDE9003113AA287CADF854A0032371
:102B30004D2151F02BFCA24B9FEDA28A01225A722B
:102B40000621A14A284653F053FE039B022B0CBFDB
:102B50009E4A9F4A062128464FF0000A53F048FE3D
:102B600089F8A2A55146384615F0A0FC94F87635B0
:102B70005FFA8AF18B420CD913AA38468DED138A7D
:102B80008DED148A8DED158A0AF1010A15F010FBFE
:102B9000ECE7384615F040FD4FF0000A4FF07C0B93
:102BA00094F876255FFA8AF94A4519D94946384694
:102BB00015F0F0F9C0B20BFB00403CAA0C2300F268
:102BC000E45003FB092C07C8ACF1900C8CE807001B
:102BD0003CAA02EB890909ED2F8A0AF1010ADFE715
:102BE00041F288310AA821F0BBFFD6F8D8029FED48
:102BF000759A03689FED77AA9B6ADFED77AA9847DD
:102C0000D6F8D80201217DF06DFD744B1B6802934C
:102C1000D86A036801211B68984784F059FF059022
:102C200084F056FFF0EE499A0690002604F500590C
:102C3000079A99F8E43E934240F0D88094F89618A9
:102C4000384615F0C7FC002800F0D08004F5405B42
:102C5000DBF8D83293F8CB300493002B00F0C68019
:102C600041F288310BA821F07BFF84F031FF059BF6
:102C7000C01A132840F2D98084F02AFF059020461C
:102C80000BF0D0FD5AF0F4F982465AF08BF9D9F8DE
:102C9000F03EDBF8D802B3F9083000EE103AB8EE97
:102CA000C00A20EE0A0A7FF0F7F950465AF082F97E
:102CB000384615F0B1FC1CEE100A12F0FBF9D9F8F9
:102CC000F03EDFED400AB3F9083000EE103AB8EEFE
:102CD000C00AA22020EE0A0AB7EE001A26F02EF84B
:102CE000B4EEE90AF1EE10FA1CEE100A4FF0000201
:102CF0000CA958BFF0EE409AF0EE408A11F0F0FFB8
:102D000008B900230C939DED0C8ADFED357AB4EE03
:102D1000498AF1EE10FAF4EEE78A48BFB0EE498A2C
:102D2000F1EE10FA80F28F809FED2E9ADFED2E8A61
:102D30004FF0000A94F876355FFA8AFB5B4540F263
:102D400096814FF00C0918AB09FB0BF903EB090056
:102D5000B0EE490A29F000FA59463846CDED110A7D
:102D60008DED121A8DED100A15F014F97C23C0B206
:102D700003FB0040B0EE680A00F2E45029F0ECF9E1
:102D80003CAB13A910A899448DED130ACDED140A9C
:102D90008DED151A29F0B4F90AF1010A09ED240A9A
:102DA00049ED230A09ED221AC4E700BFCD7A0C08C9
:102DB000BC7A0C08CB8E0C08DB7A0C08ED7A0C0878
:102DC000BD84002000000000F87A0C080D7B0C0880
:102DD0007F240C086F12833A0000C8420083002051
:102DE00000000034A4707D3F0AD7233C04F540590D
:102DF000D9F8D80203689B6A9847D9F8D80200210D
:102E00007DF070FC029BD86A036800211B6898471C
:102E1000002E40F05F812846C94A052153F0E8FCA6
:102E20003146384615F042FB70E1029B986A036810
:102E300005215B6898470BA821F09EFEB0EE498AF9
:102E4000B0EE489AF2E64FF000094FF00C0B04F593
:102E5000B26A94F876255FFA89F39A4222D9194624
:102E60003846089315F096F8089B0BFB03F13CAB32
:102E70005A18A2F16C034FF07C0CC0B2CDE90832B5
:102E80000CFB00A018AB1944543029F04FF9089BF3
:102E9000099A09F1010902ED1B0AC3ED010A83ED4C
:102EA000021AD6E7039B012B4FF0000A46D19FED93
:102EB000A5BA9FEDA59A4FF00C0B94F876355FFA02
:102EC0008AF6B34240F286800BFB06F63CAB03EB7E
:102ED0000609A9F14803089321ABB0EE680A9819D6
:102EE00029F04AF9089B09ED120AC3ED010A83EDA6
:102EF000021A33ABB0EE4B0A981929F02DF92AAB20
:102F000098198DED100AB0EE490ACDED110A8DED3C
:102F1000121A29F021F913A910A88DED130ACDED8D
:102F2000140A8DED151A29F001F90AF1010A09EDCB
:102F3000090A49ED080A09ED071ABEE79FED819AD3
:102F40009FED81BAF0EE088A94F876355FFA8AF937
:102F50004B4564D99DED0C0AB4EEE80AF1EE10FA87
:102F600035DB0C2303FB09F93CAB03EB090621AB72
:102F700003EB090029F000F933AB46ED110A06ED29
:102F8000101A06ED120A03EB0900B0EE490A29F007
:102F9000E3F82AAB03EB09008DED100AB0EE4B0A03
:102FA000CDED110A8DED121A29F0D6F813A910A84B
:102FB0008DED130ACDED140A8DED151A29F0B6F832
:102FC00006ED090A46ED080A06ED071A049E0AF105
:102FD000010AB9E74FF000094FF00C0A94F8763572
:102FE0005FFA89F6B34241D933AB0AFB063029F0C8
:102FF000B1FC1BEE900AF0EE408A74F045F807EE43
:10300000900AB8EE677A3CABC8EE877A03EB860687
:1030100009F1010967EEAA7A46ED2F7ADEE74FF053
:10302000000A4FF00C0B94F876355FFA8AF94B459D
:103030001DD933AB0BFB093029F08CFCC8EE297A83
:103040000AF1010A1BEE900A67EE808A74F01CF800
:1030500007EE900AB8EE677A3CABC8EE877A03EBCE
:10306000890967EEAA7A49ED2F7ADCE7049E84F09D
:103070002FFD069BC01AB0F5FA7F27D984F028FDF2
:1030800004F50053DDED0D7AD3F8F03E0C9A1B8960
:103090001392FCEEE77A339A1492ADF85C30349ACE
:1030A000159217EE903A359A1692ADF85E30F022EE
:1030B0001423CDE90032B121069013AA287C51F0E7
:1030C00065F96CF02FFE297C6CF026FD0BA821F031
:1030D00053FDB5E60399384615F0E8F900264FF0A0
:1030E0000C0A94F87635F1B28B4207D933AB0AFB60
:1030F0000132384615F05CF80136F2E7384615F033
:1031000069F8124A0621284653F072FB104B00253D
:1031100020465D7201F06AFB04F51650223044F03F
:10312000CBFC99F8A93265F3C30389F8A9320AA840
:1031300021F022FD40463DB0BDEC0A8BBDE8F08F8A
:1031400029110E08A4707D3F0AD7233C157B0C087B
:10315000BD8400207FB54C4BD3F8B03EDB0704465E
:1031600000F18F8000F54055D5F8D83293F8C12092
:10317000002A40F0868093F8CB30002B7ED095F962
:10318000A832002B7ADB00F5804696F8A03E002B93
:1031900077D1D6F8580D9FED3D0A6C3028F0DCFF52
:1031A000CDED020A60EEA00ADFED397A8DED010A5D
:1031B000E0EE000A8DED031AF4EEE70AF1EE10FAE4
:1031C0005CDCD6F8583D9FED337AD3ED377AF4EED8
:1031D000C77AF1EE10FA04D5D5F8D8321B7A002B55
:1031E0004CD0B5EE007AF4EEC77AF1EE10FA45D481
:1031F00004F59A403C307CF0D5FADFED277AB4EE46
:10320000E70AF1EE10FA39D8D6F8583D9FED237A47
:10321000D3ED367A67EE877AB3EE0E7AF4EEC77A9C
:10322000F1EE10FA2ADA1E4AB4F9A4101388013319
:103230009BB2138019B9B4F8A210A4F8A410B4F882
:10324000A41099421DD8002616804DF0F5FF0122EA
:1032500019214DF04DFFD5F8D80203685B699847F6
:10326000431C04F542500F4A31460C3050F096F89A
:10327000D5F8D832012283F8C12002E0084B0022A1
:103280001A8004B070BD00BFB84B00209F0CB3453E
:103290004054094A6666663F000000B4E02E65426D
:1032A000468300202C7B0C0870B52DED028B4A4B19
:1032B000D3F8B03E9B0784B004461FD400F5804588
:1032C000DFED468AD5F8580D03681B699847D0EDA5
:1032D000017AF4EEE87AF1EE10FA0FDB04F54053D0
:1032E00004F59D46D3F8D82292F8C110243649B18E
:1032F000002303A9304603934FF0D8FB04B0BDEC84
:10330000028B70BD92F8CB20002AF1D093F9A8323D
:10331000002BEDDB95F8A03E002BE9D1D5F8580D38
:1033200003681B699847D0F8A430D5F8580D03936B
:1033300003681B69984704F58C7200F1A4013046BC
:103340004FF056FCDDED037AB0EEC08AF0EEE77A7E
:10335000F4EEC87AF1EE10FA03D503A930464FF027
:10336000A5FBD5F8580D03681B699847D0ED040AF2
:10337000F4EEE80AF1EE10FAC0DBF6EE087A60EE41
:10338000A77AF4EEC87AF1EE10FA1DD584F0A0FB0E
:10339000D5F8B03E42F21072C31A9342AED9DFEDB7
:1033A000107AC5F8B00E68EE277A04F5425417EE8D
:1033B000900AF9F7A9F80C34CDE90001094A002177
:1033C00020464FF0EBFF99E79DED030A25F0B2FB95
:1033D0000028DBD192E700BFB84B0020000000348A
:1033E0000000C842487B0C0810B5044600F59C401C
:1033F00048305CF0C3FB04F59C400121BDE810405F
:10340000683065F08DB80000F8B500F580450446D9
:1034100095F9483E4BB300F5405695F85C2E96F86A
:10342000A832DB43C3F3C01363F3C30200F59C4728
:1034300000F59A4085F85C2E3C307CF0B3F9DFED66
:103440003E7A483720EE670A38465CF017FC95F85C
:10345000A03E53B938465CF0BDFBD6F8D83293F89D
:10346000CB301BB9354B00221A80F8BD95F85C3E75
:10347000DB07FAD4D6F8B40203689B6B98470028A0
:10348000F0D096F9A832002BECDB2C4E33884BB9E8
:10349000B5F94E3E33B1642213FB02F3D5F8302D5B
:1034A0009A42E2DB38465CF005FCD5F8583D9FEDCA
:1034B000247AD3ED367A67EE877AB3EE0E7AF4EE9D
:1034C000C77AF1EE10FA05D83388002BCDD0013B36
:1034D0003380CAE7B4F9A4301BB9B4F8A230A4F819
:1034E000A4303388B4F8A420B4F9A4001549934259
:1034F0003CBF013333803388D5F8082D012B01D12F
:103500000A60B2E709689142ACDD18B9B4F8A220AC
:10351000A4F8A420B4F8A4209A42A6D800233380AB
:103520004DF08AFE02220C214DF0E2FD2046BDE85E
:10353000F840FFF759BF00BF0AD7233C448300205F
:10354000E02E65424083002008B500F5804292F9E4
:10355000483E6BB300F5405393F9A832002B0EDAC6
:1035600000F54250134A06210C304FF017FF4DF082
:1035700063FE0322BDE808400F214DF0B9BDB2F94A
:103580004E3E8BB1D2F8302D642113FB01F39A42E9
:103590000ADA00F54250084A01210C304FF0FEFED5
:1035A0004DF04AFE0222E5E7BDE80840FFF71CBFE8
:1035B00008BD00BF607B0C08727B0C08F0B52DEDD8
:1035C000028B00F540555A4ED5F8D83293F8CB30DF
:1035D0008DB0044643B195F9A832002B04DB00F509
:1035E000005393F9BE352BB9002333800DB0BDECE9
:1035F000028BF0BD00F5804797F8A03E002BF3D179
:1036000001F06AFB002879D1D5F8B40203689B6BFE
:1036100098470028E8D004F59A400C304FF068FA3B
:1036200029F098F9F0EE087AB4EEE70AF1EE10FA14
:10363000F0EE408AD8DA04F5B253D3ED997A93EDDF
:10364000980A20EE270AA8F081F9DFED3A7A20EEF9
:10365000270AB2EE0E7AB4EEC70AF1EE10FAC3D919
:10366000D7F8583D93ED368A28EE278AF3EE0E7A86
:10367000B4EEE78AF1EE10FAB6D904F5B2500023A1
:1036800009A9183009930A930B930EF09FF90028AB
:103690003DD13388B4F9A42001339BB23380002A92
:1036A00040D0B4F8A420B3EB420F9FDB4DF0C4FD33
:1036B00001220C214DF01CFD1F4B002218EE900A38
:1036C000CDE90623F8F720FF1C4BCDE904010022C9
:1036D00018EE100ACDE90223F8F716FF04F542545C
:1036E0000C34CDE90001164A204600214FF056FE69
:1036F00001220C211348FAF76BFC77E7D5F8B402E6
:103700000368DB6C984700287FF47EAF6CE709A85C
:1037100029F020F9F2EE047AB4EEE70AF1EE10FA9D
:10372000B7DB61E7B4F8A220A4F8A420B9E700BF92
:103730003C830020E02E65420000084000003E402F
:10374000887B0C08C45B0020F0B52DED028B8BB09C
:10375000002307930893099305AB0446019300F5F2
:10376000B25007AB009302AA04AB03A918300EF0C5
:1037700045F804F54057054687F8800028B900252C
:1037800028460BB0BDEC028BF0BD84F095F9D7F85C
:1037900084309FED307AC31A07EE903AF8EE677ADC
:1037A000064667EE877A04F5415006AA02A91C3046
:1037B000CDED067A4FF01CFA04F5415006AA03A994
:1037C00028308DED020A4FF013FA04F5415006AA95
:1037D00004A934308DED030A04F517544FF008FAAC
:1037E000C7F8846094ED008AB5EEC08AF1EE10FA55
:1037F000C5D9DDED080A9DED070AA7F073FFDDEDE1
:10380000090AA7F06FFFDDED037A38EE087AB4EE0F
:10381000C08AF1EE10FAB4EEE77A94BF01230023D8
:10382000F1EE10FA0AD80233DDED027AB4EEE78A3F
:10383000F1EE10FA0AD8002BA1D0A1E7B4EEE78A86
:10384000F1EE10FA9CBF0133DBB2EDE7012B97D804
:1038500095E700BFBD37863570B500F54055044685
:1038600095F8CD3243F0040385F8CD324DF0E4FCF9
:10387000012211214DF03CFCD5F8D83293F8CB3021
:10388000002B43D0D5F8B40203681B689847092879
:103890000AD1204607F0E0FA30B104F5A8403030F4
:1038A000BDE8704007F0C0BA194BD3F8B402036802
:1038B0001B69984704F5005340B993F9BD35032BB4
:1038C00024D10621204607F0B3FA0DE093F9BD1587
:1038D0000229F6D195F8CD32DB07F2D40622204634
:1038E00002F00AF80028ECD00A4BD5F8B402012205
:1038F0005A7303681B6C9847034604F54250064A06
:10390000BDE8704002210C304FF048BD70BD00BFD3
:10391000B85B0020BD840020BC7B0C0808B500F516
:10392000405292F8CD32590717D56FF3820382F8CF
:10393000CD320A4B5A7B42B1002200F542505A73F5
:103940000221074A0C304FF029FD4DF075FCBDE80F
:103950000840002211214DF0CBBB08BDBD840020E2
:10396000E07B0C08F0B5054685B005F5B257684612
:10397000183713F00DFE694638460EF01BF880B17B
:1039800005F51753D3ED007A374CF5EEC07AF1EE1A
:1039900010FA08D8354A002328462380D373FFF74E
:1039A000BDFF05B0F0BD2846FFF7CEFE064628460F
:1039B0000BF0E8F910B928460BF0BEF9A378002EF9
:1039C00018BF00200343DBB2A370002BE9D063785B
:1039D000A8BB83BB23780133DBB2082B237003D150
:1039E0004EB338460DF076FF2378092B02D13846C6
:1039F0000DF068FF2378092B1DD94FF485732380C0
:103A00004DF01AFC022210214DF072FB84F060F898
:103A10006368C01A47F23053984209D905F54250FD
:103A2000134A02210C304FF0B9FC84F051F8606069
:103A30002846FFF711FF0D4B6278DA73B1E726785D
:103A4000002EF8D0013EF6B22670002BF3D0002EE7
:103A5000F1D166704DF0F0FB324610214DF048FB7D
:103A60002846FFF75BFFE6E748830020BD8400207F
:103A7000F87B0C0800F5405393F8CD325B0701D575
:103A8000FFF7EABE7047000073B5044600F5B25078
:103A900001A9183004F540550DF0FAFCAB6C8342D7
:103AA00006460BD004F58043D3F8580D76F0F6FFA8
:103AB000AE644DF0C1FB3E214DF0FAFA04F580569C
:103AC00095F94C1096F9682996F8683991421BD0FF
:103AD000FF2B19D004F58043D3F8580D76F0DEFFA4
:103AE00096F8683985F84C304DF0A6FB95F84C20D7
:103AF00018214DF0FDFA04F5425095F94C30034A77
:103B000004210C304FF04AFC02B070BD087C0C0858
:103B10002DE9F0438FB0054683F0DAFF00230593CB
:103B200006930793089309930A930B930C930D93B1
:103B300005F5B25804AB019308F1180803AB0093E4
:103B400006460BAB08AA05A940460DF037FEDFED8F
:103B5000487A9DED077AB4EEE77AF1EE10FA07465F
:103B600032DB9DED0A7AB4EEE77AF1EE10FAACBFE3
:103B70000124002405F54059404699F88030002B77
:103B800008BF00270DF02CFE8046FFB9444605F51E
:103B9000005393F94C3E012B29D164B1D9F8D832A6
:103BA00093F8CB403CB1D9F8B40203685B699847FD
:103BB00080F00100C4B299F85030CBBBCCB9C9F841
:103BC00054600FB0BDE8F0830024D3E7002CDDD0B3
:103BD00005F5415028304EF067FF90ED007AF7EE82
:103BE000007AB4EEE77AF1EE10FAD0DCCEE70024EA
:103BF000E1E7D9F85400301AB0F57A7FE1D9C9F875
:103C00005830012405F5804389F85040D3F8603DD1
:103C100083F80C444DF010FB22461D214DF068FA4C
:103C2000144A05F5425002210C304FF0B7FBC8E7AB
:103C300014B1C9F85860C4E7D9F8580043F698237E
:103C4000361A9E42BDD905F58043C9F8544089F81B
:103C50005040D3F8603D83F80C44C9F858404DF00B
:103C6000EBFA22461D214DF043FA034AD9E700BF83
:103C700000000034207C0C083A7C0C080B4B10B57B
:103C8000012204465A7283F023FF04F58042D2F8E1
:103C90008C3EC31A142B08D9C2F88C0E04F5B05010
:103CA0000430BDE8104040F07FBE10BDBD84002050
:103CB0002DE9F743044604F5405600F5165000235D
:103CC00038300DF107018DF8073044F06BFCD6F861
:103CD000D80290F9C030026883B3083BDBB2012BF5
:103CE00095692BD93221A84704F1100011F05CFB33
:103CF000204B04F542581F684FF0000908F10C08EA
:103D0000F86A0368DB69984701281ED183F0E0FE5A
:103D100041F28733A0EB09029A42054605D9164ABB
:103D2000062140464FF03AFBA9462046FFF7A6FF82
:103D3000B86A036803215B689847E1E704F500531C
:103D40009269B3F8CC159047CEE70121D6F8D80296
:103D50007CF0C8FCD6F8D8020368DB6A984758F0B4
:103D600015FEF86A03681B68012103B0BDE8F04343
:103D7000184700BF00830020587C0C0870B504462B
:103D800000F542502DED028B184A194E9FED198A0D
:103D900006210C304FF002FB2046FFF789FF20463A
:103DA000FFF76CFF20460AF03DFD3368986A036810
:103DB00003215B68984759F05BF9054659F0F2F822
:103DC00004F50053D3F8F03EB3F9083000EE103A92
:103DD00004F54053B8EEC00AD3F8D80220EE080A22
:103DE0007EF05AF9284659F0E5F8D8E77C7C0C08B3
:103DF000008300206F12833A2DE9F047044600F556
:103E000042502DED028B2A4ADFF8AC9006210C308F
:103E10004FF0C4FA2046FFF74BFF59F029F904F59B
:103E20004056054659F0BEF8B7EE000AD6F8D8025B
:103E30007EF032F9284659F0BDF883F049FE41F290
:103E4000873A074683F044FEC01B5045D9F80080EE
:103E500017D99FED188A284659F0A4F8B0EE480A01
:103E6000D6F8D8027EF018F9284659F0A3F8204673
:103E7000FFF704FFD8F82800036803215B68984720
:103E8000E9E7284659F08EF8B7EE000AD6F8D802CE
:103E90007EF002F9284659F08DF82046FFF7EEFE35
:103EA000D8F82800036803215B689847CAE700BF79
:103EB000AC7C0C080000000000830020F7B500F582
:103EC00040530446D3F8D83293F9C030032B2BD09B
:103ED000364E652500F58047013D15F0FF050CD0F5
:103EE000D7F8883E4BB93368986A036814215B6839
:103EF000984720460AF096FCEEE704F54050012171
:103F00000C30F9F74DFE04F5005378B993F9B83544
:103F100053B1092B08D08DF8070004F516500DF1A8
:103F20000701383044F03EFB03B0F0BD93F9B825EB
:103F3000032A34D8DFE802F002252D30D3F8F03E12
:103F4000B3F9082040F2B5339A422ADD04F5165041
:103F500001250DF1070138308DF8075044F022FBA0
:103F600004F54250124A02210C304FF017FA114B5F
:103F70005D720E4B1C68A06A036805215B68984758
:103F8000F9E7D3F8F03EB3F9082040F2B5339A428E
:103F900007DD2046FFF7F2FE2046FFF72DFF092A36
:103FA000C2D000238DF80730B7E700BF00830020A0
:103FB000D07C0C08BD84002000F542500B46024A1C
:103FC00004210C304FF0EAB9F07C0C0810B504461F
:103FD0004DF032F9002205214DF08AF804F54250E7
:103FE000034ABDE8104004210C304FF0D7B900BFA0
:103FF000FC7C0C0813B50B464AB100F54250009208
:104000000421054A0C304FF0C9F902B010BD02B0CE
:10401000BDE81040FFF7D0BF147D0C0808B500F5CF
:104020004250064A04210C304FF0B8F94DF004F923
:10403000BDE80840002208214DF05AB8287D0C0840
:1040400038B504460D4683F043FD04F540533DB9B1
:10405000D3F8C422C3F8C8020AB9C3F8C40238BDF1
:10406000D3F8C822801A642884BF0022C3E9B12291
:10407000F5E7000037B5044600F59A403C307BF088
:1040800077FB04F54052C0F3803592F8AA32C3F3AF
:104090004001A9421DD065F3410304F5425482F862
:1040A000AA320C346DB14DF0C7F802220B214DF04D
:1040B0001FF8094A0221204603B0BDE830404FF006
:1040C0006DB94DF0B9F82A460B214DF011F8034AAD
:1040D000F0E703B030BD00BF407D0C085C7D0C08EC
:1040E00038B50A460C460621054601F005FC28B104
:1040F000054A137843F00803137038BD214628465B
:10410000BDE8384006F094BEDC84002038B50A468D
:104110000D461521044601F0EFFB28B1094A13783A
:1041200043F00803137038BD04F5425004210C30ED
:10413000054A4FF033F929462046BDE8384006F0DD
:1041400077BE00BFDC8400206C7D0C0838B50A46C1
:104150000D461521044601F0CFFB28B1094A13781A
:1041600043F00803137038BD04F5425004210C30AD
:10417000054A4FF013F929462046BDE83840FFF7BD
:10418000AFBF00BFDC840020947D0C0838B50A4620
:104190000D461B21044601F0AFFB28B1094A1378F4
:1041A00043F00803137038BD04F5425004210C306D
:1041B000054A4FF0F3F829462046BDE83840FFF79E
:1041C0008FBF00BFDC840020AA7D0C0838B50A46EA
:1041D0000D461121044601F08FFB28B1094A1378DE
:1041E00043F00803137038BD04F5425004210C302D
:1041F000054A4FF0D3F829462046BDE8384006F07E
:1042000017BE00BFDC840020BC7D0C0810B500F593
:10421000405494F8AA329A0623D4D4F8B40203681E
:104220001B689847032808D005D802280ED194F8B7
:10423000A802C00914E01B28F9D194F8A80200F0E4
:10424000A000A0F180035842584109E0B4F8A80248
:1042500020F4FE4020F07F0080B2003818BF01201B
:1042600010BD0120FCE7000038B500F540550446BC
:1042700095F8CD32184A43F0080300F5425085F80E
:10428000CD3202210C304FF089F84CF0D5FF0122DD
:1042900017214CF02DFF2046FFF7B8FF38B1284614
:1042A0000122BDE8384015210C30F9F791BED5F850
:1042B000B40203681B689847062806D104F5AA4093
:1042C0004830BDE8384007F0BDBF20460B21BDE8AF
:1042D0003840FFF705BF00BFD07D0C0870B500F572
:1042E0004055D5E9B1239B1A41F2883293420646E4
:1042F00011D9D5F8B40203681B6D9847044695F8A8
:10430000CD32C3F3C003A34213D034B13046BDE86D
:104310007040FFF7A9BF0024F1E74CF08DFF224663
:1043200017214CF0E5FE95F8CD3264F3C30385F810
:10433000CD3270BD0B46013B1146062B18D8DFE885
:1043400003F00406080A0C13150006F071BDFFF710
:10435000C7BEFFF7FBBEFFF7D9BE00F540500122F4
:1043600014210C30F9F734BEFFF710BFFFF72EBF52
:1043700070470000F8B5044604F500574CF05CFFA8
:10438000012205214CF0B4FE97F8A235072B98BF07
:10439000304A204694BFD55C0125FFF737FF68B14E
:1043A0002D4A2E492046FFF725FE04F540500122F4
:1043B00010210C30F9F70CFE002514E004F54056EE
:1043C000D6F8B4020368DB6C984798B196F82D389C
:1043D00083B196F92C38012B0CDC214A2149204667
:1043E000FFF708FE0125294620460322BDE8F840D4
:1043F000FFF7A0BFD6F8B4020368DB6C984718B18A
:10440000D7F8503E190715D4D6F8B40203681B68D4
:104410009847032803D1D7F8503EDA070DD4D6F8D1
:10442000B40203685B6A984768B90C492046FFF7F5
:10443000C3FDD8E70A4A0949D1E70B4A0749204694
:10444000FFF7D8FDB8E7D7F8503E5B07EDD5074A30
:10445000F4E700BFB87E0C08F07D0C08FA7D0C086C
:10446000007E0C08137E0C08237E0C08337E0C089B
:1044700038B5044615464CF0DFFE012206214CF00B
:1044800037FE2046FFF7C2FE98B104F540500122E6
:1044900007210C30F9F79CFD144A15492046FFF717
:1044A000A9FD0025294620460422BDE83840FFF733
:1044B00041BF04F54053EDB2D3F8B4020368DB6C9E
:1044C000984768B104F50053D3F8503E1B0707D551
:1044D00035B1084A06492046FFF78CFD0125E1E782
:1044E00003492046FFF768FDDCE700BFF07D0C08BC
:1044F000527E0C08007E0C082DE9F041044604F5BC
:1045000000574CF099FE012208214CF0F1FD56F0C5
:104510009DFF97F89135072B98BF384A04F5405610
:1045200098BFD55CD6F8D83293F8CB8088BF0225E7
:10453000B8F1000F0BD132492046FFF73DFD0025B1
:10454000294620460522BDE8F041FFF7F3BE20468C
:10455000FFF75CFE60B104F54050012212210C30DF
:10456000F9F736FD274A26492046FFF743FDE6E7DF
:10457000D6F8B4020368DB6C984768B196F82D381A
:1045800053B196F92C38012B06DC1F4A1F492046EF
:10459000FFF730FD0125D3E7D6F8B4020368DB6CE2
:1045A000984718B1D7F8503E190713D4D6F8B4027B
:1045B00003681B689847032803D1D7F8503E9A0731
:1045C0000BD4D7F8503EDB0609D40D492046FFF73F
:1045D000F3FCB5E70C4A0A49D9E70D4AC3E7D6F818
:1045E000B4020368DB69984706460028EDD1094A02
:1045F00003492046FFF7FEFC3546A1E7C07E0C08C4
:104600003B6A0C08F07D0C08007E0C084C7E0C0800
:104610005A7E0C086F7E0C08F8B500F5005504466C
:1046200095F99135BBB300F54056D6F8387297B37B
:1046300083F04EFA05F6A86595ED000ADFED167ACF
:104640009FED161ADFED160AC71B20EE270A8D20F4
:1046500024F074FBBCEEC00A10EE103A9F420CD25C
:1046600096F8CD329A0716D520460021F9F70AFEB2
:104670002046BDE8F840FFF7D1BC0CD996F8CD3202
:104680009B0708D420460121F9F7FCFD2046BDE830
:10469000F840FFF731BFF8BD00007A440000804FBA
:1046A000000000002DE9F341074600F59A403C3038
:1046B0007BF05EF807F54054C0F38048019083F02A
:1046C00007FA94F8D0324345454606460DD007F523
:1046D000425084F8D0820C30002D41D03B4B3C4AF4
:1046E000C4F8D46202214EF059FE94F8D03207F596
:1046F000005843B394F8D1322BBBB8F9BE3E9FEDBE
:10470000350A9FED351ADFED350A07EE903AF8EEDF
:10471000E77A40F2571027EE800A24F00FFBBCEE38
:10472000C00AD4F8D40210EE103A361A9E420AD9C2
:10473000012307F5425084F8D132294A234B022144
:104740000C304EF02BFE98F9BD3E002B94F8CD3284
:104750000DDC6FF3451384F8CD3202B0BDE8F08173
:104760001A4B204AC4F8D48284F8D182BAE7C3F342
:104770004012AA42F1D065F3451384F8CD329B066E
:10478000EBD5194BD3F8B40203681B69984700288E
:10479000E3D04CF051FD01221F214CF0A9FC38461A
:1047A000FFF734FD48B107F54050012221210C30BC
:1047B00002B0BDE8F041F9F70BBC98F8BD1E3222FB
:1047C000384602B0BDE8F041FFF7B4BD887E0C0862
:1047D000977E0C0800007A440000804F0000000023
:1047E000AD7E0C08A27E0C08B85B002008B5044B17
:1047F00001221A7083F060F9024B186008BD00BFF7
:104800005183002054830020014B00221A7070470E
:10481000518300202DE9F041044683F04DF92A4BE5
:10482000B4F8BE201988294E914205460ED01A8050
:10483000274B18603378A3B1002434704CF0FCFC93
:1048400022461321BDE8F0414CF052BC3378214F91
:10485000DBB93B782BB11E4B1F4A1B68C31A93422E
:1048600001D8BDE8F0810123337004F54053D3F83B
:10487000D80290F8CB3013B103689B6A98474CF08C
:10488000DBFC012213214CF033FC3B78002BE8D0F9
:104890003378002BE5D00E4A10491368EB1A8B428F
:1048A000DFD904F540541560D4F8D80290F8CB3025
:1048B000002BD6D000217BF015FFD4F8D802036876
:1048C000BDE8F0415B6A1847528300205083002006
:1048D000548300205183002080841E0040420F003A
:1048E0002DE9F84300F5405500F500580446D5F889
:1048F000B40298F8A4740368DB6C9847014650B979
:1049000095F9A832002BA5BFD5F8D83293F8CB0083
:10491000012180F0010104F5115909F128094846E7
:1049200060F040FCD5F8D83293F8CB300646002B27
:104930007BD0002865D03E4B93F9A832002B04DBD6
:1049400002463C49484660F007F898F96E7457B142
:1049500095F9A832002B0EDA04F5405001220F2100
:104960000C30F9F735FB4CF067FC3246BDE8F843F4
:1049700009214CF0BDBBD5F8B40203685B699847C8
:1049800058B195F9A932002B07DA95F8CD32DA073C
:1049900003D498F8A434DB07DED53146484660F0EE
:1049A00067FCDFED257AB4EEE70AF1EE10FA05DDDB
:1049B0000A220921204600F09FFFD4E7023F032F7F
:1049C00011D801A353F827F0B1490108D9490108CA
:1049D000F7490108FD4901080A221521204600F087
:1049E0008BFF0028BFD10A220621204600F084FF59
:1049F0000028B8D1DCE70A221121F6E70A221521A6
:104A0000F3E797B198F8A4347BB9094B93F9A8322E
:104A1000002B06DB04F54250084A05210C304EF00D
:104A2000BDFC4CF009FC0022A0E7BDE8F88300BF04
:104A3000B85B0020C87E0C080000C842D17E0C087C
:104A400070B500F5405300F59A453C3586B093F8B3
:104A50005010044628467AF039FE02A812F098FD5C
:104A600004F5B25002A918300CF054FF04F580434D
:104A7000049AC3F8342D059AC3F8382D28467AF0E5
:104A800077FE82061AD528467AF080FE04F59A450C
:104A9000FDEEC07A2C3504F5805417EE901A0222F0
:104AA000284617EE906A12F079FD94F8D438DB07A7
:104AB00006D401223146284612F070FD06B070BDC2
:104AC0000121284612F0FCFD0028F2D0F6E7000094
:104AD00070B500F5804486B0B4F8BC3E8B420D46FC
:104AE000164603D1D4F8B83E934221D082F0F0FFAD
:104AF000D4F8B43EC31A132B1AD9C4F8B86EA4F86C
:104B0000BC5EC4F8B40E4CF097FB044682F0E8FF9C
:104B1000084B094A1B68CDE90453084B0193084B25
:104B20000093CDE90201074B074920464CF010F9EC
:104B300006B070BD58830020E87E0C08007F0C088A
:104B4000C0540C08FC370C08FB7E0C0838B500F587
:104B500040540D4694F8A932C3F380138B420BD016
:104B600021B14CF069FB11214CF0A2FA94F8A93262
:104B700065F3861384F8A93238BD0000F0B52DED39
:104B8000048B00F540568BB0D6F8D83293F8CB3072
:104B9000054600F58044002B67D096F9A832002B1B
:104BA00063DBD6F8B40203685B699847002861D1DB
:104BB000D4F8580D9FED440A6C3027F0CDFA0AAABC
:104BC000CDED080A8DED091A8DED070A12E90700EF
:104BD00004AB01AF83E8070087E80700384627F0F9
:104BE00029F8D4F8583D05F59A400C30D3ED368AB3
:104BF000B0EE409A4DF07CFF27F0ACFED4F8603D5B
:104C0000D6F8B402D3EDDB9A0368DB6CB0EE408AD1
:104C10009847DFED2E7AB4EEE79AF1EE10FA02DC57
:104C200096F8B0320BB100283AD0DFED297A68EE61
:104C3000A78AF3EE0E7AF4EEE78AF1EE10FA2FDC93
:104C4000F0EE087AB4EEE78AF1EE10FA28DCF5EE21
:104C5000C09AF1EE10FA23DAD4F8580D03689B6F6E
:104C600098470BB0BDEC048BF0BDD4F8580D036829
:104C70009B6F0FE005F50055D4F8580DD5F8F02ED0
:104C80000368B2F90820002A03DCD6F8AC22022A15
:104C9000EED1DB6F0BB0BDEC048BBDE8F0401847E4
:104CA000D4F8585DDFED0B0A2B68D3F88060D4F898
:104CB000603D40F2AB1093EDC90AB7EE001A24F044
:104CC0003DF82846B047CCE79F0CB3450080BB4475
:104CD000E02E65420000000000F5405090F8B00260
:104CE000704700002DE9F04100F54055064695F863
:104CF000A832B1EBD31F0C4648D0254B00221A60D6
:104D000000293FD04CF098FA12214CF0D1F995F8D7
:104D1000A83264F3C71385F8A83284F001086BF059
:104D200041F941466BF01AF906F50057B8F1000F4A
:104D300006D097F826351BB982F0CAFEC7F82805B9
:104D400087F8268514B3B7F874355B071ED5D5F8F8
:104D5000D83293F8CB30CBB1D5F8B40203685B6995
:104D6000984798B9D5F8B402036820219B69984701
:104D700060B106F540500122BDE8F0410D210C3034
:104D8000F9F726B94CF058FA1C21BEE7BDE8F081CE
:104D9000588300202DE9F04F2DED0A8B00F540558A
:104DA0008DB0D5F8D83293F8CB60044600F5804733
:104DB0001EB90121FFF796FF0BE095F9A822002A02
:104DC00065DAD5F8B40203689B6C9847064600285C
:104DD00041D04FF0000B95F9A822B24E002AC0F244
:104DE0005581D6ED007AB4F9A420B8EE677A1AB9E5
:104DF000B4F8A220A4F8A420B4F8A430DFEDAA6A85
:104E000007EE903AF8EEE77A67EEA67AB4EEE77A24
:104E1000F1EE10FAACBF012100212046FFF796FE0B
:104E200095F9A822002A95F8A922B8BF4BF0010BEA
:104E3000530697F8A02E48BF4BF0020B0AB14BF077
:104E4000080B3268594620460DB0BDEC0A8BBDE810
:104E5000F04FFFF73DBED5F8D832204693ED0C8ACF
:104E6000F9F7E0FAB4EEC80AF1EE10FAB1D5D5F8C8
:104E7000D83293F8A130032BABD14AF0E9FC4FF4C0
:104E8000801142224AF09CFC3146204692E797F876
:104E9000A0AEBAF1000F03D0824A0023136098E756
:104EA000D7F8580D93F8079003685B6F98478046D2
:104EB0000090D5F8B40203685B69984720B1D5F833
:104EC000AC32022B00F0E480B9F1000F0CBF4FF0C0
:104ED000000B4FF4007BB7EE00BAB8F1000F02D020
:104EE0004BF4806B009604F59C4808F16808404636
:104EF00063F036FB0130D7F8580D9FED6C0A9FED3B
:104F00006CCADFED6C8A0CBF012302236C3008EE03
:104F1000103A27F021F90CABCDED0A0A8DED0B1AF2
:104F20008DED090A13E907000DF10C0E0DF1180CB7
:104F30008CE807008EE80700704626F07BFED7F865
:104F4000582DDFED5D7A92ED36AA2AEE27AAB4EE4F
:104F5000CC0AF3EE0EBAF1EE10FA04F59A40B4EE74
:104F6000EBAAC8BF4BF4807B0C30F1EE10FAC8BF3F
:104F70004BF4807BF0EE40AA4DF0BAFD27F0EAFC3E
:104F8000B8EEC88A04F59A40B4EEC80AF1EE10FAF9
:104F900000F13C0098BF4BF0800BF0EE409A7AF0A5
:104FA00001FC68EE288AB0EEC09AB4EEE89AF1EE01
:104FB00010FA204648BF4BF0400B09F021FD0028B5
:104FC00046D14BF0200B0196404663F0C9FA012808
:104FD0004FD14BF0100BB2463249B9F1000F53D00C
:104FE000009B002B50D0F4EECCAAF1EE10FA4BDC73
:104FF000B4EEEBAAF1EE10FA46DCF4EEC89AF1EE4C
:1050000010FA41D8B4EEE89AF1EE10FA3CD5019BC3
:10501000D3B3BAF1000F37D00A68B4F9A40007EE91
:10502000902AB8EE677A18B9B4F8A200A4F8A400E0
:10503000B4F8A43007EE903AF8EEE77A67EE8B7A90
:10504000B4EEE77AF1EE10FA19D501320A60C2E641
:1050500004F53C500C304DF027FDDFED187A90ED53
:10506000007AB4EEE77AF1EE10FAAAD400230193A5
:10507000AAE7404663F074FA0130ADD1A9E70121F7
:105080002046FFF72FFEA6E60022DFE70121C4E657
:10509000B9F1000FB0EE08BA0CBF4FF0000B4FF49F
:1050A000007B1DE758830020CDCC4C3E9F0CB345C0
:1050B0000080BB440000C842E02E65420000484327
:1050C00030B500F5CD530833044693E8070089B0A6
:1050D00002AD85E807009FED1D7ADDED047A77EEDD
:1050E000877A9FED1B7ACDED047AD4ED2B7AF0EE22
:1050F000E77AF4EEC77A04F59A40F1EE10FA00F17F
:105100000C000BD5B4F9A23007EE903AF8EEE77A2E
:10511000F7EE006A86EEA77A84ED2B7AD4F8AC30ED
:10512000019301AA29464DF089FD2046FFF732FE82
:105130002046FEF769F92046FEF740FA2046FEF7C2
:1051400009F82046FEF7B0F809B030BD0AE81C4166
:105150000000003410B504462DED028B1D2057F0E1
:10516000A5FD60B304F54053D3F8B40200F0C2FAD1
:10517000192108EE100A04F5885043F0AFFE02280A
:105180001AD00338012808D804F53C500C304DF0F3
:105190008BFC90ED008ABDEEC88AB8EEC88A9FED00
:1051A000090A28EE000ABDEC028B04F59C40683029
:1051B000BDE8104063F05ABA9FED038AEDE7BDECFD
:1051C000028B10BD0AD7233C00000000134A026086
:1051D000134A426002F1740181601249C16002F514
:1051E000205101610839416124398161A2F5716161
:1051F000C16101F55C51016202F55761416202F53E
:105200001861816202F68411C16202F6881102F609
:105210008C124263044A01638263704734900C0825
:10522000205100201C790020D02C00201C2953D8AC
:10523000DFE801F0130F171B27232F1F522B5233C8
:105240005252373B3E424652524A525252525252A8
:105250004E0000F59D404430704700F5AB4054309F
:10526000704700F59E400430704700F59E40403086
:10527000704700F5A6401C30704700F5A840783014
:10528000704700F5A7406C30704700F5A8403030FB
:10529000704700F5AA404830704700F5A6405C30E2
:1052A000704700F5A7401830704700F5A240FAE7B4
:1052B00000F5A9403430704700F5A54058307047DC
:1052C00000F5AC401030704700F5AC4060307047DE
:1052D00000F5AD407C3070470020704773B50B6817
:1052E00005461B6C08460C4616469847034605F5CE
:1052F00042500F4A009604210C304EF04FF84BF00C
:105300009BFF236805461B68204698470A210246F2
:1053100028464BF0EDFE074B93F8A9329B0641BFA0
:10532000054A137843F00403137002B070BD00BF48
:10533000047F0C08B85B0020DC84002038B50C4AE0
:10534000182305460C464AF0F7F878B1214628465E
:10535000FFF76CFF30B10146064A2846FFF7BEFF53
:10536000002038BD28464AF02DF8F9E70120F8E77B
:10537000847F0C08247F0C0810B500F50053002230
:1053800083F8A02F094B044693F8A81200F5804338
:1053900004F54054D3F8580DC90974F02BF8D4F82B
:1053A000B4020368BDE81040DB681847B85B002012
:1053B00070B50546086803685B690C461646984751
:1053C00090B1306803685B69984768B905F5405348
:1053D000D3F8D82292F8CB2032B193F9A832002B1F
:1053E00002DB2846F9F734F804480AF0BFF82068D1
:1053F0000368BDE870409B68184700BF1884002010
:1054000070B500F540550446D5F8B4020B4E03685C
:10541000DB6998473074D5F8B40203681B68984775
:10542000F070D5F8B40203685B6C9847014604F548
:10543000B0500430BDE870403FF000BBBD84002098
:1054400070B52DED028B244B93F8CD32DB0782B083
:1054500006460D461446B0EE408AF0EE608A06D548
:1054600000232B60236002B0BDEC028B70BD56F0B0
:10547000EDF8037F002BF3D0F36A9FED181A1B6839
:105480009FED170AB3F9083007EE103AB36A1B68AC
:10549000B3F9083007EE903AB8EEC77AF8EEE77A3B
:1054A00067EE000A68EE811A27EE800A28EE011ADC
:1054B00001A9684624F036FBDFED0A6A9DED007A0B
:1054C000DDED017A27EE267A67EEA67A85ED007A81
:1054D000C4ED007AC7E700BFB85B00200AD7233CC1
:1054E000530469390000C84270B52DED028B88B0B5
:1054F000002302930393364B93F8CD3213F0010F40
:105500000646B0EE408A06AD02AC03D156F09EF8D6
:10551000037F5BB994E8030085E803009DED060A6C
:10552000DDED070A08B0BDEC028B70BDB36ADFED9C
:10553000296A1B68B3F9083007EE903AF36A1B68D2
:10554000B3F9083007EE103AB8EEC77AF8EEE77A0A
:1055500027EE267A67EEA67AF1EE476ACDED026A6B
:10556000DFED1D6ACDED037AB0EEC77AB4EEE67AD0
:10557000F1EE10FA06D5F0EEE77AF4EEE67AF1EE07
:1055800010FAC7D403AA21461448F8F791FFDDEDBD
:10559000027A9DED037AF0EEE77AB0EEC77AF4EE88
:1055A000477AF1EE10FACCBFB0EE670AB0EE470AC8
:1055B000204626F08DFA04A88DED040ACDED050AEB
:1055C00026F038FB204688EE000A26F0B1FAA1E763
:1055D000B85B00205304693900000034B82B002068
:1055E000094B93F9A822002A0CDAB5EEC00AF1EEB5
:1055F00010FA07D9D3F8D83293F8A100C31E584245
:105600005841704700207047B85B0020436A1B6810
:1056100093F8CB3043B1054B93F8A80200F0A000FB
:10562000203818BF0120704701207047B85B002068
:1056300010B5436A04461868D1B102217BF062F8C4
:10564000236A9FED0C1A18680368F0EE410ADB6AC2
:10565000B0EE410A9847236A074A1868D2ED000A5B
:1056600003689FED040A5B6EBDE8104000211847F7
:105670000121E3E7000000002851002010B5436A33
:1056800004461868002930D002217BF03BF8236AD9
:10569000186873F07FFE636A1B6893F8A130012BD2
:1056A00004D8236A0121186874F00EFC6369186835
:1056B00077F01AFD6369186877F076FD63699FEDEE
:1056C0000C0A186877F09CFF6369186878F00AF88C
:1056D000236A9FED071A18680368BDE81040DB6A6B
:1056E000F0EE410AB0EE410A18470121CDE700BFB4
:1056F0000000000013B5044601A90C4809F00CFA9B
:1057000010B1019802B010BD6369186876F0F6FB1D
:1057100018B9074BD3F8300DF4E7064801AA032166
:1057200011F072FF0028F4D0EBE700BFB82B002087
:10573000B86B0020E478002070B504462DED028B94
:1057400000296AD18368B3F96258642DB8BF642513
:10575000FFF7D0FFA8426268A4BF324B93F8A9526A
:10576000B2F93430ACBFC5F380150125002BDBBF87
:1057700063691B685B4293EDC48AC8BF07EE903A29
:10578000B2F93230C8BFB8EEE78A002BB8BF5B422F
:105790009BB25B4207EE903AA368F8EEE77AB3F962
:1057A0006268F4EEC87AF1EE10FAD8BFB0EE678AFC
:1057B0002046642EB8BF6426FFF79CFF6369A26B86
:1057C0001B68D2ED001A93EDC61AD3ED0E0A311AFA
:1057D00000EE101AB8EEC00A23F092FD6368B3F928
:1057E0003230002BB8BF5B429BB25B4201EE103AF5
:1057F00040F29720B8EEC11AF0EE480A23F09EFA64
:1058000063692946186876F01DFCBDEC028B63695C
:10581000BDE87040186877F065BF9FED030A00256A
:10582000EEE700BFB85B002000000000436A186884
:1058300003681B691847000038B52DED028B03681B
:105840000446D3F880309847236B2A481B68F0EE53
:10585000408AB3F9085009F071F84FF47A72041EC7
:105860004FF000012846D8BF4FF4FA7423F0A4FA91
:105870008442B6EE000A2ADD07EE900AB8EEE77A17
:1058800007EE904A27EE007AF8EEE77A87EE278A4D
:105890004FF46D7038EEC00AF5EE087AB1EE400AAA
:1058A00080EE270AB7EE001AFEEE000A23F046FA51
:1058B000F7EE007A77EEC07A28EE000A20EE080AAA
:1058C00020EE080AA7EE880ABDEC028B38BD031B48
:1058D00007EE103AC4F57A74B8EEC77A07EE904A2C
:1058E00027EE007AF8EEE77A87EE278A38EE008A0C
:1058F000CEE700BFB82B00202DE9F04F2DED028B35
:1059000000F5804900F5405899F8C04E89F8C02E3E
:105910000546D8F8B402036883B01B680F461646E4
:105920009847B84221D105F500551A2E85F824650F
:1059300007D130B905F68465D9F8583D2A68C3F80F
:10594000FC208C4B93F8A932980606D401242046FB
:1059500003B0BDEC028BBDE8F08FB442F6D0864AAE
:10596000137843F002031370F0E7022E0CD01B2FC4
:1059700012D105F59E403146403003B0BDEC028B9C
:10598000BDE8F04F01F05AB939462846FFF7D6FC7A
:1059900004460028EBD1DAE739462846FFF746FCF3
:1059A0000446019018B9284649F00CFDCFE7D8F815
:1059B000D83293F8CBB003685B699847019A05F534
:1059C000A6435C338BF0010A9A4208BF0120BBF169
:1059D000000F08D10198036851465B689847044658
:1059E00048BB664A22E098F9A832002B80F2B480C6
:1059F000002800F0B180DFF87CB1DBF8B402036866
:105A00005B6998470446002840F0A6800198FFF79C
:105A100013FFABF54050B0EE408AF8F703FDB4EE4B
:105A2000C08AF1EE10FA40F39780554A0199284652
:105A3000FFF754FC8BE705F54A5101AA343128469B
:105A400005F50054FFF7B4FC0198C8F8B40284F8D7
:105A5000246503681B689847014605F59D5032464A
:105A600010304AF0FBFE05F5425000210C3054F096
:105A70001BFF94F96E3423B105F5115028305FF007
:105A80001BFCD8F8B40203681B689847C21E50423A
:105A9000504104F6546289F8E80DD9F8583D12686F
:105AA000C3F8F82004F68462D9F8583D1268C3F8A8
:105AB000FC20012F01D00B2F06D104F66C64D9F81D
:105AC000583D2268C3F8FC202846FFF799FC294B73
:105AD00093F8A9329B063FF542AF37E705F500532F
:105AE00093F86824002A3FF475AFB3F88424D107F3
:105AF0007FF570AF93F8A424002A3FF46BAFD8F879
:105B0000D82292F8CB20002A3FF464AF93F82435D2
:105B10000A2B7FF45FAF98F9A832002BFFF65AAF3B
:105B2000184A01992846FFF7D9FB00240FE71648C9
:105B300009F068F90028D1D1D8F8B40203685B698C
:105B400098470028CAD0019803685B6998470446C3
:105B50000028C3D10D4A69E7019803681B6998477B
:105B60000028E4D0084809F03BF904460028DED1BB
:105B7000074A5BE7B85B0020DC8400202A0D0E0892
:105B80004C7F0C08707F0C08B82B00205E7F0C083F
:105B90002AC00D080148FFF7AFBE00BFB82B002098
:105BA00013B504468DED010A62F072FC6369A26BC5
:105BB0001B6892ED001A93ED0E0AD3EDC60A01A9F7
:105BC00061F0F4FA9DED010A02B010BD436A186855
:105BD00003685B6A1847000038B5436A1C6894F88C
:105BE000CB10054661B920467AF08CFD6B6A1B68C4
:105BF00093F8A10018B1012814BF0320022038BD7A
:105C0000164803783BBBFFF7EBFC20BB144A92F825
:105C1000A83203F0A003202B17D0B5EEC00AF1EE96
:105C200010FA10D592F8AA325B070CD40121204655
:105C30007AF068FD6B6A1B6893F8A130012B0CBFEA
:105C400002200320DBE70221F1E7204602217AF05F
:105C500059FD0420D3E70120D1E700BF18840020BC
:105C6000B85B002010B52DED028B134B93F8CD32AD
:105C7000DB07044604D59FED110ABDEC028B10BD75
:105C800055F0E4FC037F002BF5D0636B186855F0EA
:105C900007FEA368DFED0A7A03F6AC0292ED008AF4
:105CA00003F50B63D3ED000A28EE278A23F0F4FEF8
:105CB00028EE000AE1E700BFB85B0020000000000A
:105CC0000000C8420148F8F71DBC00BFB82B0020F7
:105CD0000148F9F7ADB800BFB82B00200148FFF725
:105CE0000BBE00BFB82B002070B52DED028B7D4D93
:105CF00095F8A9328CB000260446580604960596FD
:105D000003D56369186875F06DFF95F8CD32D90732
:105D10005DD463689B899A071BD573484CF0C4FE19
:105D2000DFED727A90ED007AB4EEE77AF1EE10FAD8
:105D30000FDD4BF081FA3D214BF0BAF96C48092296
:105D40000521FFF7D9FD20B9092202212046FFF7DE
:105D5000C5FF636893F95430CBB365489FED658AFE
:105D6000F9F766F8E3689FED647A1B68D3ED0A7A69
:105D7000F4EEC87AF1EE10FAB8BFF0EE477AB6EE5C
:105D8000000A27EE800A2046FFF7AEFB8DED040ADD
:105D9000B0EEC00AB4EEC80AF1EE10FACDED050A75
:105DA00006D5F0EEE00AF4EEC80AF1EE10FA0ED4D1
:105DB00095F8AA321B0704D44BF03EFA49214BF068
:105DC00077F995F8AA3243F0080385F8AA3295F8D6
:105DD000AB326FF3820385F8AB32606909960A969D
:105DE00009AD2A4604A90068012375F065FF6369BF
:105DF000186877F0D9F96369186876F0B1FAA36882
:105E00008DED060ACDED070A8DED081AD3ED007A67
:105E1000F5EEC07AF1EE10FA52DD384B9FED388A7C
:105E2000B3F9643500EE903AF8EEE00A2046CDED85
:105E3000030AFFF75FFCA368DDED030AD3ED001A48
:105E40009FED2A0AB7EE002A07EE900A31EE822A69
:105E5000B8EEE71A22EE082A61EE881A22F0AEFEAA
:105E6000DFED287A20EE270ADFED277A20EE270AD9
:105E7000A5F008FDDFED257A20EE270A06A820EE22
:105E8000088A25F0D7FEB4EEC08AF1EE10FA17D5D5
:105E9000C8EE006A63699DED067ADDED077A27EEAC
:105EA000267A67EEA67A8DED067ACDED077A1B6825
:105EB000D3F88823C3F89423D3F88C23C3F898230A
:105EC000236A13491C682846FCF70AFB0B9B0093C6
:105ED00095E80C0006A9204673F00EFB0CB0BDEC53
:105EE000028B70BDB85B0020D878002000002F44E2
:105EF000B82B00200000003400007A43B84B00208B
:105F00000000C8420AD7233C35FA8E3C0AE81C41FF
:105F10000C83002013B504460191FFF7E5FE0199BB
:105F2000204602B0BDE81040FFF706BC0148FEF76E
:105F3000D9BE00BFB82B002000487047445C002049
:105F40000148F8F7CDBA00BFB82B002030B50F4D8F
:105F500087B0002304466946D5F8600D009301938D
:105F6000029376F015FAD5F8600D02A976F064FA7E
:105F7000009B0393019B04930222029B059303A9B8
:105F8000204611F011FE204607B030BDB86B00204E
:105F900000207047002070470020704700207047A5
:105FA0000020704700207047002070470020704795
:105FB00000207047002070479FED010A704700BF26
:105FC000000000000020704700207047002070474C
:105FD0000120704700207047002070470120704763
:105FE0000020704701207047012070470020704753
:105FF000012070470120704700207047004870471B
:106000009C7F0C08004870479C7F0C08836893F8BD
:10601000C038DB0706D5002380F83C30024B022253
:10602000C3F8AC2201207047B85B002090F83C30E8
:1060300043B9836893F8C038DB0742BF034B0122A2
:10604000C3F8AC22002380F83C307047B85B0020D6
:10605000012380F83C3070472DE9F0432DED0C8B87
:10606000F0EE409A20EE000A97B00025A0EEA00ABC
:1060700004468946B0EE41CAF0EE60AA90461F463B
:10608000019502950395049505950695A5F010FEDA
:10609000F7EE00CAB4EEEC0AF1EE10FAC8BFCCEE8F
:1060A000807AA36803F67C0203F5086392ED009AF8
:1060B0009FEDC5DAD3ED000AC4BF69EEA79A6AEE78
:1060C000A7AAB0EE690A23F0E7FCA36829EE0D9AAF
:1060D00003F67C0203F50863D2ED008AD3ED000AD3
:1060E00029EE009AB0EE6A0A23F0D6FCA36868EEA7
:1060F0008D8A03F6940203F69803D3ED000A92ED1D
:10610000008A68EE808AB0EE4C0A23F0C5FC636812
:1061100028EE0D8A93F9703028EE008A002B00F0EB
:10612000D980236A9FEDA90A18686C3026F014F80C
:10613000B0EE60AACDED080A8DED091A8DED070AC3
:1061400022F0A6FDBDEEC0BAA14940F6B8321BEE62
:10615000100A22F021FE434207EE903A6368F8EEFF
:10616000E77A93ED1A7A67EE877AB0EE4A0ACDEDB8
:10617000017A22F08DFDFDEEC0BA40F6B8329449A6
:106180001BEE900A22F008FE42426368039507EE78
:10619000902A93ED1B7A93F97030F8EEE77A022B90
:1061A00067EE877ACDED027A6ED18A4BB3F964350A
:1061B0000AEE103AB8EECBBAB8EECAAA236AB4EE29
:1061C000CABAF1EE10FA1A683DDDA368DFED820A63
:1061D000A16B92ED051AD1ED001A03F67C0393ED45
:1061E000007A27EE0D7A3AEE4B0AC7EE200A23F02A
:1061F00087F8DDED017A37EE800A8DED010AB8EE01
:10620000EB0A236AB4EECA0AF1EE10FA1A6834DD1A
:10621000A368A16B92ED061AD1ED001A03F67C0378
:10622000D3ED000A20EE8DDADFED6B0A3AEE400A7C
:10623000CDEE200A23F064F8DDED027A37EE800A15
:106240008DED020A20E0B1EE4A0AB4EEC0BAF1EEDA
:1062500010FAD4D5A368A16BDFED5F0AD1ED001A67
:1062600092ED051A03F67C0393ED007A27EE0D7A82
:1062700030EE4B0AC7EE200AB9E7B1EE4AAAB4EEF7
:10628000CA0AF1EE10FAC3D4236AD3F800C00CF1A5
:1062900084030FCB12AD85E80F000EAE0AAD86E881
:1062A0000F0085E80F0004AB01AA2946604673F091
:1062B000BFFD636893F97030022B16D1DDED047ACF
:1062C00039EE279ADDED057A78EEA78ADDED067ABC
:1062D00038EE278A89ED009AC8ED008A87ED008A9A
:1062E00017B0BDEC0C8BBDE8F083F0EEE99AF0EE50
:1062F000EAAAF4EEE9AAF1EE10FA48BF6D46CDED38
:10630000009ACDED0AAAD5ED007ADFED340AB0EEA1
:10631000CCCAF4EECC7AF1EE10FAD8BF35468DED4A
:106320000ECA95ED007ADFED2E7A87EE270AAD20B2
:10633000B7EE001A3CEEC00A22F000FDE369D3ED8F
:10634000937A04A820EE270A25F006FFF0EEC07A23
:106350008DED061AB0EEC91A31EE671A8DED040AFA
:10636000B0EEC11A39EE000ACDED050AB520F1EE06
:10637000410A22F0E3FCB0EE409A9DED050AB0EE32
:10638000E81AF0EEC07A31EE671A38EE800AB0EE05
:10639000C11AF1EE410ABA2022F0D0FCF0EE408A98
:1063A0009DED060AB0EEC81AF0EEC07A31EE671A1B
:1063B00038EE000AB0EEC11ABF20F1EE410A22F019
:1063C000BDFCB0EE408A85E70000C8429F0CB34593
:1063D00048F4FFFFB84B002000007A4400000000A2
:1063E00000A08C4510B52DED028B836A044686B063
:1063F000186855F055FAE36A1868B0EE408A55F00F
:106400004FFA636B8DED010A186855F049FA05AB38
:10641000B0EE401A03A92046DDED010A04AAB0EE51
:10642000480AFFF719FE636A186890F8CB10002934
:106430003AD17AF067F92046FFF7FEF9636A1B68E4
:1064400093F8A1100129B0EE408A3DD0032944D031
:1064500051B9236A0121186874F0ECFB236A1868AB
:1064600072F082FF9FED208A236AA268186892F872
:10647000C02803689DED030ADDED040A9DED051AB1
:1064800092074CBFDB6B9B6B9847236A174A1868CF
:10649000D2ED000A036800215B6EB0EE480A98470F
:1064A00006B0BDEC028B10BD114B93F9A922002A56
:1064B00006DBD3F8AC32022B04D190F8A1300BB933
:1064C0000121B6E70221B4E7236A186874F0B2FB31
:1064D000236A186872F05EFFC4E7D9790029C3D136
:1064E0002046FFF723FDBFE70000000028510020F1
:1064F000B85B0020836893ED140AB5EEC00AF1EE94
:1065000010FA01DCFFF792B97047000070470000F5
:10651000002070470120704702207047002070471C
:1065200000207047012070470020704781F0010073
:1065300070470000012070470120704700487047F5
:1065400034800C080048704740800C0838B5436917
:106550000446186875F0F4FD18B96369186876F098
:1065600073FF636920461D68FFF7EAFC6368B3F9AF
:106570003820B3F9363000EE903A434201EE102A4B
:1065800000EE103AB8EEC11AF8EEE00AB8EEC00A12
:10659000284675F0C1FC636920461D68FFF7D0FCF2
:1065A0006368B3F93820B3F9363000EE903A4342CD
:1065B00001EE102A00EE103A2846B8EEC11AF8EEA5
:1065C000E00AB8EEC00A75F021FD012038BD0000D8
:1065D00030B52DED028B0446436985B01D68FFF789
:1065E000AFFC6368B3F93820B3F9363000EE903A67
:1065F000434201EE102A00EE103AB8EEC11AF8EE4E
:10660000E00AB8EEC00A28465B4D75F085FC2046CE
:10661000FFF75EFBB5F9643508EE103A236A186897
:1066200003689B6E9847B8EEC88AF0EE400A02AA4B
:1066300001A9B0EE480A2046FEF702FF2046FFF708
:1066400011FB236B1B68B3F90830F0EE408A00EEB3
:10665000103A2046B8EEC00AFFF734FB2046B0EEF1
:10666000408A8DED030AFFF76BFC6368B3F936309F
:1066700001EE103A434200EE903AB8EEC11AF8EE3D
:10668000E00A2B20B0EE480A22F058FB20468DEDA0
:10669000030AFFF7A1FA042813D8DFE800F0032F5C
:1066A000252A4B00236A186872F05EFE236A0021D7
:1066B000186873F009FC63699FED300A186876F07A
:1066C0009FFF236ADDED020A18689DED010A036849
:1066D000B0EE681ADB6A98476369186877F002F8C9
:1066E00005B0BDEC028B30BD236A0121186873F040
:1066F000EBFB236A186872F04DFEDCE7204D2B7827
:1067000063B963689FED1F1ADFED1C0A93ED040A5D
:10671000452022F013FB284608F010FF20469DED8F
:10672000030AFFF73DFA16488DED030A03A908F0A6
:106730003FFFC6E7636A0221186879F0E3FFB5F905
:106740006435114800EE103A02AA01A9B8EEC00A59
:1067500060F05CFA20469DED030AFFF721FA0B4832
:106760008DED030A08F0F4F963699DED030A1868DA
:1067700075F058FCA5E700BFB84B002000000000F2
:106780001884002000007A44B07900204C5B00207F
:106790000020704790F8B931002B14BF1B20032054
:1067A00070470000002070470120704790F890016A
:1067B000062804D0A0F1090358425841704701202F
:1067C00070470000012070470120704790F8B90120
:1067D000034A044B002814BF10461846704700BFF8
:1067E000D8800C082DD30D0890F8B901034A044B4A
:1067F000002814BF10461846704700BFE4800C08FC
:106800002DD30D0890F890010A3818BF0120704769
:1068100090F8B9312BB9044BD3F8A00E00F0010069
:1068200070470020704700BFB84B002090F89031AF
:1068300023B9034B187880F001007047002070479F
:10684000FC83002038B590F89041012C054601D01A
:10685000002038BDC368186803681B699847002882
:10686000F6D1EB681B68204683F8B848F1E70000D2
:10687000C3681B68002283F8B82801207047000015
:1068800070B52DED028B002380F8B931B0F870306F
:10689000012B84B004460D4601D8002946D0636A16
:1068A000254E1B6893F8CB3073BB2448072384F82C
:1068B00090310368022B02D10021FBF753FC9FEDBE
:1068C000208AE368F0EE480A1868B0EE481AF0EE45
:1068D000481AB0EE480A012578F08AF984ED738AE7
:1068E00084ED748A84ED758A84F8B85104F59A7041
:1068F00026F01AF9134803F0B3FD96F8AA326FF3A5
:10690000C30386F8AA3211E096F9A832002BCCDA3C
:1069100004F13C0028F0BAF905460028C5D120460C
:10692000FFF70AFB084A02214CF038FD284604B064
:10693000BDEC028B70BD00BFB85B00200C83002053
:1069400000000000A47F0020EC800C0810B5044675
:10695000064890F8803F012B03D100F67C7026F0AA
:106960004BF9002384F8B93110BD00BFB86B00208B
:1069700010B52DED028B094B0446D3F8640DB0EE33
:10698000408A77F0CDFC9FED060A28EE008A0120B0
:1069900084ED748ABDEC028B10BD00BFB86B002083
:1069A0000AD7233C10B52DED028B094B0446D3F8D2
:1069B000640DB0EE408A77F0C3FC9FED060A28EE26
:1069C000008A012084ED758ABDEC028B10BD00BFEA
:1069D000B86B00200AD7233C10B52DED028B094B74
:1069E0000446D3F8640DB0EE408A77F0B7FC9FED13
:1069F000060A28EE008A012084ED738ABDEC028B22
:106A000010BD00BFB86B00200AD7233CC3681B68C9
:106A1000186975F0D7BD000038B5D0F89431044638
:106A20000D461BB981F054F8C4F8940181F050F878
:106A3000D4F89431C01A4FF47A73B0FBF3F0B4F881
:106A40009231984209D32046FFF776FA2B88044A00
:106A500006214CF0A3FC012038BD0020FCE700BF5C
:106A600008810C0890F89031052B05D1054BD3F81F
:106A70006C3DD86875F01EBDC36818680368DB6894
:106A8000184700BFB86B002008B590F89031052B6F
:106A90000BD1094BD3F86C3DD868243025F0CAF8E7
:106AA000BCEEC00A10EE100A08BDC368186803687F
:106AB0009B689847F4E700BFB86B002090F89031CE
:106AC0008B4206D00A2B80F8901102D10148FCF7C6
:106AD000D1BF7047B82B002073B501231E4E80F83C
:106AE0007530D6F8B432834205460A4614D10124E3
:106AF00085F8B941D6F8B402019203681B6898473B
:106B0000019A0146154849F0A9FE96F8A9329A065D
:106B10001BD4204602B070BD01910321FFF7DEF8BF
:106B2000019A04460028E2D185F875004AF084FBFA
:106B30001B220A214AF0DCFA96F8A9329B06E8D516
:106B4000074A137843F0040303E0054A137843F03F
:106B500002031370DDE700BFB85B0020683F002030
:106B6000DC84002030B585B004460D4601466846F9
:106B7000FFF7ECF9694604F13C0028F039FEC8B98A
:106B80004AF05AFB1B220A214AF0B2FA0D4B93F845
:106B9000A9329B0604D50C4A137843F00403137002
:106BA0002046FFF7C9F9094A04214CF0F7FB002001
:106BB00005B030BD2946204605B0BDE83040FFF79E
:106BC0008BBF00BFB85B0020DC8400201C810C0858
:106BD00030B585B004460D4601466846FFF7B6F964
:106BE000694604F13C0028F027FEC8B94AF024FBAE
:106BF0001B220A214AF07CFA0D4B93F8A9329B061E
:106C000004D50C4A137843F0040313702046FFF7B1
:106C100093F9094A04214CF0C1FB002005B030BDB6
:106C20002946204605B0BDE83040FFF755BF00BFFC
:106C3000B85B0020DC84002058810C087FB5054635
:106C40000E4605F13C0401466846FFF77FF96946A8
:106C5000204628F0F1FDC0B92046694628F0C8FD5D
:106C6000044690B94AF0E8FA1B220A214AF040FA99
:106C70000D4B93F8A9329B060FD42846FFF75CF919
:106C80000A4A04214CF08AFB04E031462846FFF70B
:106C900023FF0446204604B070BD054A137843F034
:106CA00004031370E9E700BFB85B002090810C0873
:106CB000DC84002030B5044685B00F4808F090F819
:106CC0000546B0B1072384F8903100230193029365
:106CD0000393E36801A9186877F0BCFAE3681868C1
:106CE000036801A95B680022984704480021FBF76C
:106CF00039FA284605B030BDB82B00200C8300209F
:106D0000F0B5424FD7F8382DD7F8343D2DED028B32
:106D10001343D7F8302D134387B005460C460CD1EA
:106D200048F096FD40F275124FF4801107B0BDECAB
:106D3000028BBDE8F04048F043BD806978F026FD45
:106D40002046B0EE408A10F053FC03283AD1EB689D
:106D500001A9186877F05AFB064698B3DDED017A71
:106D60006368009338EE678A294BDFED2A7A93F93E
:106D7000A8329FED290A2948002BA8BFB0EE670A68
:106D800038EE008A009BBDEEC88A002118EE102A5A
:106D90009342ACBF00930092FBF7E4F96B6918686B
:106DA00076F052FBDDED007A1D48B8EEE70A314679
:106DB00008F07EFE00212846FFF780FE07B0BDECFC
:106DC000028BF0BD94E80F0002AE86E80F00D7F802
:106DD000343D04936A46D7F8383D05930221304686
:106DE00010F012FC78B94AF027FA022215214AF075
:106DF0007FF9DDED037AF8EEE77A77EE887AFDEE3B
:106E0000E77ACDED007A0026AEE700BFB86B002030
:106E1000B85B0020000000000000C8420C83002086
:106E2000FC83002030B52DED028BC36887B004468B
:106E300018680D4677F0DEFA00284BD194F89021BF
:106E400000230093019302936AB93148039303A985
:106E50000493059308F05EFE28B1039B0093049B06
:106E60000193059B029394ED730A9FED2A8AE368D0
:106E7000DDED000A9DED011ADDED021A1868B4EE91
:106E8000C80AF1EE10FAAABFDFED237A9FED230ABC
:106E900020EE270A77F0ACFED4ED747AF4EEC87ACF
:106EA000F1EE10FA07DBE3689FED1B0A186827EE86
:106EB000800A77F035FAD4ED757AF4EEC87AF1EEFF
:106EC00010FA07DBE3689FED140A186827EE800AC2
:106ED00077F036FAE3682946186877F0B1FD054681
:106EE00088B10F4B1B68022B09D0032B03D10D4B2C
:106EF00093F995351BB10A480021FBF753F901219D
:106F00002046FFF7DBFD284607B0BDEC028B30BD05
:106F1000FC830020000000340000C8420000000094
:106F20000C830020B84B002010B52DED028BC368F8
:106F3000DFED348A1B684269D3ED0A0A9FED328A7D
:106F400093ED060AF4EEE80A0446F1EE10FA106832
:106F5000B8BFF0EE480A74F0C5FDE36862691B68CB
:106F60001068D3ED0A0A93ED060AF4EEE80AF1EE92
:106F700010FAB8BFF0EE480A74F02CFE6369186886
:106F800074F0BCFF18B96369186875F0F7FFE3681F
:106F900062691B68106893ED080A93ED0C1AD3ED33
:106FA000070AB0EEC00A74F0B7FFE36862691B68B5
:106FB000106893ED080A93ED0C1AD3ED070AB0EEB2
:106FC000C00A75F023F86369186875F0B9F818B944
:106FD0006369186876F038FA00210C48FBF7C2F8AC
:106FE0000B4861F0DBFB0B4AB2F8AA3223F4816351
:106FF000A2F8AA32BDEC028B20460221BDE8104067
:10700000FFF75CBD0000003400007A430C830020D1
:10701000207A0020B85B002010B50C4B0446D3F852
:107020006C0D90ED0B0A90F8502000F11C0176F0E9
:1070300059FE07480368022B02D00821FBF792F89B
:1070400020460521BDE81040FFF738BDB86B002091
:107050000C830020F0B52DED028B4A4DDFED4A8AFE
:10706000B0EE408A8FB00446D5F86C0D0E46174638
:1070700076F0AEFCF0EEC87AF4EEE87AF1EE10FAB3
:1070800007D49FED420AD5F86C0D28EE000A76F081
:1070900005FDD5F86C0D90ED0B0AB0EEC00A0FB1EE
:1070A000B1EE400A76F0EAFC0023D5F86C0D0793A8
:1070B00002AA07A90893099376F00CFDDFED347A54
:1070C0009DED027AB4EEE77AF1EE10FA56DD022277
:1070D00007A90AA810F068FD71680191304610F008
:1070E00087FA019902460AA810F058FAE3680AA93B
:1070F000186877F0A5FC10B92648FDF7B5F8A06927
:1071000078F042FB02684368D5F86C0D049303A93C
:107110001C30039224F0C0FC05A88DED050ACDEDCE
:10712000060A24F087FD1C4B1B68022B1BD0D5F8E8
:107130006C3D1948D3ED0A7AF4EEE87AF1EE10FAD4
:10714000B8BFD3ED047AF4EEC07AF1EE10FA4FF046
:10715000000110D5DFED117AB4EEE70AF1EE10FA76
:1071600009DDFBF71FF804212046FFF7A7FC0FB04D
:10717000BDEC028BF0BDFAF7F5FFF4E72046FFF710
:107180004BFFF4E7B86B0020000000340000C84259
:1071900000009643B82B00200C8300200000FA4327
:1071A00008B50748D0F8A03E9B0704D50121A0F5FB
:1071B0000050F7F703F8BDE80840024808F0D8BAD5
:1071C000B84B0020FC83002030B589B00446FEF7A0
:1071D0001DFA30B10021204609B0BDE83040FEF76D
:1071E0004DBA636A0221186879F08CFAE36818686E
:1071F00003685B69984701461048FCF721FF636903
:10720000186876F06FFA236A1D686369186875F06C
:10721000A7F805AC20460A498DED020ACDED030A18
:107220008DED041AFBF75CF9079B009394E80C00C2
:1072300002A9284672F060F909B030BDB82B0020D1
:107240000C83002038B50446FEF7E0F9054628B166
:1072500020460021BDE83840FEF710BA636A0221DB
:10726000186879F04FFA29462046BDE83840FEF705
:1072700051BE00000148002105F0FEBB0081002046
:1072800030B5174D9FED170A05F5804389B00446C8
:10729000D3F86C0D76F086FD01462846FCF7D0FE4B
:1072A0006369186876F01EFA236A1D6863691868B6
:1072B00075F056F805AC20460B498DED020ACDED70
:1072C000030A8DED041AFBF70BF9079B009394E872
:1072D0000C0002A9284672F00FF909B030BD00BFBA
:1072E000B82B0020000000000C83002030B589B0CE
:1072F0000446FEF78BF930B10021204609B0BDE805
:107300003040FEF7BBB9636A0221186879F0FAF9D8
:10731000E368186803685B69984701461048FCF702
:107320008FFE6369186876F0DDF9236A1D6863696A
:10733000186875F015F805AC20460A498DED020A6B
:10734000CDED030A8DED041AFBF7CAF8079B0093F5
:1073500094E80C0002A9284672F0CEF809B030BDBE
:10736000B82B00200C83002030B52DED028B83B0AC
:107370000446FEF74BF920B9636A1B6893F8CC30DA
:1073800043B90021204603B0BDEC028BBDE830407C
:10739000FEF774B994F89831DA071DD4E3681D68D4
:1073A0002B6828469B689847D5ED097A94F8983160
:1073B000B4EEE70AF1EE10FA4CBF0122002262F3AC
:1073C000000384F8983107D4204603B0BDEC028B4B
:1073D000BDE83040FFF7F8BE94F898319B0734D4ED
:1073E000E368DFED458A1B686269D3ED0A0A9FED09
:1073F000438A93ED060A1068F4EEE80AF1EE10FAFB
:10740000B8BFF0EE480A74F06DFBE36862691B6870
:107410001068D3ED0A0A93ED060AF4EEE80AF1EEDD
:1074200010FAB8BFF0EE480A74F0D4FB636918682C
:1074300074F064FD18B96369186875F09FFD94F8DD
:10744000983143F0020384F898312D4BD4F8A021F1
:10745000D3F8303D9B1A07EE903AB8EEE78AF1EE8A
:10746000047AB0EEC87AB4EEE77AF1EE10FA38D5C5
:1074700094F8983143F0040384F89831204684ED61
:10748000678AFEF731FC6369A26B1B68D2ED001AB4
:1074900093EDC61AD3ED0E0AB1EE480A21F030FF83
:1074A00063691B6840F2AA4093EDC31AD3EDC40A86
:1074B00021F044FC2046FEF773FB12488DED010AD3
:1074C00007F046FB63699DED010A186874F0AAFD98
:1074D0006369186803B0BDEC028BBDE8304076F0FC
:1074E00001B9D4ED677A68EE277AF5EEC07AF1EE4D
:1074F00010FAC3D5BCE700BF0000003400007A4397
:10750000B86B00204C5B002030B52DED028B83B0B2
:107510000446FEF77BF820B9636A1B6893F8CC3009
:1075200043B90021204603B0BDEC028BBDE83040DA
:10753000FEF7A4B86369DFED347A1B6894ED710A35
:1075400093EDC31AD3EDC40A20EE270A40F2C440DB
:1075500021F0F4FB2046FEF723FB236A186803683A
:107560009B6EB0EE408A9847284BB3F9643507EE1E
:10757000903AB4F8BC316425F8EEE77A13FB05F3D2
:10758000B4EEE70A07EE103A94F9BE31F1EE10FAC4
:10759000D8BFF0EE407A13FB05F39FED1D0AF8EE1D
:1075A000C76A07EE103AF4EE407AB8EEC77AF1EE09
:1075B00010FA58BFB0EE670A6846CDED006A8DED4F
:1075C000017A24F089FB236ADDED010A1868B4F81A
:1075D000C03102689DED000A126B13FB05F301EE4A
:1075E000103A0121B8EEC11A90476369B0EE480A1B
:1075F000186874F017FD6369186876F073F803B0C3
:10760000BDEC028B30BD00BF0000C842B84B00206B
:1076100000007A4430B590F8B83185B00446F3B133
:1076200068460FF0B5FF3F4869460AF0C3F950B10C
:1076300004F13C0028F0C8F8002384F8B83104F5C0
:107640009A7025F071FA94F890310A2B2DD8DFE862
:1076500003F0294B4F534B572C5B5F2C630000F515
:107660009A7025F061FA04F13C0590B194F840302D
:10767000012B0ED194F89031012B0AD1284627F026
:1076800011FF50B12046FEF757FC274A02214BF06C
:1076900085FE284627F034FFD5E72046FEF74CFC50
:1076A000224AF3E72046FFF77BFD94F844303BB9CC
:1076B00094F8463023B994F840309A1E534253410F
:1076C00094F8B92162B35BBB84F8B931184BD3F895
:1076D000B40203681B689847014616482D2205B07E
:1076E000BDE8304049F0BAB82046FFF76DFDDCE751
:1076F0002046FFF7A7FDD8E72046FFF7BBFDD4E7FC
:107700002046FFF7BDFDD0E72046FFF7EFFDCCE7B1
:107710002046FFF729FEC8E72046FFF7F5FEC4E73D
:1077200005B030BD10420020DC810C0804820C083A
:10773000B85B0020683F00202DE9F0412DED028B61
:10774000074684B008460E460FF052FF03288046D5
:107750006D4628D1FB68186876F0B2FC012822D16A
:107760002148294607F0D8F90446B0B17B69DDED20
:10777000007A1B68F8EEE77A93EDF27A77EEC77A33
:107780004246FDEEE77A17EE901AC829CDED007A51
:10779000B8BFC82130460FF001FF204604B0BDEC51
:1077A000028BBDE8F081114B0FCB85E80F0030460E
:1077B0000FF01EFF014628460FF082FF0446002806
:1077C000EBD07B69DDED017A1B68B8EEE78AD3ED7B
:1077D000F27A284638EE678A0FF00AFFBDEEC88AB3
:1077E000024618EE101AD5E7B82B0020E4780020E6
:1077F00010B543699FED126A1B68D3EDF06A93EDF3
:10780000F17AD3EDF27A86B066EE866A27EE067AD2
:1078100067EEC67A68460C46CDED006A8DED017ABA
:10782000CDED027A24F05CFC03A920468DED030A1D
:10783000CDED040A8DED051A10F0E6F906B010BD85
:107840000AD7233C30B5083204461D460FCA84E8E7
:107850000F00134301BFAB68A360EB68E36063688C
:1078600085B093B920460FF0C3FE03AA014628460F
:107870000FF0CAFE60B10399019120460FF0B8FEE7
:107880000199024620460FF089FE204605B030BD22
:10789000696801912846F1E730B50B6985B0044667
:1078A0000BB94B6953B30023C4F8B43108310FC985
:1078B0006D4685E80F0029462046FFF73DFF98B941
:1078C000124B0122D3F8301D28460FF067FE49F015
:1078D000B3FC0222152149F00BFC2046FEF72CFBDD
:1078E0000B4A02214BF05AFD29462046FFF79AFA2F
:1078F00010B90848FCF7B8FC05B030BD0123C0F84A
:10790000B43105B0BDE83040FFF70EBBB86B0020C6
:1079100038820C08B82B002070B51A4B04460E466E
:107920000FCB88B06D4685E80F0020462946FFF74B
:107930005FFFE368186876F05DFD98B1E36818684A
:1079400003681B69984768B1E3682946186876F0B0
:10795000C3FB38B947F07CFF40F295624FF48011C9
:1079600047F02EFF214604A82B463246FFF76AFF58
:1079700004A92046FFF756FA10B90348FCF774FC37
:1079800008B070BDE4780020B82B002070B5154B0E
:107990000C4606460FCB88B06D4685E80F00294699
:1079A0003046FFF725FF2B462246314604A8FFF755
:1079B00049FF6288A388122A4FEA132305D1227E49
:1079C000D20744BF03EB83035B00227A07EE903AB1
:1079D000C2F34002B8EE670A04A93046FFF73AFB4B
:1079E00008B070BDE478002038B504460D46FFF7B6
:1079F00093FF0023C4F89431AB88A4F8923138BDCA
:107A00007FB50D460446FFF787FF05F108010FC952
:107A10006E4686E80F00134306D1234BD3F8342D6E
:107A2000D3F8383D0292039304F5D0720121304619
:107A30000FF0EAFD94F8983170B923F0050343F094
:107A4000050384F898312046FEF776FA174A062196
:107A50004BF0A4FC04B070BD23F0070384F8983108
:107A60000023C4F89C31E36862691B68106893EDD9
:107A7000080A93ED0C1AD3ED070AB0EEC00A74F0B1
:107A80004BFAE36862691B68106893ED080A93ED8E
:107A90000C1AD3ED070AB0EEC00A74F0B7FA082149
:107AA0002046FFF70BF8D5E7B86B002064820C087E
:107AB0002DE9F0438DB06D4688461C4607461346B7
:107AC0000A4601462846DDE91469FFF7BBFE95E842
:107AD0000F0084E80F0007A80FF05AFDB8F8043033
:107AE000F3B9B8F80010013105AA89B207F13C00DA
:107AF00027F084F8A0B1234605AA39462846FFF7A7
:107B0000A1FE95E80F0086E80F00BDF81630A3F13E
:107B100052025342534189F800300DB0BDE8F08362
:107B200094E80F0086E80F000023F4E770B58B8817
:107B300092B004460D461646002B44D10DA80FF016
:107B400027FD298801310BAA89B204F13C0027F0F6
:107B500055F8002837D0BDF82E10132903D014D8BB
:107B60001039012913D833462A46214603A8FFF7C6
:107B700069FE03AB214607A80BAAFFF763FEE36883
:107B800007A9186876F09CFF01E0522901D012B0D5
:107B900070BD07AD03A80FF0FBFC28460FF0F8FC02
:107BA0000DF10B03CDE90053324603AB0BA9204680
:107BB000FFF77EFFE0689DF80B3000682A4603A9B6
:107BC00076F054FFE3E70120E1E7000070B5214BB8
:107BD00004460E460FCB88B06D4685E80F00204660
:107BE0002946FFF705FEE368186876F003FC98B1B4
:107BF000E368186803681B69984768B1E368294619
:107C0000186876F069FA38B947F022FE40F2166239
:107C10004FF4801147F0D4FD214604A82B4632468C
:107C2000FFF710FE04A92046FFF7FCF820B90A4828
:107C3000FCF71AFB08B070BD0023C4F89431B38878
:107C4000A4F8923104AA31462046FFF76FFF0028BE
:107C5000F0D1ECE7E4780020B82B0020F0B5324BEF
:107C600004460E460FCB91B004AD85E80F002046C8
:107C70002946FFF7BDFDE368186876F0BBFB98B1B5
:107C8000E368186803681B69984768B1E368294688
:107C9000186876F021FA38B947F0DAFD4FF4DF6260
:107CA0004FF4801147F08CFD0CAF08A80FF070FC6A
:107CB00038460FF06DFC0DF10F03CDE900732A4635
:107CC00008AB31462046FFF7F3FEE0689DF80F3021
:107CD00000683A4608A977F00FFA20B91348FCF774
:107CE000C3FA11B0F0BD0023C4F89431B388A4F8EE
:107CF000923108AA31462046FFF718FF0028EDD040
:107D00000B4B1B68022B09D0032B03D1094B93F9B2
:107D100095351BB106480021FAF744FA01212046A7
:107D2000FEF7CCFEDDE700BFE4780020B82B002092
:107D30000C830020B84B002037B504460D467FF079
:107D4000C7FEC4F8A801D5ED027AF5EEC07AF1EECF
:107D500010FA17DD9FED137A67EE877AFCEEE77A6B
:107D6000C4ED697A2046FEF7E7F8D4F8A4214FF471
:107D70007A73B2FBF3F30C4A062103B0BDE830403E
:107D80004BF00CBB5CF02EFD0023009395F90D2009
:107D900095F90E3095F90C105CF0C0FCC4F8A40104
:107DA000E0E700BF00007A447C820C0810B5B1F90E
:107DB0000A30A0F8BC3191F90C3080F8BE31B1F92D
:107DC0000D30A0F8C031B1F90F3007EE903AF8EE5F
:107DD000E77A0446C0ED717A7FF07AFE0A21C4F892
:107DE000C8012046BDE81040FEF768BE38B504461D
:107DF0000D467FF06DFEC4F8B001D5ED027A9FED1F
:107E0000047A67EE877AFDEEE77AC4ED6B7A38BDC7
:107E100000007A444A7C06480B46003A91F910105B
:107E2000D3ED030A93ED020A18BF0122FAF7C4B991
:107E30000C83002070B51B4E0446D6F8B4020368CC
:107E400086B01B680D469847042806D16B88102B16
:107E50000FD0732B20D000201CE0D6F8B4020368AA
:107E60001B6898470328F6D194F89031062BF2D17D
:107E7000ECE705F108010FC902ACDFED0B0A84E85D
:107E80000F00002309480093B0EE600A1A4621460D
:107E900002F028F906B070BD20462946FFF7BAFF68
:107EA0000120F7E7B85B002000000000A47F00205D
:107EB00038B5D1F8093007EE903AF5EEC07AF1EE18
:107EC00010FA05460C4605DD0B7A022B03D01ED9AD
:107ED000032B0ED038BD154B9FED150AD3F8640D5A
:107EE00027EE800A76F01CFAD4F80930C5F8D031B4
:107EF000F0E70E4B9FED0E0AD3F8640D27EE800AD3
:107F000076F01EFAD4F80930C5F8D431E2E7074B11
:107F10009FED070AD3F8640D27EE800A76F01EFA6B
:107F2000D4F80930C5F8CC31D4E700BFB86B0020D5
:107F30000000C84210B5044C237813B1034860F028
:107F400027FC207810BD00BFFC830020207A002091
:107F500013B5094B01910446D3F8640D03681B69FE
:107F6000984730B10199204602B0BDE81040FEF7B5
:107F700053BD02B010BD00BFB86B002090F898311F
:107F800013F0010018BFC3F380007047094A03468D
:107F900092F8850568B192F88425043A012A07D839
:107FA0005B6A1B6893F8A100431E58425841704712
:107FB00000207047B87B002010B504467FF088FD94
:107FC000D4F8B031C01AD4F8AC3123EAE373984244
:107FD0004FF0000084BFC4F8AC01012010BD0000C8
:107FE00010B503680446DB6D9847D4F8AC3123EA3A
:107FF000E37398424FF000003CBFC4F8AC0101208D
:1080000010BD000008B504480321FAF7ABF8BDE83D
:1080100008400148FAF792B90C83002070B51C4B58
:108020000446D3F8640D03681B690E46984705465D
:1080300010B90025284670BDD4F894315BB97FF0A3
:1080400047FDB4F89231C4F8940123B1114A537832
:1080500043F0010353707FF03BFDD4F89421B4F852
:108060009231801A4FF47A72B0FBF2F09842E0D36A
:1080700023B9084A537843F0010353702046FDF7B3
:108080005BFF3388044A06214BF088F9D2E700BF32
:10809000B86B0020DC84002008810C0810B590F833
:1080A0009031042B0446164B0AD1D3F8640D0368B3
:1080B0001B69984718B12046FEF7AEFF002010BD9F
:1080C0000A79D3F86C3DDFED0F6A93ED0E6A07EE87
:1080D000902A0A7E920748BF9FED0B7AF8EE677AE6
:1080E00048BF67EE877A86EE267AB0EEC77AB4EE9E
:1080F000E77AF1EE10FAACBF01200020DFE700BF05
:10810000B86B0020DB0FC9400000803B13B5094B62
:1081100001910446D3F8640D03681B69984730B198
:108120000199204602B0BDE81040FEF775BC02B0D0
:1081300010BD00BFB86B002010B504467FF0C8FC2E
:10814000D4F8A831C01AD4F8A43198424FF00000F6
:1081500084BFC4F8A401012010BD000038B5054655
:108160000C467FF0B5FCD5F8C831C01A23894FF40E
:108170007A725343984294BF0020012038BD00001A
:10818000C368186808B190F8B808704710B50121A5
:1081900004460A4803F0F0FF28B120460321BDE859
:1081A0001040FEF78BBC47F053FBBDE8104040F297
:1081B0006B124FF4801147F003BB00BF0081002019
:1081C00090F89031022B04D0032B04D1034803F024
:1081D000A3BF012070470020704700BF008100202E
:1081E00038B50C4BD3F8A05E90F89031032B0446C1
:1081F00005F004050AD1084803F0A6FF94F8903171
:1082000035B110B9023B5842584138BD0020F5E75E
:108210000120FAE7B84B00200081002010B50F4A7A
:10822000137843F0800313700D4B93F9A822002AB2
:10823000044609DBFEF73EFD70B920460822BDE882
:1082400010400921FDF74ABDBDE8104001220E2172
:1082500003F10C00F5F7BCBE10BD00BFDC840020AC
:10826000B85B0020F8B5D0F8B44105465CB1012CEC
:108270001AD047F0EDFA40F643024FF4801147F070
:108280009FFA012407E0184BD3F8640D03681B69BB
:10829000984710B900242046F8BD2846FEF744FE52
:1082A0000123C5F8B431F6E7104F97F9A832002B37
:1082B000F0DA436A1B6893F8A160012EEAD13C30E2
:1082C00026F0F2FC04460028E5D1D7F8D83293F81E
:1082D000CB3033B132460D2107F10C00F5F778FEB3
:1082E000D9E73446D7E700BFB86B0020B85B002061
:1082F00038B5674B03F5FA52D3F8B43293420446CB
:108300000D4601D0002095E04B885D2B74D8512B91
:108310002ED8103B9AB20F2A48D92046FDF70CFE02
:108320006B885C4A04214BF039F87CE0BC3B0D2B98
:10833000F3D801A252F823F027840108278401080A
:108340001B8301081B8301081B8301081B83010891
:108350001B830108278401081B8301082784010867
:108360001B8301081B8301081B8301082784010864
:10837000523B0B2BD1D801A252F823F07384010891
:108380001B8301083D840108518401081B830108F7
:108390001B8301081B8301081B8301081B83010841
:1083A0001B8301081B830108798401080F2BB4D8B3
:1083B00001A252F823F000BF4B8401080583010895
:1083C000598401085F8401086D8401085184010803
:1083D0003D8401081B8301081B8301081B830108DE
:1083E0001B8301081B8301081B8301081B830108F1
:1083F0001B83010865840108732B46D006D8702BB7
:1084000040D0722B89D1FFF7EBFD1AE04AF2CF6220
:10841000934234D081D8C92B0DD8BB2B86D8B23B20
:10842000012B3FF67AAF2046FDF786FD29884FF0F5
:10843000EBF8012038BDCF2BF5D06EE72046FFF7D3
:1084400079FD00283FF45EAFEDE7FFF7E7FDF8E7C1
:108450002046FFF707FFF4E7FFF720FEF1E7FFF7FD
:1084600077FDEEE7BDE83840FFF788BDFFF78EFDEA
:10847000E7E7FFF74BFEE4E7FFF75EFEE1E7FFF714
:108480006DFEDEE7FFF798FDDBE7FFF7BBFDD8E702
:10849000B85B00208C820C0890F89031032B0BD035
:1084A000062B06D0012B0AD1C368186803681B6825
:1084B0001847044801F008BA034803F0B7BE00208B
:1084C000704700BFA47F0020008100208B88012B13
:1084D00005D00B693BB94B692BB9CB681BB9044874
:1084E0000021FAF73DBA024800220831FAF75ABAD9
:1084F000B82B002010B54B885D2B04460A464BD89C
:10850000512B05D8103B99B20F291FD9002091E0BB
:10851000523B0B2BFAD801A151F823F06F860108CA
:108520000D850108298601083F8601080D8501088F
:108530000D8501080D8501080D8501080D850108CF
:108540000D8501080D850108778601080F2BDDD800
:1085500001A151F823F000BF3786010849860108C0
:108560005186010859860108698601083F8601087D
:10857000298601080D8501080D8501080D85010872
:108580000D8501080D8501080D8501080D8501087F
:108590000D85010861860108B32B76D016D8732BA0
:1085A00070D00ED8702B6AD0722BAFD1D1ED027A79
:1085B0009FED3A7A67EE877AFDEEE77AC0ED6B7A47
:1085C00037E0B22BA2D1FFF773FC32E0C92B23D8DE
:1085D000BB2B9BD9BC3B0D2B98D801A151F823F0A4
:1085E00033860108338601080D8501080D850108D1
:1085F0000D8501080D8501080D850108918601088A
:108600000D850108918601080D8501080D85010879
:108610000D850108918601084AF2CF6293427FF4EA
:1086200075AFFFF7C3FB04E002F108012046FEF737
:1086300067FB012010BD1146FFF7C8FAF9E71146A4
:108640002046FFF729F9F4E71146FFF765F9F0E74F
:108650001146FFF79BF9ECE71146FFF7C5F9E8E78C
:108660001146FFF7CDF9E4E7FFF790FDE1E711468A
:10867000FFF7F4FADDE71146FFF75EFBD9E7FFF7F6
:10868000B5FBD6E7FFF7C6FBD3E7FFF71FFFD0E741
:10869000034802F10801F9F72DFECAE70000C842BD
:1086A0000C830020704700007047000070470000F6
:1086B00090F8280080F0010070470000024B4360F2
:1086C00040F60503038170470001020490F855014C
:1086D000704700000F20704700207047002070474F
:1086E00000207047002070470048704738830C080E
:1086F0000048704744830C0808B5094800F500534A
:10870000D3F8F03EB3F9083000EE103AB8EEC00AE4
:10871000F5F7F8FEBDE808400248FDF741BA00BF92
:10872000B82B0020D07C002010B514482DED028B12
:108730001C4600F5005300F58040B3F96435D0F8CD
:10874000580D08EE103A036882B09B6ECDE9002107
:108750009847B8EEC88AF0EE400ADDE90021B0EE95
:10876000480A0748FCF76CFE0548FDF77BFA84EDE4
:10877000000A02B0BDEC028B10BD00BFB82B002078
:10878000D07C0020F8B51C4D05F5005405F5804659
:108790002846D6F8607DF5F7A3FEB4F9A03501EEC2
:1087A000103AB4F99E3500EE903A434200EE103A8A
:1087B000B8EEC11AF8EEE00AB8EEC00A384673F017
:1087C000ABFB2846D6F8606DF5F78AFEB4F9A03504
:1087D00001EE103AB4F99E3500EE903A434200EEB5
:1087E000103A3046B8EEC11ABDE8F840F8EEE00A9B
:1087F000B8EEC00A73F00ABCB82B002038B5124D91
:10880000124CD5F8580D03689B689847692100F110
:108810009402204647F0FAFCD5F8580D0368DB684F
:1088200098476A2100F19402204647F0EFFCD5F802
:10883000580D03681B6998476B2100F1940220468C
:10884000BDE8384047F0E2BCB86B0020683F00202C
:10885000014806F0C5BA00BFB82B00203C307DF0BF
:1088600011BD000008B546F0F3FFBDE808407222D4
:108870004FF4801146F0A4BF08B546F0E9FFBDE80B
:10888000084066224FF4801146F09ABF08B546F0C2
:10889000DFFFBDE8084080224FF4801146F090BF12
:1088A00073B51E4E0546D6F8B4020268126B9047A7
:1088B000044668B396F9A932002B2CDBD6F8D832DF
:1088C00093F8CB4024B396F8A83203F0A003202BF2
:1088D00021D1D6F8B402026812689047052808D062
:1088E000D6F8B402026812689047A0F110035C4207
:1088F0005C410B4A02F63C530193B3680093D2F8F3
:10890000603DD2F8582D214628467DF069FC04468A
:10891000204602B070BD0024FAE700BFB85B00201B
:10892000B86B00203C30FFF7BBBF000038B5114DDD
:1089300004461148F6F77CFA95F9A832002B14DAB0
:10894000236A93F8A120012A06D0D5F8B4020021A9
:10895000BDE83840FCF792BE0D2105F10C00F5F79B
:1089600037FB95F9A832002BEFDB2046BDE83840F5
:108970007DF072BFB85B0020B82B00203C30FFF7C1
:10898000D5BF0000012070470120704701207047CB
:108990000120704711207047012070470020704768
:1089A00000207047002070470048704788840C08FA
:1089B0000048704790840C0838B5436904461D6828
:1089C000806976F0E7FE23F0C5FFDFED1B0A28463D
:1089D00073F088F86369A0691D6876F0DBFE23F008
:1089E000B9FFDFED150A284673F0F4F863691868DB
:1089F00074F0C4FA6369DFED110A18689FED0E1A6E
:108A0000B0EE600A73F088FA6369DFED0C0A18684B
:108A10009FED091AB0EE600A73F0F8FA63691868FE
:108A200073F08EFB18B96369186874F00DFD0023AC
:108A30002364012038BD00BF00803B4400007A431E
:108A400070B52DED028B88B00446FCF7DFFD70B1E8
:108A500020460021FCF712FE63699FED310A186879
:108A600008B0BDEC028BBDE8704074F0C9BD636A0C
:108A70000221186877F046FE2A4B93F8A9325B066C
:108A800003D56369186873F0ADF89FED258A6069B6
:108A90008DED018A8DED028A8DED038A8DED048ABC
:108AA00003AA01A90068012373F006F96369186835
:108AB00074F07AFB236A1D682B68DE6C63691868A2
:108AC00073F04EFC0122CDED060A8DED071A05A9C3
:108AD0008DED050A2846B0EE480AB0476369B0EE4E
:108AE000480A186873F09EFA6369186874F0FAFD12
:108AF000236C8BB17EF0ECFFE36BC01A236C9842C1
:108B00000AD309480C220521FCF7F6FE20B90648D5
:108B10000C220221FCF7F0FE08B0BDEC028B70BD08
:108B200000000000B85B0020B82B002038B50446D8
:108B30000D467EF0CDFFC4E90F0538BD0720704714
:108B400001207047002070470020704701207047C7
:108B50000048704728850C080048704730850C088D
:108B600038B52DED028B002380F83C30C368DFED73
:108B7000338A1B684269D3ED0A0A9FED318A93ED6F
:108B8000060AF4EEE80A0446F1EE10FAB8BFF0EE79
:108B9000480A106872F0A6FFE36862691B681068F3
:108BA000D3ED0A0A93ED060AF4EEE80AF1EE10FAA4
:108BB000B8BFF0EE480A73F00DF8636920461D68EF
:108BC000FDF7BEF96368B3F93820B3F9363000EE2B
:108BD000903A434201EE102A00EE103AB8EEC11A64
:108BE000F8EEE00AB8EEC00A284673F095F963691A
:108BF00020461D68FDF7A4F96368B3F93820B3F97E
:108C0000363000EE903A434201EE102A00EE103A60
:108C1000B8EEC11AF8EEE00AB8EEC00A284673F0C2
:108C2000F5F9084BD3F86C0D75F078F80648082173
:108C3000F9F798FABDEC028B012038BD0000003432
:108C400000007A43B86B00200C83002030B52DED76
:108C5000048BC3689FED898A1B684269D3ED0A7A49
:108C6000DFED870A93ED060AF4EEC87AF1EE10FA0A
:108C70000446A8BFF0EE670A106889B072F032FFB0
:108C8000636920461D68FDF75BF96368B3F9382016
:108C9000B3F9363000EE903A434200EE103A01EE5E
:108CA000102A2846774DB8EEC11AF8EEE00AB8EE61
:108CB000C00A73F031F9D5F86C0D75F071F9A5F5AE
:108CC000805393F8CD32D90747D4D5F86C3D1A8B31
:108CD000D20742D593ED0A9AB4EEC89AF1EE10FA93
:108CE000B8BF93ED049AE36A186852F0D9FDD5F83D
:108CF000643DD3ED067AA36B20EE270AD3ED007A0C
:108D0000F0EE498AE0EE278AB0EE490AF5EEC08A15
:108D1000F1EE10FAD8BFDFED5C8AF0EE680A1FF0C2
:108D200009FF28B9D5F86C0DB0EE680A74F0B6FEEC
:108D3000636893F95130272B0FD0A36A186852F05B
:108D4000AFFDF0EEC07AF4EEC87AF1EE10FAB0EEB4
:108D5000407A20D5002384F83C30236B1B68B3F99C
:108D6000083000EE103A2046B8EEC00AFCF7AAFF21
:108D70002046FCF715FF2046B0EE408AFCF746FC83
:108D8000002848D00021204609B0BDEC048BBDE886
:108D90003040FCF773BCD5F86C3D9FED3C0AD3ED39
:108DA0000F7AD3ED0B6AA36B27EE800AF4EEC86A44
:108DB000D3ED007AF1EE10FA67EE277A10DB9FED23
:108DC000341ADFED310A552037EE800A1FF0B6FF66
:108DD000012384F83C30D5F86C0D74F04FFEBCE7ED
:108DE0009FED2C7AF4EEC76AF1EE10FA05D89FEDEC
:108DF000261ADFED290A5920E6E7F0EEE66AF4EEDE
:108E0000C86AF1EE10FAE3D594F83C30002B08BFA5
:108E1000B0EE670ADCE7636A0221186877F072FC3B
:108E20001E4805F095FEB0EE480AD5F86C0D74F0BA
:108E3000B9FF01461A48FBF703F96369186874F033
:108E400051FC236A1D686369186873F089FA05ACE0
:108E5000204614498DED020ACDED030A8DED041A6A
:108E6000F9F73EFB079B009394E80C0002A9284603
:108E700070F042FB09B0BDEC048B30BD0000003443
:108E800000007A43B86B002000000000E02E65422D
:108E90000000B442000000B40000B4C24C5B0020EB
:108EA000B82B00200C83002008B5064BD3F86C3D8E
:108EB000D868243022F0BEFEFCEEC07A17EE900A8D
:108EC00008BD00BFB86B0020024BD3F86C3DD868DA
:108ED00073F0F0BAB86B00200B2070470120704788
:108EE00000207047012070470020704700487047FD
:108EF000C8850C0800487047D0850C0801207047D1
:108F000008B5DFED237AF4EEE70AF1EE10FA2DED65
:108F1000028BF0EE408AB0EE608A35DDDFED1D7A1F
:108F2000F4EEE70AF1EE10FA2ED5F6EE007A70EEC6
:108F3000E77ADFED196A9FED190ADFED190AF0EE05
:108F4000E77A87EEA67A8720B7EE001A30EE470A56
:108F50001FF0F4FEDFED137A9FED131ADFED130A15
:108F600020EE270A8A2020EE280A1FF0E7FE30EEC6
:108F7000080ABDEC028BDFED0A0ABDE808408D202F
:108F8000B7EE001A1FF0DABE9FED050AEFE700BF4B
:108F9000AC1C5A3ED578493F8FC2753E9A99993F8D
:108FA00000000000FAEDEBBA9A99993E9A9999BEA1
:108FB00030B52DED048B7D4BB3F9643500EE903A5E
:108FC000F8EEE00A83B0044601AA6946B0EE600AF2
:108FD000FCF736FAA06976F0DDFBE369D0ED008A94
:108FE000D3ED946AD3ED977A90ED016AA3689FED73
:108FF000701ADFED700A27EEE80A68EEA68A03F61B
:109000009403E6EE278A05463B20DFED6B7AB0EE4F
:10901000E87AB4EEE77AF1EE10FA58BFB0EE677A6C
:10902000DFED667AC7EE275AF7EE007A77EEE57A3B
:109030009DED007A67EE877A93ED007A67EE877A86
:109040009FED5F7AA6EE260A87EE879A1FF076FEDE
:109050003C209FED571ADFED570AB0EE408AB0EE84
:10906000680A1FF06BFE626B564B1268DFED567A92
:10907000B2F90820D3ED006A9FED541ADFED540ACF
:1090800007EE102AB8EEC77AF0EE408A27EE277A6C
:10909000DFED507AA6EEA77A4520F4EE007AA7EE2F
:1090A000678ABAEE000A28EE000A83ED007A8DED99
:1090B000000A1FF043FEDDED017A9FED477A474B32
:1090C0008DED000AF0EEE77AF4EEC77AF1EE10FAD1
:1090D00051D593ED007ADFED427A77EE277AB2EE42
:1090E000007AF4EEC77AF1EE10FA58BFF0EE477A44
:1090F000C3ED007A67EEA87ACDED017A636A18684D
:1091000090F8CB10002939D177F0FCFA636A1B681C
:1091100093F8A110012939D0032940D039B9236A25
:10912000186870F0D1FE236A186870F01DF9236A80
:10913000DDED010A18689DED000A0368B0EE491ADA
:10914000DB6A9847204695ED028AFCF775FB2046BE
:10915000F0EE400AB0EE480AFFF7D2FE236A6268DA
:109160001868D2ED020A036801215B6E984703B0CC
:10917000BDEC048B30BD00221A60BFE7194B93F998
:10918000A932002BB4BF01210221BDE7236A186870
:1091900070F09AFE236A186870F0FCF8C7E7D97976
:1091A0000029C4D12046FCF7C1FEC0E7B84B00201F
:1091B00000000C4400000CC40000FA4400409C4530
:1091C000000034425C8300200AD7233D00A08C4578
:1091D00000A08CC58FC2753F000000346083002062
:1091E0008FC2F53CB85B00200E207047002070470E
:1091F0000020704700207047002070470020704713
:109200000048704768860C080048704768860C085C
:1092100070B52DED028B436A1B6893F8CB30044682
:10922000FBB9052384F848302046FCF705FB636A48
:1092300002211868B0EE408A77F064FA94F9503051
:10924000E2696BB3D2F8F8515D4394F84820052ADF
:109250004FD8DFE812F02B005F008400B100DF0080
:109260001E01836A1B68B3F90830002BB8BF5B424C
:109270009BB2B3F57A6FD4D2C36A1B68B3F90830D6
:10928000002BB8BF5B429BB2B3F57A6FC9D27EF0B8
:109290001FFCE36CC01A40F6C4139842C1D8C3E760
:1092A00094F95150D2F8FC215543CEE7226A94F943
:1092B000511010689FED801A49F6404253435143C4
:1092C00000EE103A00EE901A0268F8EEE00A926B97
:1092D000B8EEC00A9047DFED797A41F293139D42D0
:1092E00038EE278A05DD94F950308BB1012384F8DC
:1092F0004830236A62681868D2ED020A0368B0EE4B
:10930000480ABDEC028B5B6EBDE870400021184737
:109310000223ECE7226A9FED681A106849F6404282
:10932000534300EE103A0268B8EEC00A926BF0EEBA
:10933000410A9047DFED627A38EE678A05F50C55F1
:10934000B5EEC08AF1EE10FA05F1270543F2BA43F3
:10935000D8BF9FED598A9D42CBD80423C7E7236A23
:109360009FED551A186894F9513049F6404253431D
:1093700000EE903A0268F8EEE00A926BB0EE410A15
:109380009047DFED4F7AE36938EE678AD3F8F8311A
:10939000B5EEC08AF1EE10FAD8BF9FED478A002BD8
:1093A000B8BF5B4242F228329342A2DD41F29413ED
:1093B0009D429EDD03239AE7236A9FED3F1A1868BA
:1093C00094F9513049F64042534300EE903A026816
:1093D000F8EEE00A926BB0EE410A9047DFED387A82
:1093E000E36938EE678AD3F8F831B5EEC08A03F541
:1093F0000C53F1EE10FA03F1270344F24E62D8BF8A
:109400009FED2D8A93423FF674AF2E4B9D42FFF69F
:1094100070AFA2E7236A94ED111A1868D4ED100A10
:10942000036894ED0F0A1B6B00219847DFED237A48
:1094300094F95020E36938EE278A1AB393ED7E7AC7
:10944000D4ED0F7AB8EEC77A77EEC77A9FED1E7A21
:10945000F0EEE77AF4EEC77AF1EE10FA3FF649AF94
:109460000D2294F849101948FCF746FA024618B93B
:1094700001461648FCF740FA47F0DEFE162147F099
:1094800017FE36E793ED7F7AD4ED107AB8EEC77AFF
:10949000DAE70D2294F849100C48FCF72DFA024641
:1094A00018B901460948FCF727FA47F0C5FE022221
:1094B0000D2147F01DFE1CE700000000CDCC4C3E06
:1094C0008FC2753E6DEEFFFF0000FA43B82B0020FF
:1094D00073B5474D0446D5F8B40203685B6B9847F3
:1094E00018B90026304602B070BD95F9A932002B9C
:1094F0005FDBA36A1B68B3F90830002BB8BF5B427F
:109500009BB2B3F57A6FECD2636A1B6893F8CB60B9
:10951000002EE6D095F9A832002BE2DBD5F8B40294
:1095200003681B689847002584F8490084F8485070
:109530007EF0CEFAE36AE064A4F850501B68B3F9F9
:109540000830B3F5967F43DD012384F8513047F0AE
:1095500073FE152147F0ACFD264BB3F9643501EEDF
:10956000103AE369B8EEC11A93ED7E0A8DED011A47
:10957000F1EE410A5320B8EEC00ACDED000A1FF00B
:10958000DDFBE36984ED0F0A93ED7F0A9DED011A7F
:10959000DDED000AB8EEC00A54201FF0CFFBE369EE
:1095A00084ED100AD3ED807AF8EEE77AC4ED117AF3
:1095B00098E7D5F8B40203681B689847012890D053
:1095C000D5F8B40203681B689847002891D188E752
:1095D00013F5967F01DAFF23B7E7A36A1B68B3F997
:1095E0000830002BACBF0123FF2384F85030AEE7D6
:1095F000B85B0020B84B0020042070470120704762
:1096000000207047012070470048704700870C0811
:109610000048704708870C08012909D0232907D082
:10962000042905D0034BD3F8A40E00F001007047C5
:1096300001207047B84B0020C36B23B990F841005C
:1096400080F001007047002070470000034BD3F802
:10965000A40E80F00400C0F380007047B84B0020D7
:10966000012380F84230184670470000002380F83C
:10967000423001207047000070B52DED028BC368A9
:109680000446186890F9BB3886B0B0EE408A0BB338
:1096900090F8BC68F6B174F013FD01281AD1274880
:1096A00019213FF04BFC07EE900AF8EEE77AF4EE52
:1096B000C87AF1EE10FA0DDD214BB3F9063F07EE43
:1096C000903AF8EEE77AF4EEC87AF1EE10FA18DB89
:1096D000002012E01B4B0FCBFDEEC87A02AD85E8EF
:1096E0000F0017EE901A012228460DF057FF01AA2D
:1096F000022128460DF088FFE8B906B0BDEC028BC8
:1097000070BDBDEEC88A8DED018A002529460E4840
:10971000E563F8F727FD6369186873F095FEDDEDE2
:10972000017A0A48B8EEE70A314606F0C1F984F832
:1097300041500120E1E70026E7E700BFB83C0020E8
:10974000B84B0020E47800200C830020FC8300202C
:1097500010B52DED048BC2689FED149A1268436911
:10976000D2ED0A0ADFED128AF4EEC90AF1EE10FA20
:109770000446B8BFF0EE680A1868B0EE408A72F08E
:10978000B1F9E268636912681868D2ED0A0AF4EE6A
:10979000C90AF1EE10FAB8BFF0EE680AB0EE480A56
:1097A00072F018FABDEC048B012010BD00000034EB
:1097B00000007A4313B5C36842691B68F0EE400AA3
:1097C00093ED080A93ED0C1ACDED010A0446B0EEB4
:1097D000C00A106872F0A0FBE36862691B68106839
:1097E00093ED080A93ED0C1ADDED010AB0EEC00A04
:1097F00072F00CFC012002B010BD000010B52DED80
:10980000028BC36842691B68044693ED0C1AD3EDC2
:10981000070A1068B0EE408A72F07EFBE368626966
:109820001B68106893ED0C1AD3ED070AB0EE480AD6
:1098300072F0ECFBBDEC028B012010BD1FB5C36BB9
:10984000022B0BD0032B1DD0012B22D1C36818682B
:109850000368DB6805B05DF804EB1847806975F0B4
:1098600093FF0D4B59689A6802911B68019301A9F7
:10987000039220F099FAFDEEC07A17EE900A05B037
:109880005DF804FB4369186805B05DF804EB72F0FD
:1098900011BE0020F3E700BF98830020C36B012BAB
:1098A0000AD003DC2BB19FED070A7047023B032B64
:1098B000F9D84369186802E0C3681B68186972F038
:1098C00081BE00BF0000000030B5C26B012A89B024
:1098D0000C4604D0022A0AD0002009B030BDC3686B
:1098E000186803681B6809B0BDE8304018470B4B87
:1098F000586899681B680193094B02901B78039183
:10990000002B04AD18BF032201A928460EF04CF924
:1099100095E80F0084E80F000120DEE7988300201F
:10992000DC8300207FB5C36B022B0FD0032B23D029
:10993000012B25D1C368186803689B689847BCEE63
:10994000C00A10EE100A07B05DF804FB806975F0DC
:109950001BFF0D4B014658689A6804901B680393DF
:1099600003A8059222F098F801A88DED010ACDED2B
:10997000020A22F05FF9E2E7436918682430F8E749
:109980009FED020ADDE700BF988300200000000081
:1099900010B52DED028B01239FED1C8AC363C368B4
:1099A000044684B018688DED018AF0EE480AB0EEE6
:1099B000481AF0EE481AB0EE480A8DED028A8DED95
:1099C000038A75F015F9E3688DED018A8DED028A41
:1099D0008DED038A186801A974F03CFCE3681868EF
:1099E000036800225B6801A9984730B945F030FF51
:1099F000BB224FF4801145F0E3FE05480021F8F743
:109A0000D1FB04B0BDEC028B10BD00BF0000000014
:109A10000C83002030B589B00446FBF7F7FD70B128
:109A20001D4805F037FD014618B1636A1B6893F8BD
:109A3000CC10204609B0BDE83040FBF71FBE636A7A
:109A40000221186876F05EFEE368186803685B69B7
:109A5000984701461048FAF7F3FA6369186873F0FB
:109A600041FE236A1D686369186872F079FC05ACD1
:109A700020460A498DED020ACDED030A8DED041A48
:109A8000F8F72EFD079B009394E80C0002A92846E6
:109A90006FF032FD09B030BDB82B00200C830020E0
:109AA00010B52DED028BC368DFED298A1B68426972
:109AB000D3ED0A0A9FED278A93ED060AF4EEE80A31
:109AC0000446F1EE10FAB8BFF0EE480A106872F0E2
:109AD00009F8E36862691B681068D3ED0A0A93ED20
:109AE000060AF4EEE80AF1EE10FAB8BFF0EE480A02
:109AF00072F070F8E36862691B68106893ED080AF9
:109B000093ED0C1AD3ED070AB0EEC00A72F004FA16
:109B1000E36862691B68106893ED080A93ED0C1AFC
:109B2000D3ED070AB0EEC00A72F070FA63691868E4
:109B300073F08AFC6369186873F020FA0648002104
:109B4000F8F730FB054B00221A70BDEC028B10BDFC
:109B50000000003400007A430C830020DC830020E6
:109B60000223C363FFF79CBF0523C363FFF798BFBE
:109B70000423C363FFF794BF10B50446FFF7F8FF53
:109B8000074A0023936053601360064A9360536052
:109B90001360002384F8403084F84230012010BD67
:109BA000A4830020B08300200323C363FFF778BFA2
:109BB00030B50623C363C36842691B6893ED080A86
:109BC00093ED0C1AD3ED070A044685B01068B0EE89
:109BD000C00A72F0A1F9E36862691B68106893ED2E
:109BE000080A93ED0C1AD3ED070AB0EEC00A72F022
:109BF0000DFA6369186872F0A3FA18B963691868F6
:109C000073F022FC7DF064FF0C4D0346284601A949
:109C100040F8043B236A1B6800245B6F03930194A4
:109C2000029421F07FFB0023EC61AC616C616C62FB
:109C30002C6285F82C3005B030BD00BF6883002051
:109C4000024BD3F8A40EC0F3C0007047B84B0020FD
:109C50002DE9F0432DED028B9946C36B274C062B63
:109C600085B080460E461746B0EE408A36D0FFF7E4
:109C70009FFF96E80F00224D85E80F0097E8070048
:109C8000103585E8070084F82D900023B9F1000F06
:109C900030D084ED0A8A63627DF01AFF03AB206046
:109CA00002AA01A9304621F06FFC94ED092ADFEDEC
:109CB000157AD4ED0A1A9DED031ADDED020A9DED29
:109CC000010AD8F83C10104822EE272A3A46F7F746
:109CD000E5F905B0BDEC028BBDE8F083B9F1000FEA
:109CE000C7D194F82D30002BC3D04369186873F0A6
:109CF000ABFBBEE7A36284ED098ACDE76883002051
:109D00006C8300200AD7233CB82B002038B50B4DBC
:109D10000446284605F02CFD2B786BB194F84130B1
:109D200053B90123064884F841305AF0D7FEBDE804
:109D3000384004485EF02CBD38BD00BFFC830020D5
:109D400020500020207A002070B52DED028B88B0C5
:109D50000446FBF75BFC054680B1294805F09AFBF9
:109D6000014618B1636A1B6893F8CC10204608B00E
:109D7000BDEC028BBDE87040FBF780BC636A9FEDD1
:109D8000218A1868022176F0BDFC60698DED018A98
:109D90008DED028A8DED038A8DED048A2B4603AA90
:109DA00001A9006871F088FF63698DED008A186869
:109DB0000368B0EE480A2A4669465B6898476369BB
:109DC000186873F0F1F96369186873F08BFC236A03
:109DD0001D682B68DE6C6369186872F0C1FA012295
:109DE0008DED050ACDED060A8DED071AB0EE480A95
:109DF00005A92846B04708B0BDEC028B70BD00BF76
:109E0000B82B002000000000A1B1DFED0F7A20EE9A
:109E1000270A33B1DFED0D0A0D4801220021F8F7C2
:109E2000CBB922B160EEA70A0948F8F743BADFEDD3
:109E3000070AF9E722B10648B0EE600AF8F776BAE9
:109E40000348F8F7AFB900BF0AD7233C0000000071
:109E50000C8300202DE9F0432DED028B8BB00446DE
:109E6000164606A802220F461D46B0EE408AF0EEC6
:109E7000608A0DF099FE284806A95AF0F1FF804645
:109E800058B947F0D9F90522162147F031F9404673
:109E90000BB0BDEC028BBDE8F083E36B032B02D06B
:109EA0002046FFF781FE9DF858309DF854209DF81C
:109EB0005010F0EE680AB0EE480A2046FFF7A4FF03
:109EC0007DF006FE154BD7F800901860144BD7F8BC
:109ED00004E0D7F808C0134AC3F80090C3F804E0C0
:109EE000C3F808C00023137096E807000E4F0F4E0A
:109EF000CDF80C9087E8070095E8070086E8070092
:109F0000CDE90076E16B0A48CDF810E003AACDF860
:109F100014C0F7F77FF8BAE72050002064830020D0
:109F200098830020DC830020A4830020B0830020DD
:109F3000B82B002010B588B000240594069407942F
:109F40009DF82C4002949DF82840CDE9003405ABE3
:109F5000FFF780FF08B010BD2DE9F04F2DED028B0B
:109F60008FB091469DF86C709DF868B0002F14BFBB
:109F70000322022204460AA80D46B0EE408A9A4601
:109F8000F0EE608A0DF010FE4D480AA95AF068FF05
:109F9000064658B947F050F90522162147F0A8F8AF
:109FA00030460FB0BDEC028BBDE8F08F454AE36B45
:109FB000D2F8A42E12F0400F0DF11C082AD0012B6C
:109FC00002D02046FFF7E4FC5B46F0EE680A5246FA
:109FD000B0EE480A49462046FFF716FFE3681868C6
:109FE00003683A465B682946984700230493059323
:109FF000069307930893099304AB0093CDF804806C
:10A000003B462A46E16B3048F7F704F8012384F811
:10A010004030C5E7022B02D02046FFF7A1FD002FFC
:10A0200049D0E3684146186874F0F0F940B92268F5
:10A0300003905268012120469047039B1E46AFE7DC
:10A04000224B1B782BB963699DED070A186872F0E3
:10A050002BF952464946DFF874A0DFF884905B463E
:10A06000F0EE680AB0EE480A2046FFF7CDFE2968F8
:10A070006A68AB68164D8AF80070164F29606A60EE
:10A08000AB600023BB607B603B60C9F80830C9F857
:10A090000430C9F800307DF01BFD0F4B6A68296859
:10A0A0001860AB680892CDE90079099307919AF896
:10A0B00000304246A6E763699FED080AC6E700BF85
:10A0C00020500020B84B0020B82B0020DC8300205B
:10A0D00098830020A48300206483002000000000F7
:10A0E000B08300202DE9F0472DED028B8EB00446A1
:10A0F0006F489DF860A00E469046B0EE408A9946A3
:10A10000F0EE608A5AF0ACFE054658B947F094F874
:10A110000522162146F0ECFF28460EB0BDEC028B5E
:10A12000BDE8F087634BD3F8A43E590648D5E36BEE
:10A13000012B02D02046FFF72BFCE368314618685C
:10A1400074F07EFC054618B947F076F80222E0E785
:10A1500053464A46F0EE680AB0EE480A41462046A9
:10A16000FFF752FED6ED027AE16B0391F8EEE76A53
:10A17000D6ED037ACDED056AB8EEE77AD6ED017A31
:10A180008DED067AF8EEE77A3046CDED077A0DF0E0
:10A190002FFA00220BAB089209920A920B920C92B2
:10A1A0000D920193C21E08AB009303995342534191
:10A1B00005AA4148F6F72EFF012384F84030ABE7AB
:10A1C0000027E068089709970A97006805AB08AA76
:10A1D000314674F0F5FB054600289DD0E36B022B59
:10A1E00002D02046FFF7BCFC5346F0EE680A4A4610
:10A1F000B0EE480A41462046FFF706FE9DF81430AF
:10A20000002B50D0E3680BA9186874F0FFF8804663
:10A2100030B9236801215B682046984745467BE7B3
:10A22000264B1B782BB963699DED0B0A186872F0F9
:10A230003BF8234B089A1A60099ADFF89080DFF800
:10A2400090905A60DFF874A00A9A9A609DF81430D2
:10A250008AF80030C8F80870C8F80470C8F80070B0
:10A26000C9F80870C9F80470C9F800707DF030FCB6
:10A27000D6ED027A134BE16B1860F8EEE76AD6ED83
:10A28000037ACDED0B6AB8EEE77AD6ED017A8DED63
:10A290000C7ACDE90089F8EEE77A9AF80030CDED36
:10A2A0000D7A0BAA85E763699FED070ABEE700BF39
:10A2B00020500020B84B0020B82B0020DC83002069
:10A2C000988300206483002000000000A483002005
:10A2D000B08300202DE9F0470E4611461A46C36BA5
:10A2E0008AB0052B9DF84C9005460DD0CDED050AA2
:10A2F00004928DED030A0291FFF736FCDDED050AAD
:10A30000049A9DED030A0299184C194F9DF84830A4
:10A31000DFF868A0DFF868802846FFF775FD0023A6
:10A320000022A36063602360BB607B603B608AF8AF
:10A33000002096E8070088E807007DF0C9FB0D4B78
:10A340001860B9F1000F0ED06268A3682168079108
:10A3500008920993CDE900789AF80030E96B064835
:10A3600007AAF6F757FE0AB0BDE8F08798830020E9
:10A37000A483002064830020B82B0020DC8300200D
:10A38000B08300202DE9F0470F461946C36B8AB011
:10A39000042B9DF85090054616460BD0CDED050ACE
:10A3A0008DED040A0391FFF7E3FBDDED050A9DED5A
:10A3B000040A03991A4C9DF84C309DF84820DFF8A8
:10A3C00070A0DFF870802846FFF71EFD0023A36011
:10A3D0006360236000238AF8003097E8070088E86C
:10A3E000070096E807000F4F87E807007DF070FB35
:10A3F0000D4B1860B9F1000F0ED06268A368216898
:10A40000079108920993CDE900879AF80030E96B2B
